:020000040800F2
:1000000000000120BD170508591805084DB9010861
:10001000A1B7010859180508591805080000000083
:100020000000000000000000000000005918050852
:1000300059180508000000005918050881C8000873
:1000400059180508591805085918050859180508B8
:1000500059180508591805089D9E0008A59E000816
:10006000AD9E0008B59E0008BD9E0008959C000846
:10007000A99C0008BD9C0008D19C0008E59C0008D4
:10008000F99C00080D9D0008591805085918050825
:10009000591805085918050859180508C59E00087B
:1000A000B9BF0008B5BE0008C9BF0008A5BE00085A
:1000B000DDBE0008EDBE0008FDBE0008B5980008D2
:1000C000A9980008E9980008DD9800085918050863
:1000D00059180508615A04086D5A0408795A040829
:1000E000CD9E00085918050859180508D9BF000801
:1000F00091BF00085918050881BF0008219D00081C
:1001000059180508591805080DBF000859180508A1
:10011000855A0408915A04081DBF000879E90408AB
:10012000359D0008499D00085D9D0008719D0008EF
:10013000859D000800000000000000000000000095
:10014000000000000000000000000000A589040875
:10015000999D0008AD9D0008C19D00089D5A0408A6
:100160001D99000811990008591805085918050823
:100170005918050859180508000000000000000083
:100180005918050859180508591805085918050877
:1001900059180508591805080000000059180508E5
:1001A00000000000000000000000000059180508D1
:1001B0005918050859180508000000000000000043
:1001C000000000000000000000000000000000002F
:1001D00000000000000000000000000059180508A1
:10800000084A0346D0F8E4005268D3F8F010121A78
:1080100000209142B8BFC3F8F020012283F81C2150
:10802000704700BF001000E030B4046900234168CD
:108030004025E46882690C3154624469956053605C
:1080400093631160C2E90333C2E90533C2E9073320
:10805000C2E90A33C2E90C3394B1C2694FF48030EB
:10806000E468116054629062C2E90133C2E90333EB
:10807000C2E90533C2E90733C2E90B33C2E90D3364
:1080800030BC7047114A037A0168D35C10B4CC58F5
:10809000CA1824F00104CC501368DB07FCD4037D1C
:1080A0001F2B09D9203B20225DF8044B02FA03F371
:1080B00043F01803CB60704720225DF8044B02FAAE
:1080C00003F343F018038B60704700BF70B90508D5
:1080D0001B4B016803F57D7C02E02C3363452BD0FC
:1080E0001A688A42F9D170B593F804E0427996454E
:1080F0000BD02C33634505D01A688A42F4D02C3358
:108100006345F9D14FF0FF3070BD9E468468002270
:10811000DEF80C50A54208D001320EF10C0E032AF5
:10812000E7D0DEF80C50A542F6D1DEF81050C66854
:10813000B542F1D150B270BD4FF0FF30704700BF73
:10814000203705084368426D30B49A61EFF311821D
:10815000502383F312884168D2B2856C0B68046D9A
:1081600023EA050323430B6082F311884369816886
:108170001A68096822F00102D0E908541A60826A7C
:108180001D605C615A60D0E90B429C60DA6000239C
:10819000B0F86C2030BCCA6203777047002A4FEAFF
:1081A000014C034630B508BFE64600F1C00514BFD8
:1081B0008E468C46002419680C3353F8042C43F87F
:1081C000084C41EA0C0142EA0E02AB4243F80C1C97
:1081D00043F8042CEFD1D0F8C03043EA0E03C0E9D5
:1081E0003144C0F8C03030BD83695969B3F810C05C
:1081F0000A6830B49C6822F0010224680A60E268D0
:1082000022EA0C02E260027D00681F2A06D9203AA9
:108210000824456894402C4242D0FEE708240568B3
:1082200094402C42F9D1202404FA02F28260254ABB
:108230001278002A32D01A7F012A36D0D3F80021D2
:108240000132C3F80021EFF31181502282F312882A
:108250005868C9B29D6C0268DC6C22EA05022243B0
:10826000026081F311885A699968D3E90D40096861
:1082700014605061D3E90F40546090605C6CB3F8B7
:10828000B400D4600124C8621068204310601A8AC8
:108290001C7783F8FD40CB681343CB6030BC70473C
:1082A000202404FA02F2C260C1E70022D3F80401DC
:1082B00083F8FD2001300A68C3F8040122F00102AE
:1082C0000A60EBE7A801002010B40C4C6368002B97
:1082D00011DD002004F1080C0146DCF8AC3003F19C
:1082E000C00259600C339342FBD1013063680CF536
:1082F000867C8342F1DC5DF8044B7047A8010020C6
:10830000704700BF024B03EB401393F855047047CE
:10831000A8010020D0E90920131A5842584170479B
:1083200090F8573830B53BB990F85518012490F8BB
:108330005638DAB2914200D830BD04FA03F2B0F8F0
:108340005E5801332A43A0F85E28F2E7037902461B
:1083500013F0010006D0D2E90731D2685B1A013A66
:1083600003EA0200704710B50379044613F00103D5
:108370000ED0FFF7EBFF034650B1226A6369E16854
:108380009B5C0132B2FBF1F0DBB201FB10222262F6
:10839000184610BD03799B070AD5436A8269D154F8
:1083A000436A02690133B3FBF2F102FB113343620A
:1083B00070477047017170470379014613F002005E
:1083C00007D00B69D1E90921013B521A1A40D2B2F8
:1083D000981A704710B584464FEA810E102312F4A4
:1083E000004F4FEA420214BF0E240724013B92B211
:1083F000CCF80040F444F2D100EB81128C0103511F
:10840000122042F8213010BD10B584464FEA810E8B
:108410000424130B013C4FEA021203EB430392B214
:1084200003F11803CCF80030F444F2D100EB01134F
:108430000A018450062043F8214010BD704700BF58
:10844000704700BF00EB4000024B03EBC00393F802
:1084500049057047A8010020064B93F8F825824291
:1084600006D900EB400003EBC003D3F84C0570477E
:1084700000207047A80100200B4890F8FC1589B136
:1084800001EB4101002300F5A760490010B41C4630
:1084900050F82320063302B114608B42F8D15DF806
:1084A000044B7047704700BFA80100200B4890F8AC
:1084B000FC1589B101EB4101002300F5A7604900DB
:1084C00010B41C4650F82320063302B114608B42CE
:1084D000F8D15DF8044B7047704700BFA801002039
:1084E000214B1B78002B3DD12DE9F0431F4C94F814
:1084F000FC25AAB304F5A7624FF0500E1C4F4FF0B5
:108500002C0C1C4E1D4607E0013394F8FC1552F864
:10851000180B8B42056023DA117C0029F4D05068D7
:108520004FF0FE08810AA1F580115229314498BF0D
:1085300091F8F483EFF311818EF31288D0F8249030
:108540000CFB0878C9B209F10109C8F82890D0F8E5
:10855000148048F00108C0F8148081F31188D3E733
:10856000BDE8F083704700BF00000120A801002093
:10857000401901202037050800EE100AB8EE400A25
:10858000704700BFBCEEC00A10EE103A98B27047B8
:1085900007280AD800EB8000054B03EB4013B3F823
:1085A0000006B0FA80F0400970470020704700BF15
:1085B000A8010020072807D8044B00EB8000012207
:1085C00003EB401383F80226704700BFA801002088
:1085D000072808D8044B03EB401393F8542412B136
:1085E000012283F83A247047A8010020072808D800
:1085F000054B03EB4013B3F83804B0FA80F04009A0
:1086000070470020704700BFA8010020054B93F879
:10861000F825824204D903EB4013D3F84404704791
:1086200000207047A80100200346012200205A774D
:10863000704700BF826908B50346006BD96A0244DF
:108640009A6101B18847002008BD00BF436A024615
:108650001B681B6A5B685B7813F0010008BF5077EA
:10866000704700BFC2628161704700BF704700BFA2
:10867000043070470C4B93F89822D3F894120244BC
:108680000144D2B2C3F8941283F8982293F8982246
:10869000120605D593F8982282F0800283F898227A
:1086A000024B01225A70704740190120000001203E
:1086B0002DE9F84F164FD7F89C52ED0A23D000262B
:1086C000DFF850A007F52879B0467419D7F8A01242
:1086D0004FF01003524648BF0134D1F828B0484645
:1086E000C7F8CC826410E102D8470F280BDD094B94
:1086F00003F1100153F8042B013207D18B42F9D159
:108700002546B542E1DCE802BDE8F88F661CF8E7D3
:108710004019012000000020194BD3F8D412D3F8DF
:10872000D8228A1A322A05DCD3F8EC228A1A002AC7
:1087300011DC7047D3F8DC1249B193F8E82288883D
:1087400002F001020968120100FA02F28A610022B5
:10875000C3F8EC227047D3F8DC226AB110683231DA
:10876000928810B44469C3F8EC1222425DF8044BBD
:1087700018BF1204826170473231C3F8EC1270479F
:1087800040190120074AD2F8DC324BB192F8E822B6
:108790009988186802F001031B0101FA03F3836151
:1087A0000020704740190120044B4FF4007C00204A
:1087B000D3F8F832A2F800C00B60704740190120CE
:1087C000002070470120704701207047002070474B
:1087D000134BD0F8D8105B68D0F8E02010B50446F1
:1087E000581A824200DC22B9D4F8E4200A44C4F8C2
:1087F000DC2094F8D020C4F8D830012A05D0D4F871
:10880000D4300133C4F8D43010BD04F1E801201D88
:108810003CF00CFDD4F8D4300133C4F8D43010BD92
:10882000001000E0CB070DD430B590F828308DB0A3
:10883000C468012B07D0B4F1807F01D901230377ED
:108840000DB030BD7047194B456AD3E9CA13B1EB7F
:10885000930F4FEA93024FF0020306D252085B00D7
:1088600091429BB201D2FF2BF8D9B4F1807FAB804B
:10887000E6D90122002301A9B724027728460492F1
:108880008DF814208DF828208DF804400B93CDE945
:10889000021302A9CDE90633CDE908333CF0C6FC4A
:1088A0002A68136A002BFCD1CAE700BF40190120D7
:1088B00030B590F828308BB00446012B08D0407FAB
:1088C00010B901200BB030BD002363770BB030BD71
:1088D000456A2B681A7B22BB637F002BF1D01349BA
:1088E0000220002301220290081D8DF80C208DF833
:1088F00020200993CDE9001069462846CDE90433CC
:10890000CDE906333CF092FC2A68136A002BFCD1B7
:10891000074B5B7DD84303F0010300F00100637750
:10892000D4E71B6A002BD7D00020CBE71000002033
:108930000000002030B504468BB094F82830012B9D
:1089400008D0637F0BB10023637701200BB030BDEB
:108950001B6A23B1656A2B681A7B002AF8D1637FF2
:10896000002BF2D010490220002301220290081DA2
:108970008DF80C208DF820200993CDE90010694670
:108980002846CDE90433CDE906333CF04FFC2A6894
:10899000136A002BFCD1054B5B7D03F00102DB0762
:1089A0006277D2D5C9E700BF100000200000002088
:1089B000214A002330B5044695B0101D1F4D069383
:1089C000019002200B931093139311930290207F38
:1089D00000920495CDE90E3301238DF80C300793F6
:1089E0008DF820308DF834308DF8483002F10803CE
:1089F000083A0593031D0A920C93114B0993636A7D
:108A00001A68136A002BFCD1A0B10E480A0E00F1BF
:108A10001A0342760A0A9970080C69465A7018704F
:108A2000606A3CF003FC636A1A68136A002BFCD18D
:108A300015B030BD044BEDE7200000204D86000846
:108A400029860008000000201900002010B594B00D
:108A500004465022074968464AF048FA6946606A67
:108A60003CF0E4FB636A1A68136A002BFCD114B073
:108A700010BD00BF683B0508F8B50546406A0068B0
:108A8000046A002CFCD12C7FA869002C36D0234E20
:108A9000040E052786F82D402E36B0704FEA104C94
:108AA000000A1F4C86F800C0012B70704FF00000C8
:108AB0000E68676326641668A6642E63A06520D0DE
:108AC000022B1AD15368012220651E444968E365D0
:108AD000144B84F84C0061652E6384F86020636653
:108AE000114B6A7FA3F11401686A002A08BF194676
:108AF0003CF09CFBEB6A5BB1286BF8BD04270B4E86
:108B0000CBE7084A84F84C306065E0652265E7E70A
:108B10006B6A1A68136A002BFCD1EDE70000002095
:108B20000000012035860008180001202D000020DB
:108B300000B583B08161019201A9049A00930123D9
:108B4000C2626A46FFF798FF03B05DF804FB00BFFE
:108B500070B51D46436A94B006461B681C6A002C1B
:108B6000FCD1314B0B9203F13C0230480694009249
:108B700003F14002049003F13400019202220590B7
:108B8000029201228DF820408DF80C208DF83420BF
:108B90008DF84820327F0C95101D1394CDE90944BF
:108BA000CDE90E44CDE910440790002A3AD00A0ED0
:108BB000363303F8012C0A0C99701D4C090A1A70FF
:108BC0005970706AD4E9CA32B3EB920F4FEA92013E
:108BD0004FF0020206D2490852008B4292B201D2F3
:108BE000FF2AF8D9737F8280D3B169463CF01EFB1F
:108BF000706A03681A6A002AFCD10222D4E9CB34D5
:108C0000B4EB930F4FEA930106D2490852008C420D
:108C100092B201D2FF2AF8D98280284614B070BDE2
:108C200005A9E3E73533C6E7000000204D860008BC
:108C3000401901208269F0B592F8DC308BB005460E
:108C4000012B27D0023B012B2FD892F84C31EC4658
:108C5000D2F89C2063F07F03154C13708669D6F818
:108C6000A0305F1C0FCCACE80F00D6F89C30CDE9EB
:108C700000370FCCACE80F0094E803008CE8030049
:108C8000694606F110003CF0D1FAAA6911690B6A35
:108C9000002BFCD1D2F8A0305A8852BAEA819A88C7
:108CA00052BA2A82DB885BBA6B8201200BB0F0BD1E
:108CB000B83B0508F0B590F8DC308BB00446D0F82E
:108CC000A060012B4BD034D9023B012B2ED890F859
:108CD0004D31EC46D0F89C2063F07F03434D137078
:108CE000D0F8A0305F1C0FCDACE80F00D4F89C305A
:108CF000CDE900370FCDACE80F0095E803008CE814
:108D00000300694604F110003CF090FA2269136AEE
:108D1000002BFCD173885BBAA4F8D030B3885BBA5F
:108D2000A4F8D230F3885BBAA4F8D43001200BB099
:108D3000F0BDD0F89C304FF0FF3205211A605A6028
:108D40009A60DA60D0F8E030C0F8F010B3F57A7FBE
:108D50001FD8032380F8DC3001200BB0F0BD90F861
:108D60004C2190F84D319B1A5B100133DBB236F881
:108D7000132006EB430653BAA0F8D03073885BBAD1
:108D8000A0F8D230B3885BBAA0F8D43001200BB081
:108D9000F0BD03691A7B2AB35B691BB390F8983066
:108DA00003B390F84C310122D0F89C0063F07F03AC
:108DB000C4F8A4400E49037094F84D3194F84C0166
:108DC00084F800211B1A84F8DC20D4F8A020073393
:108DD000C4F804110132D4F89C10C4E93E23C4F84D
:108DE000F410A3E7022384F8DC309FE7B83B0508C2
:108DF00001800008F8B50C4B1D685A691540054004
:108E00005D617DB1094F0126B5FA85F4C4F11F04F7
:108E100007EB840306FA04F4D3F834030368984795
:108E2000A543F1D1F8BD00BF003C0140401901202D
:108E300002692DE9F843C36812EA030828D0054601
:108E40000E464FF00047B8FA88F327FA03F21B3BAF
:108E5000D24308EA02082A61042B16D8DFE803F09F
:108E60003B30251A0300B36A002B3FD003F1FF39D2
:108E700000231FFA89F9B362746A34B1236820466B
:108E8000494698476468002CF8D1B8F1000FDAD150
:108E9000BDE8F88370680028F7D0696B036889B271
:108EA0009847B8F1000FCED1F2E7B0680028ECD0B7
:108EB000A96B036889B29847B8F1000FC3D1E7E7FF
:108EC000F0680028E1D0E96B036889B29847B8F1EF
:108ED000000FB8D1DCE730690028D6D0296C0368D0
:108EE00089B29847B8F1000FADD1D1E7EB6A1FFA0C
:108EF00083F9C1E72DE9F041DFF8B48008EB4017B2
:108F000097F854340BB9BDE8F08104460D4646018C
:108F10004AF0AAFBC0BB2448464400EB4410A6F824
:108F200038544AF0D1FB98F80030D6F85024A3B159
:108F3000D6F83C140124D2F8AC308C4003F1C001C7
:108F4000420010F4004F90B202D15A6822435A6096
:108F50000C339942F4D1BDE8F081D6F83C140124D9
:108F6000D2F8AC3001F1100203F1C001944042008C
:108F700010F4004F90B202D15A6822435A600C3369
:108F80008B42F4D1BDE8F081084B93F8D42302EB77
:108F9000420203EBC203234493F88153002DBAD05D
:108FA000012387F83A34B6E7E00500204019012094
:108FB000A801002010B5044649F0C0FA0146204639
:108FC00089B2BDE8104095E738B50B4D00EB400085
:108FD00005F5A763C40003EBC003254493ED027AB3
:108FE000D3ED037AE7EE007AB0EE670A49F0A6FA0D
:108FF000D5F83835186038BDA8010020836910B550
:109000001A4C04EB8303D3F8F8033DF00BF9B4F8E2
:1090100018340C2B0ED8DFE803F0220D0D0D1B0DBC
:109020000D0D070D0D0D1400D4F8D823D36823F4CB
:109030000063D3600122002384F8152484F81A34D5
:1090400010BDD4F8D823D36823F48053D360F1E75C
:10905000D4F8D823D36823F48063D360EAE7D4F844
:10906000D823D36823F40073D360E3E740190120C9
:1090700080699C303DF0D6B8F8B5A0F50764237937
:10908000DB0725D5657994F8543805F001073D468E
:10909000FBB1D4F848341A68D36A5B08536294F879
:1090A000583823B1B4F862380133A4F8623885F037
:1090B0000101606C42F0B8FB012384F857380023AB
:1090C00084F8553884F85638A4F85E3884F8543853
:1090D000F8BD94F85768012E03D194F8553884F8F8
:1090E00056382046FFF71CF94EB9012385EA0301E3
:1090F00084F85738606CBDE8F84042F095BB002317
:10910000394684F85738F5E770B505460726084C08
:10911000013E00D170BD94F900001BF085FA031EDA
:1091200004DB6178EA189171A278EA540434EFE71D
:10913000E03B050838B58569002D3DD02C68236AD1
:109140001B7B5BBB204647F0F7FD236A5B6803B3DC
:10915000236A5A68236A22F01F025968236A01F0C1
:109160001F019B681F33194421F01F01BFF34F8F6C
:1091700000290ADD02F12003114410488B42C0F897
:109180005C221A4603F12003F8D1BFF34F8FBFF3DF
:109190006F8F2846BDE838403CF0F6B9AB68002B2D
:1091A000D0D01A6820469B88936147F0C5FD236A9A
:1091B0005B68002BCCD1ECE738BD00BF00ED00E0D0
:1091C00038B5846904B938BD2568284647F0B4FD30
:1091D0002B6A1B7B23B92046BDE838403CF0D4B94C
:1091E000A368002BF7D01A6820469B889361BDE8DE
:1091F00038403CF0C9B900BF2DE9F843DDF82080C4
:109200000F4616460021202204461D4649F0C6FEA0
:10921000B8F1000F0CD0D8F80030B8F80A20E3817C
:109220001B0C2382D8F804306282E3821B0C238358
:10923000384647F0DBFDF30619D4431EB8B107EBFF
:10924000000C01E0013B12D31CF801EDBEF12E0F22
:10925000F8D1C01A03F10109421EB944032AA8BF7C
:109260000322082BA8BF082390461A4606E00828C8
:109270000246B9464FF00008A8BF08224FF020333D
:10928000394620462360636049F030FE164B04F1F6
:109290000800424649462381837049F027FE611E3B
:1092A000E21D11F801CFACF16103ACF1200C192BD8
:1092B00098BF81F800C09142F3D104F10A0011F87F
:1092C000013FA3F16102203B192A98BF0B70814234
:1092D000F5D1182365832D0CE6722373099BA582B3
:1092E000E361BDE8F88300BF202020002DE9F04FA6
:1092F000DFF8509485B0D9F8D402C9F8D802002B11
:109300005ED00C46154601F5FE7603EB020B1DE020
:10931000002D62D0D9F80433AB4200F0C580D9F8F3
:109320000033AB4200F0F780D9E9C231AB424BD8F1
:109330008D42C0F07281691A204642F0F5F801357D
:1093400004F5007406F500765D4539D0D9F8102390
:10935000AA42DDD8AA1AD9F82073D308396B02F0D3
:10936000070802338B4202D3BA6B93420BD93946BA
:109370001846039342F0A8F8039B0746002800F024
:109380006C81C9F820033A79002A40F01D81D7F892
:1093900028A0BAF1000F00F059813A6B0135204640
:1093A0004FF400719B1AFA6804F5007406F5007614
:1093B00008EBC3083B4602EB4822D0475D45C5D1C8
:1093C000002005B0BDE8F08F8D42B4D24FF400729A
:1093D0000021204649F0E2FDB1E74FF40072294632
:1093E000204649F0DBFD8023CA4A84F8BE310C23B5
:1093F00084F8C231D9F80013D9F8F8329142C4F890
:10940000C611C4F8CA3100F30D81C34A013BC34FF2
:1094100082FB0102C81787FB01C70A44C0EB621236
:10942000C0EB2730BE4F87FB02C7C2EB821C84F81B
:10943000C1018010A1EB0C01174420F03F00013165
:109440000843D117C1EBE71184F8C0010A4484F83E
:10945000BF21B04A934200F3F180AF4AAF4882FB8C
:109460000312D91780FB03701A44C1EB6212C1EBDF
:109470002031AB4880FB0270C2EB821784F8C51123
:109480008910DB1B104421F03F0101331943D3172E
:10949000C3EBE01384F8C4111A4484F8C3214AF6DC
:1094A0005523A4F8FE314AE74FF0FF3300274FF46D
:1094B000F072201D84F8EC31394684F8ED3184F8DF
:1094C000EE3184F8EF315223237063706123A3706F
:1094D00084F8E7314123E37084F8E631722384F89D
:1094E000E43184F8E531D9F81833C4F8E83149F0AB
:1094F00055FD5523C4F8F07184F8FE316FF0550323
:10950000C4F8F471C4F8F87184F8FC7184F8FD7142
:1095100084F8FF3113E74FF400720021204649F030
:109520003DFD804B022203CB45F6EB0322742273F0
:1095300023809023A273A370F82384F82C200822A0
:10954000C4F803006273C4F807106375D9F80013F8
:10955000D9F8F8325B1A2362D9E9C2135B1A4AF6CA
:10956000552163620023E372E3736377A377E377A4
:1095700084F82D3084F82E3084F82F3084F8313080
:10958000694BA3613E232377012384F83030802385
:1095900084F84030654BC4F84230654B84F846206F
:1095A000A4F8FE11634A03CBC4F84B101988C4F821
:1095B00047009B78A4F84F1084F8513003CAC4F8D0
:1095C0005200C4F85610BAE64FF40072002120464B
:1095D00049F0E4FC3B6CB8F1000F45D104F1200ADE
:1095E000002B00F081803B6B112253492046CDE9CE
:1095F0000088FFF701FE3B6C1A6C002A00F08180A6
:109600001B6B504611224D49CDE90088FFF7F4FD50
:1096100004F1400A4FF4E07871E0E91A204641F085
:1096200083FF8CE6FF22013B84F8C1214FF6FF72D5
:10963000A4F8BF21374A93427FF70FAFFF2384F886
:10964000C5314FF6FF73A4F8C33128E751464FF4F4
:109650000072204649F0A2FC71E6231F384A43F805
:10966000042F9E42FBD16AE6002B7F6C14BF0223BD
:109670000123C3EB0813002F3FF461AE013BBF6C25
:10968000002B01DD002FF9D1A2464FF40078002F06
:109690003FF455AE0AEB080303959A460BE000250C
:1096A000A8F12008CDE900E5FFF7A6FDBF6CCFB11A
:1096B000B8F11F0F16D93D7907F11C0E1122396838
:1096C0003B6BAAEB0800002DE9D17A79A8F12008BC
:1096D0003D6942F02102CDE900E5FFF78DFDBF6C49
:1096E000002FE5D1039D2AE6CDE9008843464FF4DB
:1096F000F0780822D9F8FC122046FFF77DFD7F6C38
:10970000C5E75046434611220C49CDE90088FFF7D2
:1097100073FD7DE7FF03FB008320088297554541D9
:1097200081808080BCB805083F00FF0029940E0DA1
:10973000C8B80508D4B80508B4B80508B8B805080D
:10974000DEADBEEF4019012048B182884FF00043E2
:109750000349B2FA82F20868D34003430B607047B2
:10976000003C014010B490F8443000F10801484A30
:10977000012BC2F81C146DD08368464CD968A342F3
:1097800021F46001D960D96841F46001D960996B16
:1097900021F440119963996B41F480119963996B9D
:1097A00021F4F8419963996B41F488419963996870
:1097B00021F47021996099689960996821F44011A9
:1097C000996099689960596821F480615960596875
:1097D00021F48051596059696FF30B01596159693E
:1097E000596148D0D9682B4C21F0E061A342D9607F
:1097F000D96841F0E061D960996B21F44011996317
:10980000996B41F480119963996B21F478219963E4
:10981000996B41F410219963996821F47021996042
:1098200099689960996821F44011996099689960E4
:10983000596821F480615960596821F48051596058
:1098400099696FF30B019961996999611AD00023A5
:1098500080F844301048114B848DC18D408D091B18
:10986000C2F82444C2F820045DF8044B93FBF1F3E2
:10987000C2F828347047D4F8041341F40001C4F846
:109880000413AFE706494B6843F400034B60DEE77F
:109890004019012000200140007AF01F80380100AB
:1098A00000230140704700BF01483CF08FBD00BF5E
:1098B000801D0120084810B4D0F84034D0F874441A
:1098C00099691A682CB1234600F588605DF8044B4D
:1098D00018475DF8044B70474019012001483CF0DF
:1098E00075BD00BFE01D0120084810B4D0F8A034B9
:1098F000D0F8D44499691A682CB1234600F59460D5
:109900005DF8044B18475DF8044B7047401901207F
:1099100001483CF05BBD00BF401E0120084810B468
:10992000D0F80035D0F8344599691A682CB123462F
:1099300000F5A0605DF8044B18475DF8044B7047D4
:1099400040190120F0B506688C680F68B569002FD2
:1099500056D02E4B3B40B3F1005F4FD007F01F0CA9
:1099600004F11F0327F01F029C442CF01F0CBFF3CF
:109970004F8FBCF1000F0BDD944402F12003DFF8A0
:1099800090E06345CEF868221A4603F12003F8D12F
:10999000BFF34F8FBFF36F8F02684FF480636B612B
:1099A00053696F602C6243B34B68F56963B31E461D
:1099B000164B3340B3F1005F1AD006F01F0226F0B9
:1099C0001F011F32224422F01F02BFF34F8F002AD3
:1099D0000ADD0A4401F120030D489342C0F87012D9
:1099E000194603F12003F8D1BFF34F8FBFF36F8FF8
:1099F0004FF480636E606B612C62F0BD3246CCE741
:109A00003B463246034FCAE7034EF3E70000FFFF31
:109A100000ED00E044000020480000202DE9F04166
:109A20000468D4E904351A7DD3E90061002D4DD0D6
:109A30001F2AA86138D820202F6800FA02F242F0CD
:109A40001802B2602A7D1F2A39D9203A202000FA54
:109A500002F242F01802FA606A68002008601060A2
:109A60003046116841F01001116093F80880A26936
:109A7000414645F013FE2D7AE2693846294645F005
:109A80000DFE274B626813F80800595D335843F008
:109A9000010333507B5843F001037B50536843F07C
:109AA00003035360BDE8F081203A20202F6800FABC
:109AB00002F242F01802F2602A7D1F2AC5D8202047
:109AC00000FA02F242F01802BA60C5E71F2A986154
:109AD0001ED8202000FA02F242F01802B2600022E2
:109AE00030460A600A6842F010020A601D7AA269D4
:109AF000294645F0D3FD0A4B6268595D735843F01F
:109B000001037350536843F002035360BDE8F081D2
:109B1000203A202000FA02F242F01802F260DEE75A
:109B200070B9050810B1036882889A61704700BF58
:109B300018B1838802681B0493617047D3B2012B6C
:109B40001DD802EB42020F4B10B54FEA820E03F50F
:109B5000217C0EF1080402E01C3363450DD01A7815
:109B60008242F9D15A788A42F6D11A59002AF3D0A2
:109B70000EF1040E03EB0E0010BD002010BD0020FE
:109B8000704700BFF83B050810B40C4C002304F2EA
:109B9000AC5C01E0152B0CD003EB430201331CF845
:109BA00002108142F6D1144494F9AE055DF8044BDD
:109BB00070474FF0FF305DF8044B704740190120AB
:109BC000D3B2022B21D802EB420270B54FEA820ECB
:109BD0000F4C002223460EF10C0503E001322C331A
:109BE000172A10D01E68B042F8D193F804C08C45F3
:109BF000F4D15E59002EF1D02C210EF1080301FBA7
:109C00000233E01870BD002070BD0020704700BF17
:109C100020370508002838D0002330B51B4D90F8B8
:109C200004C005F2AC5401E0152B2CD003EB430229
:109C30000133A15C6145F7D11544046890F805E053
:109C400095F9AE35DAB2022A1DD803EB430310486A
:109C500000224FEA830C03460CF10C0503E00132AD
:109C60002C33172A0FD019688C42F8D11979714515
:109C7000F5D159590029F2D02C210CF1080301FB30
:109C80000233184430BD002030BD70474019012018
:109C9000203705080348D0F88C300BB17C301847CA
:109CA000704700BF000001200348D0F8B0300BB16E
:109CB000A0301847704700BF000001200348D0F8CB
:109CC000D4300BB1C4301847704700BF00000120EA
:109CD0000348D0F8F8300BB1E8301847704700BFA0
:109CE000000001200348D0F81C3113B100F5867044
:109CF00018477047000001200348D0F8403113B1E5
:109D000000F5987018477047000001200348D0F80C
:109D1000643113B100F5AA701847704700000120A4
:109D20000348D0F8883113B100F5BC70184770476C
:109D3000000001200348D0F8AC3113B100F5CE701B
:109D400018477047000001200348D0F8D03113B104
:109D500000F5E07018477047000001200348D0F874
:109D6000F43113B100F5F27018477047000001207C
:109D70000348D0F8183213B100F502701847704745
:109D8000000001200348D0F83C3213B100F50B70FD
:109D900018477047000001200348D0F8603213B123
:109DA00000F5147018477047000001200348D0F8F0
:109DB000843213B100F51D70184770470000012070
:109DC0000348D0F8A83213B100F526701847704741
:109DD0000000012001380D4B0D4A00EBC000116B53
:109DE00003EB800310B4DB6F83B00A4CA34214BFB3
:109DF0004FF480034FF4001319431163126B1340A7
:109E00000193019B03B05DF8044B704700000120F3
:109E100000380240006002400138F8B500EBC00095
:109E2000114C1D46114B04EB800417460E46E06FA3
:109E3000984214BF9620952042F06CFD94F9910051
:109E4000B909C4F88C60C4F8945042F025F994F92B
:109E50009130002B07DB03F01F0001225B0904494E
:109E6000824041F82320F8BD00000120006002403C
:109E700000E100E0800AA0F58010522808D8054BC8
:109E8000034493F8F4330D2B02D8034AD05670479D
:109E9000002070472037050860B905080120FEF74B
:109EA000A9BF00BF0220FEF7A5BF00BF0420FEF738
:109EB000A1BF00BF0820FEF79DBF00BF1020FEF726
:109EC00099BF00BF4FF47870FEF794BF4FF47C4009
:109ED000FEF790BF30B1036882881B691A4214BF35
:109EE00001200020704700BF2DE9F04F0E4683B0DF
:109EF00004461546002800F0C7800268644B1344EE
:109F00009B0A644AC6F34119134493F85C0742F074
:109F100001FDC6F38103B4F804E006F003012468F0
:109F200001939EFAAEF0B0FA80F001F1FF383EFAEC
:109F300000F367D001220327009603E001303EFAC8
:109F400000F35ED002FA00F313EA0E03F6D0D4F861
:109F500000C093FAA3FBBBFA8BFB93FAA3FABAFAFD
:109F60008AFA4FEA4B0BB8F1010F4FEA4A0A07FA97
:109F70000BFB01FA0AFA2CEA0B0C4CEA0A0CC4F8A7
:109F800000C04ED9D4F80CC093FAA3FBBBFA8BFBEC
:109F900093FAA3FABAFA8AFA4FEA4B0B02294FEA6C
:109FA0004A0A07FA0BFB09FA0AFA2CEA0B0C4CEAEC
:109FB0000A0CC4F80CC0C1D193FAA3FABAFA8AFA0F
:109FC0004FEA132CBAF1070F45DCD4F820C093FAFE
:109FD000A3FABAFA8AFA93FAA3F34FF00F0BB3FA83
:109FE00083F34FEA8A0A01309B000BFA0AFA05FA5A
:109FF00003F32CEA0A0C4CEA030323623EFA00F353
:10A00000A0D1009EB8F1010F08D86268C6F3001312
:10A0100022EA0E020EFB03F31343636003B0BDE8B4
:10A02000F08FD4F808C093FAA3FBBBFA8BFB93FA2A
:10A03000A3FABAFA8AFA4FEA4B0B019E4FEA4A0A90
:10A0400007FA0BFB06FA0AFA2CEA0B0C4CEA0A0C8C
:10A05000C4F808C096E7D4F824A09CFAACFBBBFA7D
:10A060008BFB9CFAACF34FF00F0CB3FA83F34FEA7F
:10A070008B0B9B000CFA0BFC05FA03F32AEA0C0A83
:10A080004AEA0303636259E74FF0FF3339E700BF41
:10A090000000FEBF2037050800B125E770472DE915
:10A0A000F84FBB4F6023064603FB0073D3F82C44E4
:10A0B000D3F83484D3F83854002C00F05D81B8F123
:10A0C000000F04D098F90630002B40F0558125B1DF
:10A0D00095F90630002B40F04F81731CDBB2B8F1CC
:10A0E000000F04D0152288F8073088F8062015B133
:10A0F0001622EB71AA714FF0600A207E42F00AFC32
:10A1000029460AFB06FA404646F0ACF9404607EB02
:10A110000A09042240F2145899F83C34002B0CBF71
:10A120004FF01E0B4FF03E0B5946FFF7B5FF284688
:10A13000984D042259465544FFF7AEFF4C220021AA
:10A14000284648F02BFFD9F82C349FED937AB0EED7
:10A15000084A5B68F7EE003AB9F83EA44FF0000CED
:10A16000C9F840348D4B9FED8E5A9A688D4BC2F3DF
:10A170008222134493F86427D7F82C33D34007EE98
:10A18000903AF8EE677AC7EE275A07EE90AA9FED4D
:10A19000867AF8EEE77AC7EE274ADFED847AB0EEEA
:10A1A000007AE5EE877AA5EE875A25EE844A37EEE7
:10A1B000856A74EEE72ABAF5C87F0CF1010ED5BFA7
:10A1C0004FF4967278226423322307EE90EAD8BFC8
:10A1D0004FF416791344A2F13202F8EEE76AC8BFD1
:10A1E0004FF4827907EE903AD4BF41464FF4FA71AA
:10A1F00066EEA56AB8EEE77AC7EE267A07EE102A71
:10A2000001EB0902B8EEC77A37EE447A77EEE37ACB
:10A21000FCEEE77A17EE903AC7EE267AFCEEE77A84
:10A2200017EE900A07EE909AB8EEE73A07EE902AFA
:10A23000F8EEE77A23EE243A83EE277A37EE453AB2
:10A2400032EEC77AC3EE267A77EEE37AFCEEE77A4F
:10A2500017EE901AC7EE267A77EEE37AFCEEE77AED
:10A2600017EE902A02F1020909EB010BB0EE467AD3
:10A2700007EE90BAF8EE677AA6EEA77AF4EEC74A30
:10A28000F1EE10FA7CDC43EA00095FFA89F9B9F1D2
:10A290000F0F77D841EA02091FFA89F9B9F1FF0FC8
:10A2A00070D81B05000403F07F6392B200F47F00B6
:10A2B00003433F4843EA0C7300EA01210B43134375
:10A2C0006022284602FB06760027C6F844340123A4
:10A2D000C6F84874C6F84C34C6F85074C6F85474BE
:10A2E000C6F85C74C6F8607445F0C6FB96F8813415
:10A2F000202BD9B21AD196F88034012B16D0242302
:10A3000086F88134D6F840341A6822F001021A60C7
:10A310001A6822F480521A601A681A601A6842F0A9
:10A3200001021A6086F8811486F88074002194F97D
:10A330001A0041F0B1FE94F91A20A37E002A08DB2E
:10A340005909012203F01F0302FA03F3194A42F8E4
:10A350002130002194F9190041F09EFE94F9192052
:10A36000637E002A08DB5909012203F01F0302FA69
:10A3700003F3104A42F82130BDE8F88FF4461AE79B
:10A38000013171E7BEF10F0FF8D1002398E700BF4C
:10A3900040190120801D0120286B6E4E00380240BC
:10A3A000000016432037050800247449000070425D
:10A3B00000FFFF0000E100E008B1002294E57047D3
:10A3C00070B50E4C94F8F865AEB104F587640025BD
:10A3D00003E001352034B5420DD0237F002BF8D0A7
:10A3E000E06800220028F4D00135217DFFF77CFDD4
:10A3F0002034B542F1D1012070BD00BFA80100207A
:10A4000070B590F8B2311C09013C052C0FD81A4EDA
:10A41000054603F00F0306EB4402B2F86C0740FA5E
:10A4200003F2D20703D595F8B521012A01D0012006
:10A4300070BD9A402644013A104048F05FFF96F8FC
:10A4400078370E4A034402EBC30452F83320A38842
:10A4500010691840ECD0002395F8B3210221204662
:10A4600085F8B531FFF740FDD5F82021136843F09A
:10A4700008031360DBE700BF203705082C1F01200D
:10A48000014B53F82000704750280040014B43F81F
:10A490002010704750280040204B2148196C214A59
:10A4A00041F0805130B482B01964196CFF2401F07E
:10A4B000805101910199016841F480710160CA20C5
:10A4C000196C41F480611964196C01F48061009188
:10A4D0005321009D5462506251625B6FDB0013D4C4
:10A4E000114B00221149C3F85428C3F85828C3F867
:10A4F0005C28C3F86028C3F86428C3F86828C3F848
:10A50000501802B030BC7047A2F50062074BD2F879
:10A5100050289A42E4D102B030BC70470038024063
:10A520000070004000280040002000403166654275
:10A530002DE9F84FD0F894700446524B00F16406B0
:10A54000FDB227F0FF09826800F1180A103D484665
:10A55000D2F80080A3FB05352D09294645F0E6F821
:10A56000626D0023B2F5807F84F858307ED00DD81C
:10A57000102A00F083805CD8012A45D0042A16BF37
:10A580006FF400616FF008013C230EE0B2F5805FCC
:10A5900070D0B2F5803F3AD0B2F5806F15BF6FF43E
:10A5A00000616FF008013C230423324608F11806CD
:10A5B000404656F803C001EA0C01F150D4F854B0FB
:10A5C000594644F067FBBBF5807F2DD023D8BBF103
:10A5D000100F3ED036D8BBF1010F02D0BBF1040FF3
:10A5E00033D14FF0080C336852462946484643EAB7
:10A5F0000C0333604023236245F050F83B6843F07E
:10A6000010033B60BDE8F88F6FF00801CDE76FF0F5
:10A6100008013C23C9E7BBF5805F22D0BBF5803F32
:10A620001AD0BBF5806F10D108F11C064FF0080C52
:10A63000D9E7402A15BF6FF400616FF008013C2391
:10A640000023B2E7BBF1400FCBD03C364FF4006C97
:10A65000C9E74FF4006CC6E708F154064FF0080C48
:10A66000C1E708F11C064FF4006CBCE76FF008016D
:10A6700004239AE76FF40061042396E76FF4006106
:10A6800093E700BFABAAAAAA2DE9F0472422D0F88D
:10A69000205100238168C0F8942104462A6800F5FF
:10A6A000907722F001022A602B606B60AB604279E8
:10A6B000C0F824119102C0F89C3180F8903101F467
:10A6C0008051C0F89431C0F83831C0F82811110316
:10A6D000C0F8983101F40051C0F840310379C0F856
:10A6E0002C11110213F0010601F48061C0F8301141
:10A6F00003F0020140F0CA80002940F0F080C0F869
:10A70000346194F8B4314BB1D4F8443143F00803C8
:10A71000C4F844314FF40043C4F8543112F0080235
:10A72000D4F8943100F0F080002B00F02481242331
:10A730003846C4F894312B6823F001032B603CF0B9
:10A7400021FA012817D0D4F84431002B40F01681AB
:10A750006B6823F490436B60AB6823F02203AB601B
:10A76000AB6843F00803AB6038462B6843F0010345
:10A770002B6045F005F9002E5CD0D4F8FC60002E6B
:10A7800000F0DF80D4F8043104F13C08C4E90F6321
:10A7900000234046C4E91133C4E91433C4E9183333
:10A7A000C4E91A334FF48033E3654FF48063E36404
:10A7B0004FF48073A36545F0D1FA40463BF058FC56
:10A7C000D4F898A1C4F88C81BAF1200F67672ED114
:10A7D000E368626999B252B3B1FA81F94FEA591943
:10A7E00029B394F89001012821D00B46A4F87811E0
:10A7F0002221C4F89C914046C4F87421C4F89811F1
:10A800006A49C4F88C90A1676949E1676949C4F84D
:10A81000881005F124013BF0C5FC002800F0B6804B
:10A82000102384F89091C4F89C31C4F894A1736803
:10A83000C4F814312379980764D5D4F80051002D59
:10A8400056D0D4F80821002304F19C06C4F8A8309F
:10A850003046C4F8B030C4E927524022C4F8A420DE
:10A860004FF48062C4F8AC204FF48032C4E92D3339
:10A87000C4E93033C4E93233C4F8BC2045F06EFA81
:10A8800030463BF0F5FB00286ED0FEE70423C0F80D
:10A890003431B1B10C23D107C0F834317FF531AF79
:10A8A000D4F844314FF4803143F00203C4F84C1122
:10A8B00043F00103C4F844314FF40033C4F8483185
:10A8C0001FE7D3077FF51DAFD0F8443143F00203F3
:10A8D000C0F844314FF48033C0F84C3111E70823FD
:10A8E000C0F83431D3077FF50CAFD4F84431DFE73B
:10A8F000D4F8A0311A6842F080021A601A6842F057
:10A9000040021A60BDE8F0870BB194F8902124232F
:10A9100084F890213846C4F894312B6823F0010361
:10A920002B603CF02FF901283FF425AFD4F84431D7
:10A9300043BB6B6823F490436B60AB6823F02A033E
:10A9400011E7D4F8A0311A6842F480721A609A684C
:10A9500042F001029A601A6842F020021A601A68F6
:10A9600042F010021A6065E7C4F88861C4F8D47038
:10A970006860BDE8F08784F89031D8E638463CF04E
:10A9800075FAE5E638463CF071FAD2E784F89001B2
:10A990002B6843F480732B60AB6843F00103AB601A
:10A9A000AB6843F04003AB6041E700BF45240408B7
:10A9B000752404087924040838B50409013C052CE1
:10A9C0001AD80F4D00F00F0305EB4402B2F86C07E4
:10A9D00040FA03F212F0010210D00122254402FADB
:10A9E00003F3013B184048F089FC95F87837054A95
:10A9F000034402EBC30038BD002038BD104638BD0B
:10AA0000203705082C1F012070B586B000240546AC
:10AA100000F5847E0DF1040CC0F8044144F23B368D
:10AA20000594C0E93D44C0E93F44CDE90144CDE986
:10AA30000344BCE80F00AEE80F00CEF8004095F8E4
:10AA40002101A5F84C6108B906B070BDFFF7B4FF4D
:10AA50002946044690B126220C4BC28041F80C3F97
:10AA600041F096FEA2880A494FF00043B2FA82F202
:10AA70000868D34003430B6006B070BD034B41F838
:10AA80000C3F06B0BDE8704041F082BED18700089F
:10AA9000003C01402DE9F84F6D4EC0EB001306EB72
:10AAA000C303D3F8EC48002C00F08A8093F85C894B
:10AAB00005460701404641F02DFF01224FEA581399
:10AAC00008F01F08013B02FA08F2032B08D8DFE860
:10AAD00003F0ADB302B95F490B6A23EA02030B62CC
:10AAE0007B1B05F1010B06EBC3035FFA8BFB93F8AD
:10AAF000F008FFF761FF804618B1122380F807B015
:10AB000083717B1B06EBC30393F8F108FFF754FF37
:10AB1000824618B1132380F807B083717B1B06EBC4
:10AB2000C30393F8F208FFF747FF814618B11423D7
:10AB300080F807B083717F1B50462E2106EBC706B5
:10AB400096F8F428FFF7A8FA96F8F52848460E215B
:10AB5000FFF7A2FA96F8F3282E214046FFF79CFA59
:10AB600023683D4A23F04003944223602AD03B4BA4
:10AB70009C4231D103F500331A6A42F480421A62D2
:10AB80001A6A22F480421A62636843F48053636055
:10AB900023685B060CD4206840F217323049314BF1
:10ABA00001400A4322606268134043F4E06363603B
:10ABB000E36923F40063E361236843F04003236007
:10ABC000BDE8F88F234B5A6A42F480525A625A6A9F
:10ABD00022F480525A62D7E7234B9C421BD0234B6E
:10ABE0009C420DD0224B9C42CED103F568435A6A59
:10ABF00042F480125A625A6A22F480125A62C3E7FF
:10AC000003F582335A6A42F400525A625A6A22F4B5
:10AC100000525A62B8E703F5FE331A6A42F4004262
:10AC20001A621A6A22F400421A62ADE709494B69B6
:10AC300023EA02034B6153E706494B6A23EA020306
:10AC40004B624DE703490B6923EA02030B6147E7B7
:10AC50004019012000380240003001400038004017
:10AC60004000FFFFFBF0FFFF003C004000340140CC
:10AC70000050014008B51D20FFF79EFE10B190F96D
:10AC8000063053B11E20FFF797FE10B190F9063041
:10AC900003B108BD5523C38008BD5523C380F1E728
:10ACA0002DE9F04F002391B0A24E0293A24BA6F6DD
:10ACB0007C0ADFF88C9293F8DEEAA04D0EF1FF37A4
:10ACC000CDF80CE0FBB20193DFF88CB2DBF800703A
:10ACD000BB0AA3F58013522B00F2CF80534493F8A4
:10ACE000F4330D2B00F2C98015F90380039B012B6F
:10ACF00000F01681039B022B02D1B8F1080F3AD164
:10AD00000024214640460FF07FFE0FF005FF90F92A
:10AD100000C0BCF1000F18BFBCF1540F14BF4FF0BE
:10AD2000010C4FF0000C40F0F1800434A4B2102C60
:10AD3000E7D1029B002B00F0AB80814A0CE053442A
:10AD400093F8F4330D2B0ED8EB5643450ED002F595
:10AD500086724A4500F0988091680B689B0AA3F5BB
:10AD60008013522BEBD900234345F0D14B799BF84C
:10AD700005109942EBD10BF11C0B5E45A6D1029B4D
:10AD800009F586790133042B02939DD16D4A4FF06A
:10AD9000010B92F8F83502F5876A01330493049B9E
:10ADA0005B4567D0644BDAF80C7093F8F22A9AF896
:10ADB00010300193002F5DD062493B684D686248B6
:10ADC000B988002D1844039302914FEA902040F374
:10ADD000C8805B49002405E0013401F58671AC426E
:10ADE00000F0BC800B688342F6D1554B4FF486725D
:10ADF000029D02FB0434019B0322CAF80C708AF8FE
:10AE00001030029BCAF81840B3FA83F6C6F11F034C
:10AE10005800CAF80430BA7187F807B002FA00F790
:10AE2000A16C0122D4F854C0394302FA00F002FAAE
:10AE300003F3A164216D0143D4F8AC0021654149BD
:10AE40000F7899B2002F00F0708143EA0C0363651C
:10AE5000039B9D61FDF7A2F90BF1010B2046FDF765
:10AE600071F90AF1200A40F20113BBF1090F2AF827
:10AE7000043C94D111B0BDE8F08F019B012B7FF60B
:10AE80007AAF4FF000083BE7BCF1000F7FF473AFDF
:10AE90005846FDF71DF99BF805E0C3B2022B00F2FE
:10AEA000958300F1010C294A0CEB4C0C02F57D70E6
:10AEB0004FEA8C0C03E02C32904200F08783136839
:10AEC0009F42F8D113797345F5D152F80C30002B1D
:10AED000F1D01F48002142689A4207D00131243046
:10AEE00010293FF448AF42689A42F7D14B1C194AE7
:10AEF000DBB2013B03EBC30302EB830393F998300E
:10AF0000002B7FF438AFC9F808B038E7029B002B5C
:10AF10007FF413AF0BF11C0B5E457FF4D7AE2EE729
:10AF2000B8F1010F3FF4ECAE0BF11C0B5E457FF462
:10AF3000CDAE24E79C3F05084019012060B9050803
:10AF4000B0010020A80100200000FEBF2037050846
:10AF50007C00012000000120A03E0508042C00F028
:10AF6000F2804FF48671B54B01FB053319690691E8
:10AF7000002900F0FB829860013054210792C4B28E
:10AF8000AE4A83F8101183F811416B1C5360069B85
:10AF900018461E685B790593FDF79AF8C3B2022B39
:10AFA00000F2148300F1010EA5494FF0000C079A3E
:10AFB0000EEB4E0EDDF814904FEA8E0E06E00CF10B
:10AFC000010C2C31BCF1170F00F000830B689E427E
:10AFD000F5D10B794B45F2D151F80E30002BEED064
:10AFE00098462C2300EB4000954903FB0CF3DFF857
:10AFF000809203EB800391480B4419694FF48673E8
:10B0000003FB05034846C3E9078143680021434524
:10B0100007D00131243010293FF42CAF4368434559
:10B02000F7D14B1C8749DBB2013B03EBC30301EBB8
:10B03000830393F9981000297FF41CAF4FF48671B5
:10B04000814883F899404FF08C0C01FB05F17B4C53
:10B05000062A07914FEAA10100FB01F17B4800F5A8
:10B060004C7E07982044039CC0F800C10CFB01FCF7
:10B0700001EB4101C46001EB0111744C0EEB4C0E6D
:10B0800004EB81044FF05401C0F8FCE083F8981001
:10B090004FF033030799C0F8B8306D4BC0F8B44097
:10B0A00003EB01046B4BD3F82C1300F04D82072AFD
:10B0B000694B6A486A4A18BF1A466A4B18BF03466A
:10B0C0005E48B1FBF3F3B1FBF2F2013B4FF4867142
:10B0D000013A01FB05019BB2A1F8BC20A1F8743034
:10B0E0002366079B03F1580100F108033046194419
:10B0F0000023A4F858306366E36543F013FF336818
:10B10000059A43F0800333600C2A23D8DFE812F05D
:10B11000C301220022002200A101220022002200FD
:10B12000E3012200220022007D01C6F12F062D043A
:10B1300002FA06F33A4643EA0C036365039B9D61FA
:10B14000FDF72CF888E60323424A82F8F33A11B05F
:10B15000BDE8F08F394A4FF48673304603FB052370
:10B16000022259693368039123F0010333600023FD
:10B170000A930D930F93602308934FF480730E93FB
:10B18000012309930A23CDE90B3208AA43F082FD7B
:10B190000399B1F5807F00F0FD8100F2D88110297C
:10B1A00000F0028200F2E981012900F0FA8104290D
:10B1B00015BF4FF4006308233C20002006F118015E
:10B1C0000A5813430B50069B1879002840F0AB81B6
:10B1D000336843F0010333600023D9F804200133BE
:10B1E000904500F09B81102B09F12409F5D14FF017
:10B1F000FF334FF00008134A03EBC30302EB830352
:10B20000D86F194B984214BF9620952041F082FBCD
:10B21000059B0C2B00F27F81094A02EB4303B3F834
:10B220007CC84FF48673054A104803FB052300F2DF
:10B230006471A3F818C0002323E000BFA801002018
:10B2400020370508000001206B4CA4077412002071
:10B25000B00100204019012044950800D0DD06000F
:10B260001055220040771B0000600240A012002011
:10B270007C000120964200F088810133042B00F00D
:10B28000A88151F83320002AF4D1D0F88427013264
:10B29000C0F8842700EBC300DB00C0F864671944E2
:10B2A0004046234690228E884CEA060C0026A1F8E0
:10B2B00004C0BF49FEF7B0FD4FF48673BD4A40217C
:10B2C0004FF4403CBC4803FB05280423D8F81C502D
:10B2D0002A6842F010022A602A6842F014022A60AA
:10B2E000C4F8A860C4E91F66C4E92866D8F820201D
:10B2F000A1674FF48061C4F898C04FF4804CC4F843
:10B300008410E9B2C4F89C30C4F894201039039238
:10B31000D8F8B820A0FB010125F0FF00C4F8902068
:10B320004FF48052D8F80C90D940C4F88820079B7D
:10B3300009F1180209F11009226703F170029F4B0D
:10B340001A44D8F8B430C4F88CC06367CDE905015D
:10B3500044F0A4F9D5F800E0079BC4F820E0D5F844
:10B3600014E003F1B802954BC4F824E0D5F804E0EA
:10B370001A44039BC4F828E0D5F808E0C4F82CE090
:10B38000D5F80CE0C4F8DC300423C4F8C860C4F875
:10B39000E4304FF48063C4F8F060C4F8CC304FF46C
:10B3A0000033C4F830E0C4F8E030C4E93066C4E9E2
:10B3B0003A664FF40066D8F80031C4F8B890C4F883
:10B3C000D0604FF48046C4F8D830D8F8FC30C4F8C8
:10B3D000D460C4F8BC30DDE9050144F05FF92B68A6
:10B3E00063636B69A3636B68E363AB682364EB68B7
:10B3F00063642B6843F010032B602B6843F0140345
:10B400002B603B68BD880393F5E433684FF4867284
:10B4100068494FF0020E23F00103304602FB05128B
:10B420004FF48051516108AA336000230A930D93B1
:10B430000F93602308934FF480730E9301230993B5
:10B440000A23CDE90B3E43F025FC4FF400630420B2
:10B45000B4E633684FF486725649022023F00103A4
:10B4600002FB05121021516108AA336000230A93E0
:10B470000D930F93602308934FF480730E93012371
:10B4800009930A23CDE90B30304643F003FC00203A
:10B490004FF4006392E633684FF4867245493046B4
:10B4A00023F0010302FB05120121516102223360E6
:10B4B000002309910A930D930F93602308934FF48F
:10B4C00080730E930A23CDE90B3208AA43F0E2FB06
:10B4D0000020082372E633684FF486723549022053
:10B4E00023F0010302FB05124FF4807151616022C9
:10B4F000336000230E910A930D930F930123CDE93E
:10B5000008230A2308AACDE90B30304643F0C2FBDA
:10B510000823042052E64FF0000C82E65FFA83F81D
:10B5200008F1FF3367E6FFF747FA039038B1069951
:10B53000CA790221FEF7D8FC5423039AD380736C96
:10B5400043F40043736443E61D4A1E4BB8E5B1F56E
:10B55000805F22D0B1F5803F19D0B1F5806F15BF63
:10B560004FF4006308233C20042027E60223164AF8
:10B5700082F8F33A11B0BDE8F08F402915BF4FF4BF
:10B58000006308233C20002018E6DB0087E6082340
:10B590003C2013E60823042010E64FF40063042047
:10B5A0000CE60020082309E600204FF4006305E6BE
:10B5B000E9810008A8010020ABAAAAAAB0010020D6
:10B5C000882A1100A0BB0D004019012000235B68F0
:10B5D000FFDE00239B88FFDE2DE9F04F9A4C8BB0F5
:10B5E00094F8F47A1FB900200BB0BDE8F08F002268
:10B5F0002F2138460FF0E6FA06460028F3D090F8DF
:10B600000590D0F800A0A4F81894FEF703FB0028DA
:10B61000E9D0D0E9015B002DE5D0DFF8648200239A
:10B62000424601E0102BDED05168013324328D42B6
:10B63000F8D1DBB2013B03EBC302844B03EB820284
:10B6400092F998100029CED12F20C4F8D8A3A2F8DF
:10B650009800D4F82C037E4A904280F0D880000AEB
:10B66000C4F8DC137B490022A1FB00017A48C4F82E
:10B67000E823C4F8E0230A090909A0FB0202C4F880
:10B68000E4135208A4F8F82A5200A4F8F62A94F811
:10B69000152402F0FF01002A00F0C5800222504666
:10B6A0006E4984F815243BF0D9F90122384684F814
:10B6B0001524FFF781F9654BC4F8FC0A30B12F213E
:10B6C000C1804E21F279FEF70FFC604B644A0021E5
:10B6D000C4F804BBB9F10C0FC4F80C1BC4F81C1B54
:10B6E000C4F8241BC4F82C1BC4F8301B106BC4F81E
:10B6F000005B40F400101063106B00F40010009029
:10B700000098106B40F480001063126B02F480020A
:10B710000192019A4FF04002C4F8082B4FF4806266
:10B72000C4F8102B4FF48052C4F8142B4FF480420D
:10B73000C4F8182B4FF40032C4F8202B4FF003024A
:10B74000C4F8282B72D8474A02EB4902B2F898781D
:10B75000BA46083744484146002204EB870CCCF82F
:10B76000D803A0F5E560C4F8380B486801322431ED
:10B77000854260D0102AF8D14FF0FF3202EBC202AE
:10B7800003EB8203D86F394B984214BF9620952063
:10B7900041F0C0F80023D8F80420013308F1240850
:10B7A000954246D0102BF6D1002004EB8704534677
:10B7B00060222F49FEF730FBD4F8D8033AF058FC4A
:10B7C00000287FF410AFB47900276026089063004A
:10B7D0004A4602A9274803F002030493E300CDE997
:10B7E000026703F00803002600270593CDE90667EA
:10B7F00040F0F8F800287FF4F6AEA30749461D484C
:10B800001CD53BF09BF9B0FA80F04009ECE61A4AEF
:10B810001A490244A1FB0221890D013989B24A1C4F
:10B82000B0FBF2F01BE784F8141437E78A460F46A2
:10B830008FE7D8B2B9E7D2B2013A9FE73BF0DEF822
:10B84000B0FA80F04009CFE6401901200000012045
:10B85000006CDC02598B4F01ABAAAAAA1C1D012067
:10B8600000380240203705084024012000600240D3
:10B87000FD8F0008181D012000366E01819F5E16A5
:10B880007C000120F8B50E4C94F8F8759FB104F5D2
:10B89000C064C7F109070925013D0ED0A6683079BB
:10B8A000FFF78AF8217DF27908B1FEF71DFBAF4260
:10B8B00004F1A004F0D10120F8BDAB68FFDE00BFA9
:10B8C000A80100202DE9F041EFF31185502383F307
:10B8D0001288D0F800311B6813F0010304D0EDB2D8
:10B8E00085F31188BDE8F081D0F894210446D0F8A2
:10B8F00098110A4302F02102212AF0D0D0E909125E
:10B90000914250D090B23ED8194623691B1A9BB27F
:10B91000D4F89461A1620021202E84F8A411DED114
:10B92000A1698918DBD0B3FA83F77F09002BD6D041
:10B9300094F89021012AD2D00122D4F88801A4F8E9
:10B94000723184F890212122C4F89C71D4F82081AE
:10B95000C4F86C11A4F87031C4F89421B0B1144A41
:10B960000765C263134A0264134AC26408F12802DD
:10B970003AF018FC50B1102384F89071C4F89C314F
:10B98000C4F89461ABE7081A83B2C1E700234022F0
:10B99000C8F8202084F89031D8F8083043F08003AC
:10B9A000C8F808309BE7012380F8A43197E700BF6F
:10B9B0001D240408412404087924040870B5D0F833
:10B9C00020410546E369990614D5606AEB6AC0B266
:10B9D000002B73D0296B9847D5F82041236823F4B6
:10B9E00080732360A36823F00103A360A36943F07D
:10B9F0000803A361E369DA0701D501232362E36940
:10BA00009B0701D502232362E3695E0701D5042366
:10BA10002362E369180701D508232362E369590605
:10BA200015D54023236295F8B561002E30D0D5F8A6
:10BA30000031D3B12846FFF745FF95F8A431002B1C
:10BA400048D095F8B561D5F82041002E4AD0D5F8F8
:10BA5000003153B1E369DB0606D56B6B13B1984730
:10BA6000D5F820411023236270BDE3691A06F1D591
:10BA7000D5E90923934230D0A969CA5C0133D2B217
:10BA8000A2622A69B3FBF2F102FB1133AB62E1E778
:10BA900095F8B201FEF790FF236823F008032360B6
:10BAA000012385F8B5310028C1D032462021FEF7A8
:10BAB0001BFAD5F80031002BBCD1D6E7EB696A69D7
:10BAC000D054EB69EA680133B3FBF2F102FB1133A6
:10BAD000EB6181E7D5F82041B9E7236823F08003C3
:10BAE0002360B7E795F8B201FEF766FF236823F0FD
:10BAF00008032360012385F8B5310028A7D032461A
:10BB00002021FEF7F1F9A2E7BFF34F8F0549064B5D
:10BB1000CA6802F4E0621343CB60BFF34F8F00BFEB
:10BB2000FDE700BF00ED00E00400FA0508B572B6BD
:10BB3000FFF7EAFF30B583B0FEF7AEFC0320FEF757
:10BB40009FFC01284CD0324C0025324A0523C4F812
:10BB50009850C4F89C50C4F8A020C4F89430BFF3A7
:10BB60004F8FBFF36F8F4FF6FF01E2682A4B0A40F9
:10BB700013432A4AE360536F3AF0B4FC284B294937
:10BB8000A3FB0023D4F8FC209B0C42F08072C4F885
:10BB9000FC20C1F8603BD1F82C332349234AA1FB98
:10BBA000031323499B09C2F8B01F5560013B11687C
:10BBB000B3F1807F41F00101116007D34FF0E02223
:10BBC000136943F00403136103B030BD4FF0E0226A
:10BBD000F0215361072384F8231095611361EDE789
:10BBE00002210320FEF752FC0C4B12485A6C1249FA
:10BBF00042F480425A645B6C03F480430193019ADF
:10BC000002680B68026083F308884B689847FEE778
:10BC100000ED00E01B0000060005FA0500380240B8
:10BC200083DE1B4340190120D34D6210001000E059
:10BC300055CEACC5003801400000F01F800AA0F5C9
:10BC4000801052281CD80F4B034493F8F4330D2B6B
:10BC500016D8013910B40C4C04EB831CD4F82C43D7
:10BC60008BB2DCF8640B0CF66831CCF8703BB4FB9B
:10BC7000F2F2013A5DF8044BCCF8682B3AF0EEBED4
:10BC8000704700BF2037050840190120F8B5830A26
:10BC9000A3F58013522B52D804465748034493F817
:10BCA000F4030D284BD8554D860105EB8013D3F8CE
:10BCB000647BA74243D00139C3F8644B89B2C3F80F
:10BCC000701BD5F82C13B1FBF2F100220139C3F837
:10BCD000742BC3F86C2BC3F8782B93F8A12BC3F803
:10BCE000681B02F0FF015AB345490223AF1901EB6B
:10BCF0008011204687F8A13B04313AF0AFFE0123C2
:10BD0000B4F1804F87F8A13B3E4BA4EB0303B3FA99
:10BD100083F34FEA531316D0ABB93B4A944257D042
:10BD200002F58062944253D0384902F57C42944235
:10BD300018BF8C422FD002F5705294422BD0F8BD20
:10BD400083F8A01BD0E7AA1992F8A01B0129F6D00E
:10BD5000022182F8A11B2E49A06801400020A160A9
:10BD6000012182F8A11BAA19022182F8A11B626895
:10BD7000A16803B908B122F470022E4422F07002C7
:10BD800021F08001012000236260A16086F8A10BF0
:10BD900086F8A03BF8BDAA1992F8A01B0129CED0C5
:10BDA000022182F8A11B1A49A06801401948A1602C
:10BDB0000121201A82F8A11B0021B0FA80F082F83C
:10BDC000A01B124A40099442CDD00028CBD1F8BD27
:10BDD000AB1993F8A02B012AB1D002210C4A83F8A9
:10BDE000A11BA0680240A260012283F8A12B83F866
:10BDF000A11B6268A168C0E720370508401901202F
:10BE0000A42401200000014000040040000C004078
:10BE10008800FEFF0004014003689B0AA3F580131D
:10BE2000522B00D970470F4A134493F8F4330D2B6B
:10BE3000F8D8022210B40C4C407904EB831C20FA91
:10BE400002F3DCF8640B02FA03F3C26829B922EAB0
:10BE500003035DF8044BC360704713435DF8044B64
:10BE6000C3607047203705084019012003689B0A0A
:10BE7000A3F58013522B10D8084A134493F8F423E7
:10BE80000D2A0AD8407902230549D84001EB8212D5
:10BE90008340D2F8642BDB431361704720370508D9
:10BEA0004019012001490248FCF7C2BF4019012096
:10BEB0000000014010B5064C06482146FCF7B8FFCB
:10BEC00004F5C6710448BDE81040FCF7B1BF00BFDF
:10BED00040190120000001400044014002494FF098
:10BEE0008040FCF7A5BF00BF6C1901200149024842
:10BEF000FCF79EBF98190120000400400149024848
:10BF0000FCF796BFC419012000080040014902480F
:10BF1000FCF78EBFF0190120000C0040F8B5164D5B
:10BF2000164E2A69EB681A404FF00040B2FA82F3CD
:10BF3000EAB120FA03F3012A6FEA030302EA0301DC
:10BF40002B610A46F2D1D6F804718FB1013F00236C
:10BF5000BFB2C6F80431D6F8004134B12368204698
:10BF6000394698476468002CF8D10022DCE7F8BD18
:10BF7000EF6ABFB2EFE700BF001000404019012098
:10BF800001490248FCF754BF741A01200004014023
:10BF900010B5064C064804F59A71FCF749FF04F504
:10BFA00004710448BDE81040FCF742BF401901206D
:10BFB00000040140001C004001490248FCF738BF62
:10BFC000A01A01200040014001490248FCF730BF9F
:10BFD000F81A01200048014001490248FCF728BF37
:10BFE000241B0120001800402DE9F0414FF4257278
:10BFF0008EB000215E4846F0D1FF5E4B5E4E4FF0A2
:10C0000000085A6C40F222275C4D06F1440442F0CD
:10C0100001025A645A6C02F001020092009A1A6CF2
:10C0200042F001021A641A6C02F001020192019AB4
:10C030001A6C42F002021A641A6C02F002020292B6
:10C04000029A1A6C42F004021A641A6C02F004029A
:10C050000392039A1A6C42F008021A641A6C02F0F6
:10C0600008020492049A1A6C42F010021A641A6CC4
:10C0700002F010020592059A1A6C42F020021A642E
:10C080001A6C02F020020692069A5A6C42F00202E2
:10C090005A645A6C02F002020792079A5A6C42F4F0
:10C0A00080325A645A6C02F480320892089A5A6CB0
:10C0B00042F400325A645A6C02F400320992099A2E
:10C0C0005A6C42F480225A645A6C02F480220A921A
:10C0D0000A9A1A6C42F040021A641A6C02F040028A
:10C0E0000B920B9A1A6C42F080021A641A6C02F0DE
:10C0F00080020C920C9A1A6C42F480721A641B6CC7
:10C1000003F480730D930D9B55F82810002354F809
:10C110003320914226D001330E2BF8D1002008F1B4
:10C12000070840F0F7FBB845EED14FF0000840F2A9
:10C13000222755F82810002354F8332091420CD0C0
:10C1400001330E2BF8D1002008F1070840F0E2FB84
:10C15000B845EED10EB0BDE8F08106EBC30393F80D
:10C160004800F1E706EBC30393F84800D7E700BFA8
:10C17000401901200038024018480508D43F05083E
:10C18000800AA0F5801052280ED8084B034493F87B
:10C19000F4230D2A08D8064B03EB8213D3F8642B43
:10C1A000136843F001031360704700BF2037050890
:10C1B0004019012037B590F867380446032B2FD17A
:10C1C0000023204D8DF807309DF8073094F868283B
:10C1D0009A4201D803B030BD9DF8073005EBC30388
:10C1E00093F8283F8BB181F0010383B19DF80730AC
:10C1F00005EBC303D3F8240FFDF794FC9DF807303B
:10C200000133DBB28DF80730DEE70B46EDE79DF832
:10C21000073005EBC303D3F8240FFDF789FCEDE7E6
:10C22000D0E910039B7903F00103994204D003B0D5
:10C23000BDE83040FDF776BC03B0BDE83040FDF707
:10C2400077BC00BF4019012038B5044600790D467F
:10C2500050B1FEF7B1FB08B10323C380E279294650
:10C26000BDE83840FDF718BF38BD10B5044622219F
:10C27000FFF7EAFF2046FFF7F9FD20460121BDE860
:10C280001040C9E510B504460121FFF7DDFF00218C
:10C290002046BDE81040BFE538B510F8133CA0F6C5
:10C2A0006C041BBB94F858388BBBD4E909239A4221
:10C2B0001CD05A1CA169A262CB5C21695B008A4236
:10C2C00028BF002243F40073A262A4F85C380A235A
:10C2D00084F85A38012384F8583894F86738012BC9
:10C2E00001D0042B02D1606CFFF7CCFF94F85438D6
:10C2F000002B6DD194F855380133DBB2092B84F84B
:10C30000553825D12046BDE83840FCF709B894F9E6
:10C310005A586DB1B4F85C18013D20464B0801F045
:10C320000101A4F85C38FFF745FF84F85A58DDE7AF
:10C33000D4E9092384F858589A42D7D194F8673839
:10C34000012B01D0042BD1D1606CFFF78EFFCDE71C
:10C350000A2B3DD194F857382BB9B4F85E3843F026
:10C360000103A4F85E382379D9070AD5B4F85E082A
:10C37000820501D4C30718D4B4F864380133A4F893
:10C3800064380122002384F8542894F8572884F84C
:10C390005538012A1CD16179606C84F8573801F056
:10C3A0000101BDE838403FF03FBAE36AC0F34700FF
:10C3B00013B1216B9847E4E7E3696269D054E369FC
:10C3C000E2680133B3FBF2F102FB1133E361D8E71A
:10C3D00038BD00BF2DE9F041A14CA4B0D4F85C38C1
:10C3E000022B00F039829F489F4AA049121A46F05A
:10C3F0007DFD9F489F4AA049121A46F077FDD4F868
:10C400005838012B00F2C08003EB43039B4A9C4E3B
:10C4100002EB430032F8132041888388C6E9AF213C
:10C42000C6F8C432974C984D984BB2FBF1F298493C
:10C4300001FB02F20021C5F82C23D4F8882042F435
:10C440007002C4F888201A6842F001021A609960EC
:10C45000904A1868024090481A60C0F308078F4A53
:10C460005A601A6822F480221A60D96007B1FEE788
:10C470008B49A0604FF6FF000A688A4B42F40072B5
:10C480000A60E26802401343E36040F053FDBFF3EB
:10C490004F8FBFF36F8FC4F85072BFF34F8FBFF34E
:10C4A0006F8F636943F400336361BFF34F8FBFF352
:10C4B0006F8FC4F88470BFF34F8FD4F8803043F689
:10C4C000E07CC3F3C90EC3F34E33580100EA0C01FC
:10C4D000734641EA8372013B5F1CC4F86022F8D1C5
:10C4E000203810F1200FF1D1BFF34F8F636943F46F
:10C4F00080336361BFF34F8FBFF36F8F6849634B26
:10C500000A6842F480720A60196C674A41F08051EF
:10C510001964196C01F0805102910299116841F47B
:10C52000404111601268D6F8BC4202F440420192C8
:10C53000019A9A6802F00C02042AD6E9B07100F060
:10C540008B809A6802F00C02082A00F081804F4A22
:10C55000136843F480331360D5F8640F04E0D5F812
:10C56000643F1B1A642B72D813689B03F7D5474AA4
:10C57000936803F00C03082B69D0136823F08073D1
:10C580001360D5F8640F08E03D4ED6E9AF2149E7C6
:10C59000D5F8643F1B1A022B59D813689E01F7D4B3
:10C5A0000B06790843EA8413013943EA01433F4902
:10C5B00019435160136843F080731360334AD5F810
:10C5C000641F04E0D5F8643F5B1A022B3FD8136860
:10C5D0009801F7D5136C43F080531364136C324AFF
:10C5E00003F080530393039B136843F48033136079
:10C5F000D5F8641F05E0D5F8643F5B1AB3F57A7F80
:10C600002DD85368DB03F6D51368274943F400336C
:10C610001360D5F8642F05E0D5F8643F9B1AB3F595
:10C620007A7F1CD84B689E03F6D54FF400124FF06A
:10C63000006304A804924FF4C07221930723CDE94C
:10C64000082303230A9339F081FF88B3FEE7FEE74E
:10C650005B685A027FF57BAF0C4B1B6887E7FEE7F0
:10C660000020004000000000683C0000B84A0608B6
:10C6700000000020A801002067AB0608CC48050890
:10C680000000012000ED00E04019012000380240C8
:10C6900040420F00FFFFF6FE0000000810300024AB
:10C6A000003C02400003FA050070004008004020F2
:10C6B0006C4A136803F00F03062B0AD8136823F0A3
:10C6C0000F0343F007031360136803F00F03072BF6
:10C6D00069D1654B9A6842F4E0529A609A6842F4D4
:10C6E00060429A609A6822F0F0029A601A6890019B
:10C6F00059D59A6841F2883022F0030242F00202D2
:10C700009A60D5F8641F04E0D5F8642F521A82426B
:10C7100049D89A6802F00C02082AF5D1514A1368E8
:10C7200019070AD5136823F00F0343F007031360BA
:10C73000136803F00F03072B35D1DFF82C814B4E24
:10C74000D8F8083023F4E05343F4A053C8F8083075
:10C75000D8F8083023F4604343F40043C8F80830A5
:10C7600039F0C0FED8F80830C3F30313334493F80C
:10C77000C03020FA03F3C5F82C3340F0DBFB002374
:10C7800004A8CDE91333CDE91533CDE91733CDE94D
:10C790001933CDE91B33CDE91D33354B049339F003
:10C7A000D5FE08B1FEE7FEE702234FF0007204A8B1
:10C7B000CDE90633D823CDE9042301230B9339F0C7
:10C7C000C5FE00B1FEE7D8F88C3023F08073C8F8BE
:10C7D0008C30D8F88C3043F08073C8F88C30D8F89F
:10C7E000083003F00C03042B31D0082B12D0214B5E
:10C7F0002149B4FBF7F201FB02F21B498968C1F33E
:10C8000003110E4496F8C010CB409A42C5F82C3361
:10C810001FD0FEE7D8F80430D8F8042013F4800FB6
:10C82000D8F8043002F03F0218BF1449C3F388134C
:10C8300008BF1049B1FBF2F202FB03F30A4A526847
:10C84000C2F3014201325200B3FBF2F3D0E70B4BCB
:10C85000CEE724B0BDE8F08100210320FDF716FEED
:10C86000FFF752F9003C0240003802401848050822
:10C87000C0FF03000024F40040420F0000127A00C1
:10C8800010B4EFF31182102383F312880C4B4FF096
:10C89000E0200024D2B2D3F8D4120131C3F8D4126C
:10C8A0008169C3F8681FC3F86C4F016982F311886E
:10C8B000D3F8642F5DF8044B0132C3F8642F70473E
:10C8C0004019012010B4EFF31181102383F3128873
:10C8D0004FF0E0229469136913F4803F0D4B03D0AD
:10C8E0000120C3F86C0F9469D3F8D402C9B2D3F80D
:10C8F0006C2F81F311880244D3F8601B4FF47A70D7
:10C9000000FB01F31B1B5DF8044BB3FBF1F300FBD1
:10C910000230704740190120134B5B68C3F30803D2
:10C9200003BBEFF31183EBB9104B4FF0E02C10B4C5
:10C93000D3F8D422DCF81800D3F8D4128A42F7D105
:10C94000D3F8681F8842F3D8D3F8604B4FF47A715C
:10C9500001FB04F31B1AB3FBF4F35DF8044B01FB7A
:10C9600002307047AEE700BF00ED00E04019012043
:10C970002DE9F04F374C83B023781BB9012003B069
:10C98000BDE8F08F344F04F58764DFF8D0B04FF086
:10C99000000AD7F8D4324FF6FF7894F8C0910BF51F
:10C9A0003875ABF5F166019314E0B0F5606F43D0D4
:10C9B000A881B0EB0801019A584618BF01210BF07D
:10C9C000F3FD0AF1010A0BF15C0B20341435BAF1C6
:10C9D000080F2AD0CA4528D0A0696268D0E93D0175
:10C9E00046F076FE4FF6FE7397F8712F984214D0FA
:10C9F000542A04D1B7F8742F0132A7F8742FD6F84F
:10CA0000702A404502F10102C6F8702ACDD1D6F84D
:10CA10006C2A0132C6F86C2ACBE7542AD1D1B7F878
:10CA2000762F0132A7F8762FCBE70123012086F875
:10CA30006C3B03B0BDE8F08F97F8D42302EB4202C1
:10CA400007EBC202524492F881230D2AB0D1802212
:10CA5000AA77AEE7A801002040190120281A00207B
:10CA600070B546F051FE80B31A484568002D10DDC0
:10CA7000002410F8086B16B1037F012B1FD0426908
:10CA8000013400F586701368AC4243F00103136073
:10CA9000F1D1FFF741FF104BD3F88447002C0DDD97
:10CAA00003F2647303EBC4041968083333F8042CED
:10CAB000C868A34242EA0002CA60F5D170BD0023F3
:10CAC00080F8FC30FBF73EFBD9E743F027FE002857
:10CAD000CAD170BDA8010020A01200202DE9F04F9E
:10CAE000894C87B023781BB9012007B0BDE8F08FCF
:10CAF000864BD3F8D4320493FFF70EFF94F8F82551
:10CB00000192002A00F0F880814A04F5C0640027F1
:10CB1000D2F8783B02F5F16B02F6682A2646A0EBC4
:10CB200003080594B8F1000F03DBF36D434500F3F0
:10CB3000C98007EB8703744A02EB431393F8583616
:10CB400003F0FF0E002B00F08780D6F89410B36836
:10CB500070481A68CBB221F0FF01103BA0FB030321
:10CB60006D481B09C35C0B44B1895C68D368A4B2EF
:10CB700023EA0103C4F11604D360072C6CD9644A7C
:10CB80000121D2F8703A89460133C2F8703A002286
:10CB9000D6F89C30154618689C46CDE902E715E0AA
:10CBA000142D1EDC17F1080E48BF07F1170E4FEACF
:10CBB0002E1705EB2E1507F1FF3E013102FA07F79C
:10CBC00009FA0EFE8C424EEA07020AD307468C424F
:10CBD0005CF8040FA0EB0707E2D8C5F1150715258F
:10CBE000E9E7152DDDE902E762D14C4CC2F384215F
:10CBF000C2F3441004EB810104EB8000D1F8501122
:10CC0000D0F85001090241EA001102F01F00C2F3FE
:10CC1000C43204EB800004EB8202D0F85001D2F859
:10CC20005021014341EA023282EA122181EA1111C4
:10CC300001F00F010F293BD1C2F30F124FF6FF7124
:10CC40008A4235D0B2F5606F40D0AAF80C20714608
:10CC5000049A58460BF0A8FC30460137FDF768FCF3
:10CC6000019BA0360BF15C0BBB420AF1140A7FF466
:10CC700059AF019B0121059C002203EB830324484B
:10CC800004EB431380F86C1BC0F8782BA268A03427
:10CC900014F8901C126854F84C0C11F0020F116A31
:10CCA00014BF41EA80010143A3421162EED11BE7A8
:10CCB0001749D1F86C2A0132C1F86C2AB7B14FF08C
:10CCC000000EC4E7002007B0BDE8F08F0F4991F8CF
:10CCD000D43303EB430301EBC3033B4493F88133A9
:10CCE0000D2BB2D180238AF81E30B0E719465822A6
:10CCF0000B4846F0FBF8E2E7054B0122019983F867
:10CD00006C2BC3F8781BEFE6A80100204019012026
:10CD1000A0120020ABAAAAAA70B9050818480508F5
:10CD2000B41D00202DE9F0472F4FFFF7F5FDDFF888
:10CD3000C09080467E6800202C4C002E48DD0023E9
:10CD40004FF486711D4601FB0372013392F80521F1
:10CD50009E4245EA0205F6D128435FFA80FAD9F8E7
:10CD60000430C3F3080383BBEFF311836BBB4FF0B5
:10CD7000E02CD4F8D432DCF81810D4F8D422934242
:10CD8000F7D1D4F8682F9142F3D8D4F860CB4FF4A0
:10CD90007A7202FB0CF0401AB0FBFCF002FB0300BD
:10CDA000A0EB0803B3F5FA6FCCBF002005F001003B
:10CDB0000028C2D1BAF1000F04D00C4B93F8712FA8
:10CDC000542A08D05046BDE8F087FFF77BFDE7E71F
:10CDD00082460025C3E7B3F8782F50460132A3F806
:10CDE000782FBDE8F08700BFA8010020401901207E
:10CDF00000ED00E02DE9F04F874C83B00746D4F8F2
:10CE0000E09294F8E8320191B9F1000F0BD083F071
:10CE10000202B9F80410C2F34002120101FA02F250
:10CE2000D9F800108A61D4F8DC82B8F1000F09D07B
:10CE300003F00103B8F804201B0102FA03F3D8F849
:10CE400000209361013F754E4FF0E0254FF47A7B4F
:10CE5000FBB20093B9F1000F08D0D9F80010B9F86F
:10CE600004304869034218BF1B048B61B8F1000FFE
:10CE700000F0C980D8F80010B8F8043048690342BF
:10CE80004FF0010018BF1B048B610DF069F8DDF84D
:10CE900004A07368C3F30803002B40F0B080EFF3E5
:10CEA0001183002B40F0AB80D4F8D472A869D4F879
:10CEB000D4128F42F8D1D4F8681F8842F4D8D4F83D
:10CEC000603B0BFB03F1091AB1FBF3F10BFB0717F6
:10CED0007368C3F30803002B40F08A80EFF31183DB
:10CEE000002B40F08580D4F8D432A969D4F8D4025C
:10CEF0008342F8D1D4F8680F8142F4D8D4F8602B7B
:10CF00000BFB02F0401AB0FBF2F00BFB0300C31B5B
:10CF1000B3F57A7FDCD3BAF1010ABAD1B9F1000FC7
:10CF200008D0D9F80010B9F804304869034218BF96
:10CF30001B048B61B8F1000F69D0D8F80010B8F865
:10CF40000430486903424FF0000018BF1B048B6196
:10CF50000DF006F8DDF804A07368C3F30803002B96
:10CF600049D1EFF31183002B45D1D4F8D472A869CD
:10CF7000D4F8D4128F42F8D1D4F8681F8842F4D87C
:10CF8000D4F8603B0BFB03F1091AB1FBF3F10BFB87
:10CF900007177368C3F308033BBBEFF3118323BB8D
:10CFA000D4F8D432A969D4F8D4028342F8D1D4F8A1
:10CFB000680F8142F4D8D4F8602B0BFB02F0401AC2
:10CFC000B0FBF2F00BFB0300C31BB3F57A7FE0D399
:10CFD000BAF1010AC0D1009B5F1EFBB2FF2B009388
:10CFE0007FF438AF03B0BDE8F08FFFF76BFCEBE7E1
:10CFF000FFF768FC8BE7FFF765FC0746C9E7FFF71B
:10D0000061FC074664E701200CF0AAFF3FE74046B9
:10D010000CF0A6FF9EE700BF4019012000ED00E0E4
:10D020002DE9F0410746DFF86080FFF775FC154CED
:10D030004FF0E0250646D8F80430C3F30803EBB9F7
:10D04000EFF31183D3B9D4F8D432A969D4F8D42238
:10D050009342F8D1D4F8682F9142F4D8D4F860CB39
:10D060004FF47A7202FB0CF0401AB0FBFCF002FBAA
:10D070000300831BBB42DED3BDE8F081FFF722FC37
:10D08000F7E700BF4019012000ED00E02DE9F04175
:10D09000294F461E294C7B68C3F30803002B47D158
:10D0A000EFF31183002B43D14FF0E020D4F8D432BA
:10D0B0008169D4F8D4229342F8D1D4F8682F9142F0
:10D0C000F4D8D4F8600B4FF47A7202FB00F8A8EBA6
:10D0D0000108B8FBF0F802FB03884FF0E0257B68FD
:10D0E000C3F308030BBBEFF31183F3B9D4F8D432C5
:10D0F000A969D4F8D4229342F8D1D4F8682F914288
:10D10000F4D8D4F860CB4FF47A7202FB0CF0401ADA
:10D11000B0FBFCF002FB0300A0EB0803B3F57A7F41
:10D12000DDD3013EB7D2BDE8F081FFF7CBFBF3E7DB
:10D13000FFF7C8FB8046D0E700ED00E04019012072
:10D1400001302DE9F0475D4E4D1E5D4C5FFA80FACF
:10D150004FF4FA7732210520FFF74CFE7368C3F3D2
:10D160000803002B40F0A180EFF31183002B40F067
:10D170009C804FF0E020D4F8D4328169D4F8D422D6
:10D180009342F8D1D4F8682F9142F4D8D4F8600BC8
:10D190004FF47A7202FB00F9A9EB0109B9FBF0F92F
:10D1A00002FB03994FF0E0287368C3F30803002BD8
:10D1B00078D1EFF31183002B74D1D4F8D432D8F89E
:10D1C0001810D4F8D4229342F7D1D4F8682F9142A2
:10D1D000F3D8D4F860CB4FF47A7202FB0CF0401A0B
:10D1E000B0FBFCF002FB0300A0EB0903B3F57A7F70
:10D1F000DAD3013FB2D14FF47A77FA215046FFF7E4
:10D20000F9FD7368C3F30803002B52D1EFF31183C8
:10D21000002B4ED14FF0E020D4F8D4328169D4F8FD
:10D22000D4229342F8D1D4F8682F9142F4D8D4F89C
:10D23000600B4FF47A7202FB00F9A9EB0109B9FB0C
:10D24000F0F902FB03994FF0E0287368C3F3080379
:10D250002BBBEFF3118313BBD4F8D432D8F81810DA
:10D26000D4F8D4229342F7D1D4F8682F9142F3D85E
:10D27000D4F860CB4FF47A7202FB0CF0401AB0FB8A
:10D28000FCF002FB0300A0EB0903B3F57A7FDCD3CB
:10D29000013FB6D1013DBFF45BAFBDE8F087FFF7BA
:10D2A00011FBF0E7FFF70EFB9EE7FFF70BFB814654
:10D2B00078E7FFF707FB8146C5E700BF00ED00E018
:10D2C00040190120431C0A265D4D5E4C5FFA83FA2B
:10D2D00080B54FF4FA7832210520FFF78BFD6B689B
:10D2E000C3F30803002B40F09F80EFF31183002B62
:10D2F00040F09A804FF0E020D4F8D4128369D4F83B
:10D30000D4229142F8D1D4F8682F9342F4D8D4F8BB
:10D31000600B4FF47A7202FB00F7FF1AB7FBF0F7CD
:10D3200002FB01774FF0E0296B68C3F30803002B81
:10D330007ED1EFF31183002B7AD1D4F8D402D9F83F
:10D3400018C0D4F8D4329842F7D1D4F8683F9C453D
:10D35000F3D8D4F8601B4FF47A7202FB01F3A3EB0D
:10D360000C03B3FBF1F302FB0033DB1BB3F57A7F55
:10D37000DAD3B8F10108B2D14FF47A78FA215046E5
:10D38000FFF738FD6B68C3F30803002B48D1EFF3B8
:10D390001183002B44D14FF0E020D4F8D4128369DC
:10D3A000D4F8D4229142F8D1D4F8682F9342F4D81B
:10D3B000D4F8600B4FF47A7202FB00F7FF1AB7FB48
:10D3C000F0F702FB01774FF0E0296B68C3F3080325
:10D3D00093BBEFF311837BBBD4F8D402D9F818C008
:10D3E000D4F8D4329842F7D1D4F8683F9C45F3D8AA
:10D3F000D4F8601B4FF47A7202FB01F3A3EB0C0329
:10D40000B3FBF1F302FB0033DB1BB3F57A7FDCD314
:10D41000B8F10108B6D1013E7FF45BAF3EF0DAFA15
:10D42000FFF750FA0746CEE7FFF74CFA074679E7D1
:10D43000FFF748FA034698E7FFF744FA0346E3E7A5
:10D4400000ED00E04019012038B5094C04F54075A5
:10D4500002E00834AC420AD094F90620002AF8D140
:10D46000204608342021FCF73FFDAC42F4D138BD02
:10D470002C1F0120094B02460220D3F82C13B2EBDB
:10D48000910F4FEA910307D25B0840009A4280B2A5
:10D4900002D2FF28F8D97047704700BF4019012019
:10D4A0002DE9F04F7F4E85B0DFF814B24FF0010A3E
:10D4B0004FF000097C4D09E009F101090AF1010A68
:10D4C00028360BF1050BB9F1040F34D03378022B59
:10D4D000F2D19BF90330591C00F0CE80DAB29646A7
:10D4E0000C2308205FFA89F1039613FB0200D3B2E4
:10D4F000012B17D86D4B02E01C33AB4212D01C78C5
:10D50000002CF9D15E788E42F6D11E58002EF3D051
:10D51000674FB44602977E6801342437B4450DD076
:10D52000102CF8D101320C30D3B29E45E0D200234A
:10D53000039E019327E005B0BDE8F08FE4B25D4E95
:10D54000671E019407EBC70406EB840CA4009CF94A
:10D550009880B8F1000FE5D102EB420207F007070F
:10D56000019803EB82038CF884708CF899A0DB6837
:10D57000DDE90216CCF88830142321448CF8983069
:10D580003161FCF727FC9BF904305A1C70D0D9B2EA
:10D5900088460C2308275FFA89F0039613FB01776E
:10D5A000CBB2012B18D8414A02E01C32AA4213D058
:10D5B0001378012BF9D153788342F6D1D659002E36
:10D5C000F3D03B4B0024B44602935E68013424330D
:10D5D000B44521D0102CF8D101310C37CBB24345E2
:10D5E000DFD9019B039E002B3DD0019F24223048B0
:10D5F00000247B1E746102FB03003061FAF742FDD8
:10D600003046FAF711FD2346224638462A49FCF7F0
:10D6100003FC012333734FE7E4B2264E631E03EB92
:10D62000C30E06EB8E0C4FEA8E0E9CF99860002E0E
:10D63000D2D101EB410103F0070337468CF899A0E2
:10D6400002EB81028CF88430DDE90206D368704475
:10D65000CCF888301323706120468CF89830FCF7A2
:10D66000B9FB019B63B900220023C6E9042323E729
:10D670004FF0010800218CE74FF0010E00222FE748
:10D680007069FAF7FFFC3069FAF7FCFC3046FAF7EC
:10D69000CBFC3B463A4620460849FCF7BDFB01233C
:10D6A000337309E7C82801207C3E0508F83B0508CC
:10D6B0007C00012000000120C19100083591000884
:10D6C0006829012070B50E494FF0010E0D4D0E4C2A
:10D6D0000E4E35F802CB00234CFA03F20EFA03F09B
:10D6E000013312F0010F03D00C60083121F8040C53
:10D6F000102BF1D104F58064B442EAD170BD00BFB3
:10D700002C1F01208C3E050800000240001802403A
:10D710002DE9F0470646086888B00C46850ABDF832
:10D720004080A5F580159DF844A0522D55D8194686
:10D730002D4B2B4493F8F4530D2D4ED82B4FFEF761
:10D74000A5FA94F8059007EB8517A379BAF1000FB5
:10D7500001D083F001035A004FF48071DB0038469A
:10D7600002F00202CDF8088003F0080303924A4653
:10D770000493602301934FF40073CDE90613002353
:10D7800001A905933EF02EF9A379384649469F0733
:10D7900026D439F033F9164BA801022203EB851584
:10D7A000D5F8641B85F8A12B124A8D682A40062AF9
:10D7B00006D0B2F5803F03D00A6842F001020A6049
:10D7C0000344012283F8A12B2168637901F134021B
:10D7D00071600021D0183060D15008B0BDE8F087EA
:10D7E00039F0ACF9D7E700BF20370508A4240120A1
:10D7F00040190120070001000548D0F8A03223B1EC
:10D80000DB6A13B100F5287018470248704700BF63
:10D8100040190120E849050838B5184C54F8BC3CBB
:10D820001B8843B9164D002304F8AD3C85F89832A7
:10D83000C5F8943238BD54F8B82C002AF2DD54F8FB
:10D84000B41C012A488806D001230D4D24F8B00CE1
:10D8500004F8AE3CE7E78A880132121A9A42F3D103
:10D86000074D0022D5F8A03205F52870C5F8CC2266
:10D870001B69984743F006FAD5E700BF382A012014
:10D88000401901200748D0F89C321BB1064B13F811
:10D89000AE3C0BB100207047D0F8A03200F52870E4
:10D8A0005B68184740190120382A0120184A10B433
:10D8B000184C92F8983244602344174C036092F855
:10D8C000980214F8AD3C834218D892F8980283422B
:10D8D00007D300235DF8044B1A461846C1E900320D
:10D8E000704792F898021A1E5DF8044BC0F180034D
:10D8F0000CBF01200220C1E90032704792F8984223
:10D90000002201201B1B5DF8044BC1E90032704767
:10D91000401901201C1E0020382A0120104B114AFA
:10D9200093F8981212F8AD0C93F89822904293F85D
:10D9300098220FD8904204D3D3F894320020184490
:10D94000704793F89822D3F89432C2F180021044C1
:10D9500018447047801AD3F894321844704700BFB7
:10D9600040190120382A012038B5144D144C55F8BF
:10D97000BC2C937B012B08D0D4F8943203F2FF73B4
:10D980006FF30A03C4F8943238BDD4F8A0325B6A4E
:10D9900033B104F52870984743F074F955F8BC2C5E
:10D9A000D4F894325288013B514213440B4003F2A5
:10D9B000FF736FF30A03C4F8943238BD382A01208C
:10D9C00040190120F0B51C4C85B01C4B94F89822EE
:10D9D0001B4D0393134415F8AD1C94F89822029341
:10D9E000914294F8983216D899420CD294F89862E1
:10D9F0000F46C6F18006D9B9334601223F2BCDE947
:10DA000000670DD860B994F89802401AB0FA80F017
:10DA1000400905B0F0BDCB1A002701221E46EDE7F4
:10DA20006946002302A843F0DBF815F8AD1CEAE7CD
:10DA300073180222E2E700BF401901201C1E0020DB
:10DA4000382A01202DE9F047174684B000293ED03E
:10DA5000441E294DDFF8AC904FF0000A04EB01089A
:10DA6000264E0DE096F898320846994296F898327C
:10DA70001DD2C3F1800318443F281BD8A04526D0EF
:10DA800015F8AD0C14F8013F411C4844C9B280F8A8
:10DA90007C3B0B0605F8AD1CE4D5002096F89832C7
:10DAA00005F8ADAC0146994296F89832E1D3C01A18
:10DAB0003F28E3D996F898329942DFD0104B5B7833
:10DAC000002BDBD00020FFF77DFFA045D8D16946B1
:10DAD00002A8FFF7EBFEDDE9003213443F2B00D92B
:10DAE00010B904B0BDE8F08702463B4602A843F0F7
:10DAF00077F804B0BDE8F087382A012040190120EA
:10DB000000000120A012002030B585B0694602A8AF
:10DB1000FFF7CCFE58B9094C04F52875D4F8A032AB
:10DB200028465B6898470028F8D005B030BD02460B
:10DB3000012302A843F054F8EDE700BF401901208B
:10DB400038B50023124C134DC5F89C323DF03AFD18
:10DB500044F8B40CFFF750FE54F8B43C44F8BC0C45
:10DB6000A3B19A885B88D21A436802FB0333C5F8D5
:10DB70009C32FAF79DFD14F8AD2C044695F89832C6
:10DB80009A4201D0FFF7C0FFC5F8944238BD00BFEC
:10DB9000382A0120401901202DE9F041104E154688
:10DBA00082180446D6F89C320F469A420D4A88BF26
:10DBB0001D1A12F8AD2C96F898329A4201D0FFF750
:10DBC000A3FF002021462B463A46C6F8CC02D6F8E1
:10DBD000A002846A0448A446BDE8F041604700BF43
:10DBE00040190120382A0120E01B01208C461346F1
:10DBF000014662461846CFE72DE9F043484F93B0FF
:10DC0000484DFFF709FE97F8983215F8AD2C9A4267
:10DC100001D0FFF779FF0024D7F89C62C7F894423F
:10DC2000002E6DD0DFF800810AE097F8983215F8E1
:10DC3000AD2C9A4201D0FFF767FF2034A6421BD9D2
:10DC400022464146684601F079FB684643F0CEF82B
:10DC5000012201466846FFF7F5FEA3B2002BE4D18E
:10DC6000D7F8DC32002BE0D09A881B6859690A4249
:10DC700018BF12049A61D8E7FFF776FE97F898323A
:10DC800015F8AD2C9A4201D0FFF73EFF0023DFF8D4
:10DC9000989098461C46C7F894322246494609A8EF
:10DCA00001F04CFB21220021684645F077F9202243
:10DCB00069462046FFF770FF2022054609A96846FD
:10DCC00045F05CFAA3B2203450B9202D08D15BB1E5
:10DCD000A642E2D8B8FA88F0400913B0BDE8F08354
:10DCE00008F10108002BF3D1D7F8DC32002BEFD07C
:10DCF0001A689B8851690B4218BF1B049361E7E7C0
:10DD0000FFF732FE97F8983215F8AD2C9A4201D001
:10DD1000FFF7FAFE00230120C7F89432DDE700BFC9
:10DD200040190120382A0120E0B805080B4B93F870
:10DD3000CC221AB90A4A12F8AC0C70470949D1F83A
:10DD40005C28032AF6D10020054A4FF0010C83F825
:10DD5000CC0202F8ACCCC1F85C08ECE70000012072
:10DD6000382A01200020004008B50322104BC3F8D8
:10DD70005C2872B60F4B53E92A1251EA020308D10C
:10DD800000231A460A49C1F86028C1F86438FDF733
:10DD9000CDFE094B4EF6602CD3F8D4320CFB00F0CC
:10DDA0005B1842F10002C31842EBE072EAE700BFE1
:10DDB00000200040382A01204019012000210320C2
:10DDC00008B5FCF763FB72B6FDF79EFE154C08B56F
:10DDD00054F8A03C14F89A0CABB91420FFF756F98C
:10DDE00000BF54F8A03C5BB1196814F89A2C9B88CA
:10DDF00009690B4012B91BB1FFF7E0FF002BFBD004
:10DE0000FAF78AFCECE719689A880B69134020B18D
:10DE1000002BE2D10B691340FAE7002BDDD00B6930
:10DE20001340FAE7382A0120F8B53BF01DFB1B2010
:10DE3000FCF7C2FD08B12923C3801C20FCF7BCFD00
:10DE400008B12923C380144CD4F8F43113B1002352
:10DE5000C4F8F431114E01250027C4F8F06184F8AC
:10DE6000DC5104F8987C3FF07DF906F11C03C4F8FE
:10DE7000F43194F81932AB4201D02846F8BD54363B
:10DE8000D4F81002C4F80C6241F0A8FD044B3846E7
:10DE900083F82370F8BD00BF382A0120D00201208A
:10DEA00000ED00E02DE9F04F00218BB041F69462C7
:10DEB000B84845F073F80420FCF7E2FA0146052063
:10DEC000FCF7DEFA51EA000340F05781B24B0393AE
:10DED0004C220021AF48012445F060F800214C227B
:10DEE000AC4845F05BF8039BAA4AD3F87433AB4DBA
:10DEF000164614711560D361136253623FF03CF80B
:10DF0000FFF71EFE002108460BF0EAF8FAF7D0FBF7
:10DF1000B0F1000840F39B810024A14DDFF8A4E29A
:10DF200006F14C092746A24605F5077B9D4E029453
:10DF3000CDF804E004E00AF5006AD04540F3AE8075
:10DF4000019AD2F8D432C2F8D832FAF7E5FB20228F
:10DF500059465046FFF720FE12229349584645F095
:10DF60000DF90028E7D1BA4525D002998F4B01EB76
:10DF7000410203EB82034A1C8D4918460293AAEB27
:10DF800007030592049301F0D9F9029B4946059ACB
:10DF900041F84C3B049BC9F80C700292C9E9043368
:10DFA000D9F81C30C9E908330123C9F80830814B7E
:10DFB000C9F828308946039B57461222D3F8743398
:10DFC000C9F81C30A918335D013291F81C1299422E
:10DFD0000BD00024202AF5D120375946B8453846C1
:10DFE00053DBFFF7D9FD0022ECE70134152CF1D10A
:10DFF000D019714F20223946FFF7CEFD3846002355
:10E000000A2209A9099701F0B7FA074609980023DF
:10E010000A2209A90130099001F0AEFA0790002305
:10E0200009980A2209A90130099001F0A5FA069081
:10E03000002309980A2209A90130099001F09CFAED
:10E04000059009A9099800230A220130099001F0DE
:10E0500093FA0023049009980A221946013001F02E
:10E060008BFA97B10599DDE9063243EA4212049B27
:10E070005B0143EAC123A7F2BC7143EA600342EAB1
:10E08000412243EA0243C9F81C30029B642B43D06F
:10E0900057460AF5006AD0453FF752AF029B642B02
:10E0A0001ED0BA451CD00C22404C5E1C404902FBDD
:10E0B0000344AAEB07053246204601F03FF9D9F8A0
:10E0C0001C20C9F80040C9F80C700296C9E9082262
:10E0D0000122C9F80820374AC9E90455C9F828209F
:10E0E000029B002B03F1010117DC4FEA4803B3F157
:10E0F000805FC0F2AD80274B9C6834B91A461B790B
:10E100001BB11368002B40F0D980002108460BB0EA
:10E11000BDE8F04F0AF0E4BF65214C261D48DFF84A
:10E12000A8A04FF0010906FB01F432460021234F5D
:10E130000519284644F032FF32460021284644F0B3
:10E140002DFF1C4E134804F1100204F1180302992C
:10E1500040F804A0C5F8089002312F62AE6240F882
:10E16000028002440430C2F80480039AD2F8742377
:10E17000C25003445A606A62B7E74FF47A720023D0
:10E1800043F092FA0E4B40F2B27240F26D14B0FBC3
:10E19000F3F31DE0E031012000000120D027060844
:10E1A000382A012024B9050800B90508742C01207B
:10E1B00014B90508EDDB0008542C01200068214C3F
:10E1C00080510100401901203CB905085B1A013259
:10E1D00012F0030514BF21464FF4B7718B42F5DAF4
:10E1E0008549002D64D003910399D1F844138B42E3
:10E1F000C0F29C80814D01245B1A55F8041F013444
:10E200009942F9DD0133A2F2BC72039D43EA441343
:10E210003C2443EA42237A4AB0FBF2F102FB1102AA
:10E220004FF46160B2FBF0F100FB11221C20C5F835
:10E230004803B2FBF4F004FB1022521042EA4012F1
:10E2400042EAC12242EA0343C5F8743340E621465C
:10E250004C266C4BDFF8B891012706FB01F43246DF
:10E2600000214FF0020A1D19284644F097FE32465D
:10E270000021284644F092FE624B039A04F11801F3
:10E2800043F80490C8F10063D2F8740304F110025B
:10E29000BB405C4C5C4E85F805A0AF602E62A3507D
:10E2A00022445360231D585019444860686222E795
:10E2B0000C4603911D21C4F8481395E751480022EC
:10E2C0000023214626468464C463C0E91023024625
:10E2D000D56C02F14C035DB398684D1E9E64A84254
:10E2E000C2E92366DE630DD04D1CA84210D113F89D
:10E2F000481C00293FF409AF1A6401461A4643F846
:10E30000083CE5E700293FF400AF53F80C2C014628
:10E3100000293FF4FAAE81427FF4F7AE106CC56B72
:10E320000135C563186493641A46D1E7012469E78F
:10E33000344A0226294613E0D36B16635B01C2E917
:10E34000041120D003F6FF7300EB13331846536318
:10E35000C31A906352F84C7F461C1D440134C7B168
:10E360001379701E002BE7D1136916637BB103F696
:10E37000FF7300EB13335769536337B107F6FF7729
:10E3800000EB1730E4E73346E0E73046E0E733469A
:10E39000F1E7DFF880E00138CEF82443820F1B4C10
:10E3A0008300CEF818533F25CEF8FC424024CEF827
:10E3B0001403CEF808433E24CEE9C045D0B140F264
:10E3C000FF141B1942F100025B0A43EAC25303F136
:10E3D00040020C491344CEF80C2303EBC000CEF8E6
:10E3E00010334202CEF8F802C30DCEE9C711CEE9D0
:10E3F000BC238AE60123EAE7000001204403012050
:10E4000080510100E03101200068214C58B9050815
:10E410004CB905084019012010B58C18A14215D03F
:10E4200001F1FF3E013C41F2210C1EF8012F0823AF
:10E4300080EA022002B24000002A8CEA420180B247
:10E44000B8BF88B2013BF5D17445EED110BD00BF15
:10E45000704700BF2DE9F047002BDDF820A088466B
:10E4600007460CBF4FF020094FF030095646002AEE
:10E47000144616F8011B23DD11B3334601E0002CCE
:10E4800005DD13F8012B2546013C002AF7D1023D9A
:10E490003CB149463846C047013DFAD29AF80010CF
:10E4A00059B13846C047334616F8011B0029F8D148
:10E4B000A4EB0A041819BDE8F0872046BDE8F087F0
:10E4C000002C04F1FF35E4DC00240029E9D1F4E755
:10E4D00003685A1C02601970704700BF10B56FF0D6
:10E4E00000440246044404E0B3EB0E0015D1A242FE
:10E4F00014D012F8013BA3F14100192811F8010BC7
:10E50000A0F1410C98BF203300F1200EBCF1190F8F
:10E51000EAD91B1A04D10028E9D110BD002010BD92
:10E52000184610BD0378202B03D110F8013F202B93
:10E53000FBD0092BF9D02D2B63D02B2BB7EE000A83
:10E5400008BF01300278A2F13003D9B2092961D89D
:10E55000F2EE046ADFED4D7A07EE103A10F8012F63
:10E56000B8EEC77AA2F13003D9B2A7EEA67A09298C
:10E57000F0EE477AF0D92E2A50D0037803F0DF036B
:10E58000452B3BD110B442782D2A73D02B2A62D070
:10E59000A2F130030130092B63D80024002303EBE0
:10E5A000830302EB430310F8012FA2F13001303B4B
:10E5B0000929F4D9B3F59A7F1A46B7EE007A28BF35
:10E5C0004FF49A72072B09D91346DFED316A083BE5
:10E5D00027EE267A072BFAD802F007022AB1F2EECC
:10E5E000046A013A27EE267AFBD1002C3BD0C7EE15
:10E5F000877A5DF8044B20EE270A704720EE270A41
:10E60000704742780130BFEE000AA2F13003D9B260
:10E6100009299DD92E2ADFED1D7AAED1437801302C
:10E62000A3F13002D1B20929A8D8B2EE047AF0EEF3
:10E63000475A06EE902A10F8013FB8EEE66AA3F1B9
:10E640003002D1B2C6EE076A092927EE257A77EEA5
:10E65000A67AEED992E782780230A2F13003092B34
:10E660009BD9B7EE007A67EE877A5DF8044B20EE0F
:10E67000270A704782780230A2F13003092B01D8B3
:10E6800001248BE7B7EE007AB1E700BF000000007D
:10E6900020BCBE4CF8B5164D6B78BE2B25D1AC1CFA
:10E6A000144F022229464FF6FF70FFF7B5FE22886D
:10E6B0004AB1A618BE4218D2052A16D921463446B8
:10E6C000FFF7AAFEF3E721460222FFF7A5FE02228A
:10E6D000A1180634FFF7A0FE074B641B1C8041F60F
:10E6E0000F53C31A58425841F8BD0020FCE700BF41
:10E6F000004000080080000878500120F0B506793D
:10E7000006F0E003402B03D145794FF0FF3406E0DB
:10E71000602B4FF00105F8D1447905FA04F4002389
:10E72000012006F00706AB4200D1F0BD052E0FD840
:10E73000DFE806F00308101D242448B1C85CD75C4C
:10E7400078400FE020B1C856D756C71B78427841B1
:10E750000133E8E70028FBD031F8130032F81370DA
:10E76000784080B220420CBF01200020F0E7002852
:10E77000EED031F9130032F91370E6E70028E7D044
:10E7800051F8230052F82370DAE7037903F01803F5
:10E79000102B1DD003D833B9B0F80B007047182BDD
:10E7A000FAD000207047114BB0F80B0093F90030FD
:10E7B000591C0BD10E4B1B7903EB430203EB820375
:10E7C00003EBC30300EB430080B27047DBB2F3E717
:10E7D000064BB0F80B0093F901305A1C04D1044BDE
:10E7E0005B7900EB4310EFE7DBB2FAE77803012037
:10E7F00078500120032870B518D80D4BC943C600C6
:10E8000003EBC00001F00101057E427E81EA0504B0
:10E81000A2420BD042693AB14D1B106892886942FE
:10E82000694109018A40826133445C7670BD00BF52
:10E83000785001200379062B0FD1C9B20D290AD8CF
:10E84000074B59560123C2688B40134214BF084638
:10E850004FF0FF3070470021F4E7481C704700BFBD
:10E8600060B90508092917D0B1FA81F35B0999B19C
:10E87000013903604A0001F0030102F00802C1EB14
:10E8800001119300C1EB0111A3EB92038900C3EBCB
:10E89000031381809B004380704700BFB5EEC00A20
:10E8A000DFED357A0023F1EE10FA30B5C8BF30EE57
:10E8B000270A87B0D8BF30EE670ADFED307A054609
:10E8C00003A9029320EE270ACDE90033FDEEC07ABA
:10E8D00017EE904A84EAE470A0EBE4703BF0C0FECF
:10E8E000002C03A8B4BF2D2320238DF8003042F064
:10E8F0007DFA01282AD0022834D003281ED003A98B
:10E90000684644F053FB684642F070FA0446694694
:10E910002846033CE4B2224644F0E8FA00232846A5
:10E920002B5542F063FA2E22431C0DEB04012A54AE
:10E93000E81844F068FB284607B030BD302303A92F
:10E9400068468DF8013044F031FBDCE743F23002D9
:10E95000302303A96846ADF801208DF8033044F058
:10E9600025FBD0E743F2300303A96846ADF8013038
:10E9700044F01CFBC7E700BF6F12033A00007A4463
:10E9800009F0CABF38B5054658B14C1E14F8011F2E
:10E99000284619B9BDE8384009F0D2BF09F0BCFFDC
:10E9A000F4E738BD70B50546B0F8090037F0E8FA6D
:10E9B000064B0446284693F83460FFF7E6FE16B18E
:10E9C000E368184470BDA368FBE700BF78500120DE
:10E9D00038B505460C46FFF7E5FF2A7902F0070334
:10E9E00002F0E002602A29D1052B0CD8DFE803F001
:10E9F000030B0F0B1B1B6A79012393400278DBB2D8
:10EA000014B11343037038BD22EA0303FAE76A79AD
:10EA10000123934002889BB214B113430380F2E7B1
:10EA200022EA0303FAE76B7901229A40036814B1E2
:10EA300013430360E7E723EA0203FAE7052BE2D872
:10EA4000DFE803F00303050507070470DBE7048034
:10EA5000D9E70460D7E708B5202144F0B6FA0346A9
:10EA600018461BB102780133202AF9D008BD08B539
:10EA7000CB0701D4FDF75AF808BD2DE9F341002377
:10EA8000124D044600EB8106114F05F8353FB442A4
:10EA900003D1104802B0BDE8F081394628464FF056
:10EAA000000844F083FA2146684644F0ACFA20217D
:10EAB000684644F08AFA28B969462846043444F086
:10EAC00075FAE4E780F80080F1E700BF7850012094
:10EAD0008A380608AD5001202DE9FF4791460446CB
:10EAE0008A461E46FFF7A6FE421CBDF8307005465A
:10EAF000DDF834801FD0B9F1FF3F1FD0154A3146F1
:10EB0000CDE9000938462368C0474A465FFA8AF1D2
:10EB10002079FBF713F8024600B10288D3B23146E0
:10EB200038460393C2F30323120B0293CDE900523C
:10EB3000094A2368C04704B0BDE8F0877B06FAD4D1
:10EB40000C90314623683846044AC44604B0BDE8F8
:10EB5000F0476047A2280608AF280608D328060811
:10EB60002DE9F043154685B0894619466A1CBDF863
:10EB700030600D9F25D04FEA101800F00F04184A9E
:10EB8000304608F14008CDE900454346B847A8B1F2
:10EB90002A4699F80510D9F80000FBF711F868B17A
:10EBA00003880021027830460392C3F303221B0B33
:10EBB00002920C4ACDE900434346B84705B0BDE890
:10EBC000F0837306FAD4030900F00F00064ABC462E
:10EBD0000C904033304605B0BDE8F043604700BFBD
:10EBE000E2280608F42806081D29060808234840DC
:10EBF00041B240000029C0B2B8BF5040013BF7D13C
:10EC0000704700BF30B5056804468D4218D901F140
:10EC1000FF3E681E00231EF801CF082183EA0C0383
:10EC20004FFA83FC5B00BCF1000FDBB2B8BF53406E
:10EC30000139F5D17045EED16A1C22602B7030BDD0
:10EC400000236A1C22602B7030BD00BF9FED067A46
:10EC5000F7EE007A60EE870A60EE800A30EEA70ACF
:10EC600080EE800A704700BFDB0FC940DFED2D0A40
:10EC700008B543F031FCDFED2C7AB4EEE70AF1EE93
:10EC800010FA28DDDFED276A9FED287AF0EE407A52
:10EC900030EE660AF4EEC77AF1EE10FAF6DCDFED3C
:10ECA000247AB4EEE70AF1EE10FA2FDDDFED1E7ADA
:10ECB00037EEC00A20EE007A9FED1E6ADFED1E6A75
:10ECC000DFED1E7AE7EE066A20EE076AE6EE877A47
:10ECD000A6EE270A08BDDFED1A7AB4EEE70AF1EED8
:10ECE00010FADCD5DFED0F6A9FED167AF0EE407A70
:10ECF00030EE260AF4EEC77AF1EE10FAF6D4DFED24
:10ED00000C7AB4EEE70AF1EE10FACFDCDFED0E7A02
:10ED1000B4EEE70AF1EE10FACCD5DFED097A37EE62
:10ED2000C00AC7E7DB0FC940DB0F4940E4CB1641FF
:10ED3000DB0FC93F92E741B99730083C15A82ABEBE
:10ED4000DB0F49C0E4CB16C1DB0FC9BF10B5B7EE6E
:10ED5000001A0022DFED050A044644F0D9FC002326
:10ED6000A36163612362E36110BD00BFF304353F1B
:10ED7000B0EEC07AF0EEE06AF0EE407AC6FE875A56
:10ED8000F5EE405AF1EE10FA3BD086FEC75A85EEFA
:10ED9000256A9FED1D2A9FED1D3A9FED1D4ADFED6F
:10EDA0001D4ADFED1D2AF7EE005ADFED1C3A9FEDFC
:10EDB0001C5AA6EE423AE6EE223AA6EE034AE6EEE8
:10EDC000235AE6EE044AA6EE245A85EE250AF4EE0E
:10EDD000C76AF1EE10FA03D59FED127A37EE400ABA
:10EDE000F5EEC00AF1EE10FA03D59FED0F7A37EE7B
:10EDF000400AF5EEC07AF1EE10FA48BFB1EE400AD3
:10EE000070479FED070AE2E739094E3DE3B59E3EA4
:10EE100088FA163E45FE7F3F99FB243F69A2163EC5
:10EE2000A7DFA834DB0FC93FDB0F49402DE9F04FC6
:10EE30001646884689B016F8011B002900F0438267
:10EE4000144607469B46002509E0013534463846FE
:10EE5000C047264616F8011B002900F0908025299E
:10EE6000F3D16178302900F08E8002340023A1F1C3
:10EE7000300C5FFA8CF2092A4FF0000260D96C293D
:10EE800000F085807829E4D8572940F2E880A1F184
:10EE900058002028DDD801A656F820F07BF00008A5
:10EEA00053EE000853EE000853EE000853EE00083E
:10EEB00053EE000853EE000853EE000853EE00082E
:10EEC00053EE000853EE000835F000082FF100085B
:10EED00053EE000853EE000853EE000853EE00080E
:10EEE00053EE000853EE000853EE000853EE0008FE
:10EEF00053EE000857F0000853EE000853EE0008E8
:10EF000053EE000853EE000843F0000853EE0008EB
:10EF10008FF1000853EE000853EE00087BF0000864
:10EF2000BEF1050F18D9B9F1050FA8D80A2E17D1CF
:10EF300002EB820214F8011B06EB4202A1F1300C35
:10EF40005FFA8CF0A1F1610EA1F14109A1F1370640
:10EF50000928E5D86646EBE7A1F157060A2EE7D067
:10EF6000572994D825297FF474AF264625213846A1
:10EF70000135C04716F8011B00297FF470AF284601
:10EF800009B0BDE8F08FA178012303346FE714F8CE
:10EF900001CBBCF1780F3FF65CAFBCF1570F64D9E1
:10EFA000ACF1580120293FF654AF01A050F821F0F0
:10EFB000DDF0000853EE000853EE000853EE0008A1
:10EFC00053EE000853EE000853EE000853EE00081D
:10EFD00053EE000853EE000853EE000835F0000829
:10EFE0003FF2000853EE000853EE000853EE00080D
:10EFF00053EE000853EE000853EE000853EE0008ED
:10F0000053EE000853EE000857F0000853EE0008D6
:10F0100053EE000853EE000853EE000843F00008DA
:10F0200053EE0008E5F1000853EE000853EE000827
:10F03000DDF000085BF8041B38460135C9B2C04753
:10F0400007E75BF8040B0023414600903846FFF7C2
:10F0500001FA0544FDE65BF8043B1D60F9E6002972
:10F0600080D1284609B0BDE8F08FBCF1000F86D0F2
:10F07000BCF1250F3FF479AFEBE65BF804EB012020
:10F08000BEF10F0F40F221810001BEFBF0F60F2E02
:10F09000FAD8002800F01D810DF1140AD14601E0D4
:10F0A000BEFBF0F6092E4FF0300C05DD58290CBFE1
:10F0B0004FF0370C4FF0570CB44400FB16EE00092C
:10F0C00009F801CBECD1002189F8001041463846FF
:10F0D000CDF800A0FFF7BEF90544BAE65BF8049B43
:10F0E0000121B9F10F0F40F2F2800901B9FBF1F0F3
:10F0F0000F28FAD8002900F0E2800DF1140AD64654
:10F1000001E0B9FBF1F009284FF0300604DDBCF155
:10F11000580F0CBF37265726064401FB10990909E2
:10F120000EF8016BEDD100218EF80010CEE75BF8F0
:10F13000046B002EC0F2BA800DF1140AD646092ED7
:10F14000B4464FF0010108DD01EB81014900B6FB37
:10F15000F1F00928F8D80029E5D0DFF88091039371
:10F16000A9FB0163BCFBF1F00A284FEAD30301FBC2
:10F1700010CCB4BF302657260929194606440EF88C
:10F18000016BEDD8039B00218EF800109EE75BF821
:10F19000040B0121092809D901EB81014900B0FBC9
:10F1A000F1F6092EF8D8002900F089800DF1140A33
:10F1B000DFF828910393D646A9FB01C3B0FBF1F613
:10F1C0000A2E4FEAD30301FB1600B4BF4FF0300CF8
:10F1D0004FF0570C09291946B4440EF801CBEBD86F
:10F1E000039BD0E75BF8040B0121092808D901EB48
:10F1F00081014900B0FBF1F6092EF8D800295ED054
:10F200000DF1140ADFF8D4900394D646A9FB01C48B
:10F21000B0FBF1F60A2E4FEAD40401FB1600B4BF8E
:10F220004FF0300C4FF0570C09292146B4440EF82A
:10F2300001CBEBD8039C00218EF8001046E75BF869
:10F24000040B002829DB0DF1140AD64609284FF0DB
:10F25000010109D901EB81014900B0FBF1F6092E4A
:10F26000F8D800293FF45FAFDFF870900394A9FB52
:10F2700001C4B0FBF1F60A2E4FEAD40401FB1600DC
:10F28000B4BF4FF0300C4FF0570C09292146B4445D
:10F290000EF801CBEBD8039CCDE72D2140420DF1B8
:10F2A000150E0DF1140A8DF81410CFE72D217642BA
:10F2B0000DF1150E0DF1140A8DF814103FE70DF144
:10F2C000140AD6462FE70D4659E67646E4E6484648
:10F2D00013E70DF1140AD146F5E600BFCDCCCCCC36
:10F2E000F8B5114C07460D461646A06DA0B10F4962
:10F2F000FFF748FB3946A06DFFF744FB0C49A06DB2
:10F30000FFF740FB0B4933462A46A06DFFF78EFD01
:10F310000949A06DFFF736FB94F85C3013B1012367
:10F3200084F85D30F8BD00BF78500120312906080F
:10F33000853F060881E900083E2906080EB400B59D
:10F3400084B0084905AB019001A853F8042B03933E
:10F35000FFF76CFD0022019B1A7004B05DF804EB0E
:10F3600003B07047D1E40008F7B5114E07460023FB
:10F370000C46304615460F495E3600F85E3F04EBFA
:10F3800045050D4B002F18BF19460C4F43F00EFEDC
:10F39000AC4202D10A4803B0F0BD394634F8022B22
:10F3A0006846FFF7CBFF6946304643F0FFFDEFE7C5
:10F3B000785001204B2906084229060854290608DE
:10F3C000D6500120F7B500230B4E044600EB410553
:10F3D0000A4F06F88F3FAC4202D1094803B0F0BD96
:10F3E000394634F8022B6846FFF7A8FF69463046D5
:10F3F00043F0DCFDEFE700BF78500120F829060854
:10F4000007510120F8B54E1E054601F11F04054FB6
:10F4100016F8012F284639460235FFF78FFFA6421E
:10F42000F6D1F8BD5929060802460846531C05D1F5
:10F43000034B1A681B790A600B71704701497DE71D
:10F44000DD280608F929060803685A1C02601970AD
:10F45000090A03685A1C0260197070470268134653
:10F46000511C016013F802CB0360D31C5178036078
:10F4700093781B0443EA0123111D43EA0C03016046
:10F48000D07843EA00607047A0F13003092B07D918
:10F4900020F02000413819288CBF0020012070473F
:10F4A00001207047303809288CBF002001207047A8
:10F4B000413819288CBF0020012070476138192875
:10F4C0008CBF00200120704720280BD0092809D0CC
:10F4D0000A2807D00D2805D00B3801288CBF002042
:10F4E0000120704701207047A0F14103192B98BFFC
:10F4F00020307047A0F16103192B98BF2038704766
:10F5000002B3844610B5841803E0981A15D1A445B7
:10F5100014D01CF8013BA3F14100192811F8010B8C
:10F52000A0F1410E98BF203300F12002BEF1190F67
:10F53000EBD91B1A04D10028E9D110BD002010BD61
:10F54000184610BD1046704770B5044608460D4673
:10F5500041F04CFC064602E014F8013F43B132464C
:10F5600029462046FFF7CCFF0028F5D1204670BD84
:10F570001C46204670BD00BF2DE9F0430646864676
:10F580009EF800C074460EF1010EBCF1200FF7D0BA
:10F59000BCF1090FF4D0BCF10A0FACF10B00EFD0B5
:10F5A000ACF10D05B5FA85F56D09002DE8D10128FE
:10F5B000E6D9BCF12B0F3DD0BCF12D0F39D0102A6C
:10F5C0003ED04FF0FF3E9046BEFBF2FE02FB0EF730
:10F5D000FF43FFB2002014F801CBBCF1390F4CF00F
:10F5E0002009ACF1300C0DD85FFA8CFC944510DA90
:10F5F0007045264602D819D1674517D21D404FF0F5
:10F60000FF30E8E7A9F1570CB9F1600F5FFA8CFC05
:10F61000ECD801B10E6003F00103D5B9002803DA7C
:10F62000002B18BF6FF00040BDE8F08300FB08C05E
:10F63000D1E70125102A94F801C004F10104C0D1DA
:10F64000BCF1300F10D06FF0704E0F274FF0100844
:10F65000C0E7B0F1004F04D91BB14FF00040BDE846
:10F66000F0834042BDE8F08360786FF0704E0F2762
:10F670004FF01008A0F14106192E04F1010698BFC1
:10F68000203078280CBF02343446A3E701230A2235
:10F69000002171E770B50D461446FFF7DCF9064608
:10F6A000A0B1FFF7F3FF40F6340319229842A8BF38
:10F6B0001846B0F5617FB8BF4FF46170A0F5617373
:10F6C000B3FBF2F32B702378013323703046FFF73E
:10F6D000C2F90646A0B1FFF7D9FF40F6340319225C
:10F6E0009842A8BF1846B0F5617FB8BF4FF461706B
:10F6F000A0F56173B3FBF2F36B70237801332370D1
:10F70000304670BD2DE9F04116461F46404D044677
:10F71000394630464FF47A72002341F0C5FF3D4B25
:10F7200005443D4F3D4E83FB0510E9172844C1EBCE
:10F73000601183FB0103C8170B44C0EB631087FB08
:10F74000003CC317C3EBAC0386FB03764FEAE37EB2
:10F75000CEEBE61EC1EB0116A5EB860CC0EB001547
:10F760004FEA8E0684F806C0A1EB8501617103EBB8
:10F770004301A0EBC10040F2B55101FB1E332071E3
:10F78000B3F5896F33DA40F2DA218B4237DCB3F517
:10F79000B77F234FB4BF4FF0000E4FF0010E0EEBBA
:10F7A0004E0175464FEA4E0807EBC101C88A08EBC7
:10F7B0000E0C0B2107EBCC0C0CF1160C01E03CF805
:10F7C000020D984210DD0139F9D1F044012137F8DA
:10F7D000380006F5FA6E0133A17075441B1A2281B8
:10F7E0002580E370BDE8F0810131C9B2F1E703255E
:10F7F00040F296500A4F4FF00608AE46D7E7022572
:10F8000040F22940064F4FF00408AE46CFE700BF54
:10F8100080BC92C789888888ABAAAA2A73B06D1663
:10F820003C4A05080D4B10B5D3E9004354EA0302E6
:10F830000AD10146002340F2011218460B80C1F89C
:10F8400002208B710B8110BD054A1268121943F119
:10F850000003FFF757FF012010BD00BF90290120D2
:10F86000141C01202DE9F041044615460846944237
:10F87000B4FBF2F607D205FB1644134B1B5D00F8F0
:10F88000013BBDE8F0819642B6FBF2F70CD20E4B7D
:10F8900005FB176705FB1644DA5D1B5D00F8012BBD
:10F8A00000F8013BBDE8F081BA42B7FBF2F807D996
:10F8B00005FB1878044B13F8082000F8012BE7E744
:10F8C0004046FFF7CFFFF3E77CB9050830B56D4C34
:10F8D00083B0B4F8E434B3F57A7F03D94FF47A7384
:10F8E000A4F8E434B4F8E634B3F57A7F03D94FF4DE
:10F8F0007A73A4F8E634B4F8E814B1F57A7F04D941
:10F900004FF47A731946A4F8E834B4F8EA04B0F571
:10F910007A7F03D900231846A4F8EA34B4F8EC340B
:10F92000B3F57A7F4AD94FF47A73B4F8EE249A4249
:10F93000A4F8EC3447D900238842A4F8EE3480F0D0
:10F940008B80B4F8FA24B4F8FC349A4202D900232C
:10F95000A4F8FA344C4B1B88EBB14C4DAA78062A1C
:10F960004ED9297900297AD19FED497A94F8042556
:10F9700007EE903AAB7906EE902AF8EEE77AB8EE09
:10F98000E66AC6EE276A0BB137EE077AB4EEE67A7E
:10F99000F1EE10FA42DC6279032A23D83D4B03EBE7
:10F9A00042132279C4F80C35032A14D8EA213A4BC1
:10F9B00002FB0133C4F8103503B030BDB4F8EE24B7
:10F9C000B2F57A7F16D8884210D29A42B9D3002372
:10F9D000A4F8EC34B5E700222F4B2271C4F810359F
:10F9E00003B030BD00222B4B6271DAE70021A4F88E
:10F9F000E814EAE700228842A4F8EE24E5D3F5E70C
:10FA0000264901EB820191ED187A29790029ADD0C0
:10FA1000531F032BBFD9002ABDD025E067EE877A9C
:10FA2000BCEEE77A8DED017A9DF8043007EE103ACE
:10FA3000B8EEC77AF4EEC77AF1EE10FA01DD0133C1
:10FA4000DBB2EBB1102BA8BF1023DBB2934238BF5F
:10FA5000134684F804359EE7A4F8E83471E7053AC4
:10FA6000032A98D99FED0A7AB7EE000A80EE070ABA
:10FA700042F064FD2B88834228BF03462B808AE72F
:10FA80000123E2E7785001209C1E00200C24012075
:10FA90006F12033830510120B05101203C4A050853
:10FAA0002DE9F04FC74E83B096F8143500AFA3F19F
:10FAB0001702022A00F2A382C34B7B6096F824351A
:10FAC0000024DFF830A33B60C04B03F15409984693
:10FAD000D8F800B01BF0010540F0788298F90410C6
:10FAE000142911D0584643F009FC1BF4003F00F0E4
:10FAF0006082012808D0082806DC002D00F0698209
:10FB00001BEA0A0F40F05882B049B14836F04EFA6D
:10FB10000023022086F8A83512F022FE96F8B035B0
:10FB2000D6F8AC55022B00F0EF82002800F03F839E
:10FB3000A84B4FF47A7E96F80DA64FF0000C03F513
:10FB40006A794FF0640B33F8082CB2F57A7FB3F87A
:10FB5000462088BF23F808ECB2F57A7F33F8062CEC
:10FB600088BFA3F846E0B2F57A7F33F8042C88BF4B
:10FB700023F806ECB2F57A7F02D9002223F804CCF0
:10FB800033F8061C9142B3F85A10B3F85C2098BFC2
:10FB900023F806CC914293F86B2003F1650102F142
:10FBA000FF3288BFA3F85AC0632A93F86C2002F191
:10FBB000010288BF83F86BB0D2B2092A4FF000026D
:10FBC00088BF83F86CC013F83200013211F8014F7E
:10FBD000844238BF81F800C0032AF4D1BAF1010F82
:10FBE00003F1EA0318BF03F864CC9945ABD1DFF801
:10FBF000089299F80230042B00F0B3822BB9B9F8BF
:10FC00000030B3F5F07F00F21882FFF75FFE724814
:10FC100096F82016FEF726FE103096F83F16FEF7EF
:10FC200021FEB6F84E26B6F84C361343B6F85026E9
:10FC300013431BB213B10123A6F85236674B2B4076
:10FC4000002B00F0C182E90700F174826A0400F120
:10FC5000F9812B0740F14582614AD6F800361540FC
:10FC60001340C6F8AC55C6F8003615F4004300F052
:10FC70001D82002386F82B3586F83B35E80440F1D9
:10FC80001F8296F85F36022B02D1012386F85F3679
:10FC9000DFF850A153460AF1780402E006339C4293
:10FCA0000CD01A780A2AF9D19978DA78914202D3DD
:10FCB0005A79002AF2D00A201CF06AFC00234FF483
:10FCC000806086F8A83512F04BFD002800F06282B3
:10FCD000444DAB469BF8051079B19BF8000050B13C
:10FCE000534602E006339C4207D01A788A42F9D183
:10FCF0005A79002AF6D01CF04BFC0BF1060B5C4540
:10FD0000E8D199F802A0BAF1080F00F0EF8196F857
:10FD10000D36D6F80026A3F10103C2F3C031B3FAC1
:10FD200083F386F8DF165B0986F8DC3696F80E3624
:10FD3000A3F10103B3FA83F35B0986F8E23696F880
:10FD4000E134032B02D9002386F8E1342649D6F8A2
:10FD5000AC350A400B40B17CC6F80026C6F8AC357D
:10FD6000002900F0F381B6F8F836002B40F0E4816A
:10FD7000D6F8FC36B3F5000F02D30023C6F8FC36E4
:10FD8000D6F80437194A1A401AB140F20223C6F8CD
:10FD9000043796F80037013B042B02D9012386F87B
:10FDA0000037AAF1050A124BBAF1030F93F8F48356
:10FDB00040F27281B8F1000F3AD000233B60DFF8C7
:10FDC0003CA024E0785001203C4A0508C855012099
:10FDD000D0870608BA510120A85601200960000208
:10FDE000FE9FFFFDDC560120BCD45518FDFDFFFF32
:10FDF0009C1E0020BC0202000C24012013240120C0
:10FE0000ABF1060BABEB090BD84540F21D81D34695
:10FE10001AF8010F0028F3D00AF0C0FD0028EFD037
:10FE200081798B07ECD53B680122002B40F01181D2
:10FE300099F8063013B1002389F80630B6F80E376A
:10FE400003F00F02042A03D8C3F30313022B03D9D0
:10FE50004FF42063A6F80E37B6F8103703F00F0200
:10FE6000042A03D8C3F30313022B03D940F601235A
:10FE7000A6F8103796F87D1796F8892796F87C37FC
:10FE8000914205D9002286F87D2753B1A6F8802734
:10FE900096F888279A4204D2002386F87C37A6F881
:10FEA000803796F87E2796F872389A4202D9002356
:10FEB00086F87E37DFF854C30CF1800B634679680F
:10FEC00013F8032D02EB42020A4492F834A292F88E
:10FED000359292F836E213F8010F99795045DA78A5
:10FEE000A8BF50464945A8BF494672451870A8BFEB
:10FEF000724663459971DA70EDD103F1200CDC454F
:10FF0000DCD1D6F84825002A00F00E81002001211E
:10FF100002E00635AC420ED02B782B2BF9D16B7852
:10FF2000043301FA03F31342F3D0063522EA030245
:10FF30000120AC42F0D108B1C6F84825A74C6D4667
:10FF400004F10808234602E0434500F0908013F8CE
:10FF5000012F072AF8D9002304F8013F0133082BA9
:10FF6000FAD1B6F80626AD46B6F804369A4202D360
:10FF70009B4BC6F804369B4BFF229B4C03F154006D
:10FF800086F8A42813F9082C142A05D053F80C1C61
:10FF900034EA010100F0E2800C339842F2D1934B35
:10FFA0005A79022A01D100225A710C37BD46BDE8A8
:10FFB000F08F01283FF79FAD08F10C08C1457FF491
:10FFC00087AD013C022C7FF6A3AD9DE50134E4B280
:10FFD00088E51BF0400F3FF497AD1BF4057F09D077
:10FFE0003B680F2BE8D0012BE6D0991E0529E3D9F9
:10FFF000102BE1D07E4931EA0B01DDD084E57D4A4A
:020000040801F1
:1000000011467A60DA0001EBC30393F87C1021B14A
:10001000D3F88030002B00F0B9807B68134493F84C
:100020007D20002A3FF44AAD93F85C31002B7FF429
:1000300045AD182386F8143540E54FF4F073A9F860
:100040000030E2E56C4A08E63B680022002B3FF4F2
:10005000EFAE99F81130002B7FF4F0AE99F805302F
:10006000012B3FF4E5AE002A7FF4E2AEE6E688B06D
:100070002022FF21E946484642F090FF574A04E01B
:10008000424549F823303FF46CAF12F8013F59F86C
:1000900023100131F4D05EE7002389F80430B8F171
:1000A000000F00F08F8001233B6088E696F82B2537
:1000B000002A3FF4E3ADE80486F83B353FF5E1ADB7
:1000C00029067FF5DEAD96F81425182A04D84B4B87
:1000D000D340DA073FF5D5ADDFF834A10AF1780453
:1000E000ECE5AC047FF5C1AD454AB6E599F80630BC
:1000F000002B3FF40CAE99F81130012B7FF407AEC2
:10010000022389F8113002E600283FF411AD90F97E
:1001100004404FF0FF0901E080F8089020460FF0FE
:10012000B5FD0028F8D103E52B201CF031FAD6F8F4
:100130004825EBE6334A90E596F8F4060AF02EFCE3
:1001400000287FF415AEA6F8F80611E62E490B43F9
:100150000A43C6F8AC35C6F8002604E686F8A4289B
:100160001DE7D6F8003625F4805523F48053C6F8F1
:10017000AC55C6F80036B9F82030B3F57A7FBFF435
:1001800044AD4FF47A73A9F820303EE5172386F882
:10019000143542E7D6F8AC3523F00063C6F8AC3529
:1001A000D6F8003623F00063C6F8003690E5D6F89E
:1001B000003625F0800523F08003C6F8AC55C6F85C
:1001C0000036B5E4424644E7D6F8003645F0080567
:1001D00043F00803C6F800363EE500BF1E240120A8
:1001E000AE014A01D4550120010002004C2C01202F
:1001F000400002003C4A0508F6DFFFFD0041000117
:10020000F6BFFFFDF79FFFFD0004050035510120FB
:10021000DC5601202DE9F04F9B4E9C4BD6F8B428BC
:10022000DFF8988202F2DC5243452DED028B83B059
:10023000C6F8B42880F02481DFF8849201229B461E
:10024000934D09F102070192B9F80210002900F05C
:1002500002817A18AA4280F0FE80052940F2FB80D4
:10026000BBF800003C46C0F30B000BE011881446BD
:100270000A44002900F0EF80AA4280F0EC800529B2
:1002800040F2E98061888142F0D161798B07EDD13C
:1002900023885846DBF8081094F804A0009335F042
:1002A00085FEBBF80010BAEB113F00F0DA800023A6
:1002B0000193BBF804100BF11C0B5BF8140CC1F399
:1002C0000B015BF8044C3AF0B3FDC3452060BBD38F
:1002D000D6F8AC356F4CC6F80036FFF7E1FB337942
:1002E000EA226D4D03FB0242A4F18003C6F81025FB
:1002F000727903EB4213C6F80C3517F02FFD4FF05F
:10030000FF33D6F810056B6020F03CFD1CF086F939
:1003100004F22C5304F2A45103E00633994200F096
:10032000AA801A78002AF8D19C78D878844202D31F
:1003300058790028F1D096F85C3664212A7203EBD4
:100340008303B6F86026554C01FB02F203EB8303EE
:10035000DFED538A8A424FEA8303B8BF0A468B42D5
:10036000C6F8B028B8BF0B46C6F8C8280022C6F8A1
:10037000AC3886F8CC2886F8CE28A4F51972494BFB
:10038000C3F8742500220023C4E90223C4E904232E
:1003900021F08CFFB6F9E2389FED437A08EE103A6F
:1003A000B6F8DE38DFED416A07EE903AB6F8DC3891
:1003B000B8EEC88AB6F8D058F8EEE77A96F8D28840
:1003C00028EE268A67EE877A38EE280AC4ED097A85
:1003D00007EE903AF8EEE77A67EE877AC4ED0A7A8C
:1003E000FEF744FCF0EE407AB0EE480AC4ED0D7A18
:1003F000FEF73CFCF1EE407A96F8E038B0EE680A81
:100400009FED2B7AC4ED0E7A07EE903AF8EEE77A7C
:10041000A7EE870AFEF72AFC07EE905ADFED256A61
:10042000F8EEE77A84ED0F0AC6F8F48886EEA77A2C
:1004300084ED107A2FF032F914F056FE1E4B012293
:1004400001981B6886F8CD28C6F8B43803B0BDEC17
:10045000028BBDE8F08FDBF80810584635F0A6FD9A
:1004600025E7009BA11D58469A1F35F0D5FD0028B1
:100470007FF41FAF1BE7F27C003A18BF01225AE756
:100480000123019324E700BF785001202887060844
:1004900000800008B0510120780301202859012074
:1004A000DB0FC93F9C1E002017B7D13888C3E43A40
:1004B00035FA8E3CC0C9FB48141C01200490060884
:1004C00000400008114B0122032810B5044683F8B0
:1004D0007C2505D9601CBDE81040C0B20BF0CEBE33
:1004E0000B4BEA2203F59C701C7104FB0200C3F85D
:1004F000100520F047FC1EF053FE1EF035FF601C77
:10050000BDE81040C0B20BF0B9BE00BF9C1E002079
:1005100078500120054B0121D3F8FC2883F8F81806
:1005200042F40012C3F8FC28704700BF7850012045
:100530002DE9F043D0F8008087B005460C46C8F39B
:100540000D03002B3FD1394A0120394E0221B2421E
:10055000CDE90233CDE904011ED3364B9A421AD3BA
:1005600003F580439A4222D3334B9A4221D903F5B3
:1005700080339A421FD903F500339A421DD903F5FF
:1005800000339A421BD903F500339A4219D905204A
:10059000FCF798FEFBE7034601A902A803933BF092
:1005A000CFF880B14FF0FF3007B0BDE8F0830B46C5
:1005B000F2E70323F0E70423EEE70523ECE7062345
:1005C000EAE70723E8E71D4ED4F8009096F81439BF
:1005D000012B09D0012386F814393BF053F8074664
:1005E00028B1002386F814396FF00100DCE7144CC1
:1005F000236923F440732361236943F40073236167
:10060000236943F001032361C8F80090BFF34F8FC3
:100610003BF038F8236923F00103236186F814794D
:100620000028E1D12B6804332B60BDE700400008AF
:100630000040000800800008FFFF000878500120FB
:10064000003C02402DE9F0415A4E8AB03378B12B7C
:1006500071D1FEF71FF880F00104E4B2564B04F0AC
:100660000104564DB3F84332554FADF80430BD4246
:1006700063D3002C00F09C8000230596CDE907335E
:100680000993504B9B1B06934F4B1A69002A05DABE
:100690004E4A5A6002F188325A601B694FF48073E7
:1006A000022201A905A8ADF8243040F0A1F80222E9
:1006B00001A94FF6FF70414DFDF7AEFE4FF0000867
:1006C0000446BD4249D30025022202A905A8ADF87F
:1006D000085040F08DF8022202A92046FDF79CFE4A
:1006E00040BA022203A9C043ADF80C0005A840F0AF
:1006F0007FF8089878B107ABC0F104022946184486
:1007000042F04CFC9DF9240018B907A905A8FFF791
:100710000FFF8DF824009DF8253023B12A4A136974
:1007200043F0004313619DF92400B0FA80F04009C2
:100730000AB0BDE8F081012490E7AB691C3535F8BB
:10074000181CD3F8008055F8140CC1F30B013AF0D3
:100750006FFB804518BF012489E7AE8803A905A86F
:100760008DF81180C6F30B061C35B31DADF80C30A7
:1007700035F81C3CC3F30B021B0BADF80E20062210
:100780008DF8103040F034F8062203A92046FDF71A
:1007900043FE044655F8141C324605A840F028F8DC
:1007A000204655F8141C3246FDF736FE044688E70D
:1007B0000120BDE7004000083C4A050828870608DC
:1007C0000490060800800008003C024023016745B1
:1007D00038B50324134DFFF763F9FFF733FF58B122
:1007E0002B78B12B08D1FDF755FF013C17D040B94C
:1007F000FFF728FF0028F3D1013CEED10520FCF7DC
:1008000061FD09490022094B0120096883F81C2970
:1008100083F8CD08C3F8B41883F81D2938BD002823
:10082000EFD1EBE700400008141C012078500120B4
:1008300010B5074A0124074B82F87C459C74FFF7EA
:10084000C7FFFFF7E7FC2046BDE810400BF016BDE0
:100850009C1E00207850012090F89230B7EE007A6C
:10086000DFED6A6A014607EE903A90F89630684AE2
:10087000B0EE476A05EE103A90F89430F8EEE77A59
:1008800004EE903A90F89530B8EEC55A05EE903ADD
:1008900090F8983067EEA67A04EE103A25EE265AC4
:1008A000F8EEE44AF8EEE55AB8EEC44A25EE275AC7
:1008B00064EEA64A65EEA65A24EE264A64EE854A00
:1008C00065EEA75A24EE274AB0EE473AF0B590F805
:1008D000917000F16F0602F11A050024137807EEFB
:1008E000903AF8EEE77A67EE857A67EE867AFDEE63
:1008F000E77A17EE903AFA2BA8BFFA2323EAE373BC
:100900000B72537807EE903AF8EEE77A67EEA47A26
:1009100067EE867AFDEEE77A17EE903AFA2BA8BFDB
:10092000FA2323EAE3734B72937803EE903AF8EEDE
:10093000E33A63EEA57A67EE877AFDEEE77A17EE83
:10094000903AFA2BA8BFFA2323EAE3738B729388B9
:1009500007EE903AF8EEE77A67EE847A67EE867AE9
:10096000FDEEE77A17EE903AD5ED007AB3F57A7F8F
:10097000F8EEE77AA8BF4FF47A7323EAE3738B812A
:100980002B68002B3FDD90F89730B0EE436A02EE03
:10099000903AF8EEE22AA2EEE66A63EE863A83EE39
:1009A000A76AA2EEA66A65EEA77A013467EE877A97
:1009B00067EE867AFDEEE77A17EE903AFA2BA8BF3B
:1009C000FA23BC4223EAE37306F8013F00DDF0BDE1
:1009D000012C13D190F8933007EE103A90F89B3029
:1009E00006EE103AB8EEC77AB8EEC66A27EE267A57
:1009F00026EE266A0435083208316FE7B7EE007A32
:100A0000B0EE476AF6E7B7EE006ACCE70AD7233CB8
:100A1000824C050890F899306BB3B0F864308BB114
:100A200090F89A20642102EB8203C3EB0313B3FB1B
:100A3000F1F3A0F86430962312FB03F3B3FBF1F358
:100A4000A0F8663043884BB190F89A30642203EBEB
:100A50008303C3EB0313B3FBF2F34380B0F85030CE
:100A60004BB1962290F89A3013FB02F36422B3FB49
:100A7000F2F3A0F85030704790F821304BB3438B1D
:100A800083B190F82230FA22642113FB02F203EBC7
:100A90008303B2FBF1F2B3F57A7F4283A8BF4FF430
:100AA0007A738383838843B1FA2290F8223013FB50
:100AB00002F36422B3FBF2F38380C3884BB190F856
:100AC000223003EB8303B3F57A7FA8BF4FF47A7328
:100AD000C380704770B50B4C002504F56A7694F816
:100AE000913013B12046FFF7B7FE20460135FFF7DE
:100AF00091FF3046FFF7C0FF042D04F1EA04EED168
:100B000070BD00BFB051012010B5064C4FF480728B
:100B1000002104F61E1042F041FA0023C4F8203AE6
:100B200010BD00BF78500120034BD3F8240A08B150
:100B300007F006BF704700BF7850012008B50B468C
:100B400005490246D1F8240A28B10449FEF76EF996
:100B5000BDE80840E8E708BD7850012081E90008B9
:100B6000024B0146D3F8240AFDF70CBF7850012050
:100B70000048F5E7103506080CB4C30607B500D5E4
:100B800061B905A904980191FFF7D8FFFFF7F0FFBD
:100B9000012003B05DF804EB02B070470020F8E7D5
:100BA00008B5FFF7DDFFBDE80840E1E710B50446F2
:100BB0000348FFF7D5FF2046BDE81040F0E700BF2F
:100BC0005E29060810B508460749FDF787FC00288E
:100BD00015BF0124002405480548FFF7E7FF20461C
:100BE000BDE8104007F018BB632906086C29060809
:100BF00093290608034B0146D3F8240A08B107F0ED
:100C00008BBE7047785001200CB407B510F020005F
:100C10000BD079B92320FFF7EDFF05A904980191C6
:100C2000FFF78CFFFFF7A4FF012003B05DF804EB92
:100C300002B070470020F8E70FB407B504A951F8D7
:100C4000040B0191FFF77AFF03B05DF804EB04B0E9
:100C50007047194B1B682DE9F04153B30025174F1E
:100C6000DFF864801648FFF79BFFFFF75DFFFCF796
:100C7000D3FDFCF707FE044640B113200BF0CEF87D
:100C8000FFF776FF0F48BDE8F04189E73B78012B7D
:100C9000F3D040466E1CFFF7CFFF792D02D12646D8
:100CA000FFF766FFFFF740FF64203546FCF7EEF9DB
:100CB000DFE7BDE8F08100BFDC1B01208A290120AD
:100CC000AF290608C9290608254406080FB407B548
:100CD00004A951F8040B0191FFF730FFFFF748FF1B
:100CE00003B05DF804EB04B070472DE9F0410379DF
:100CF00003F0E002402A4AD009D82ABB03F00703D8
:100D0000052B1CD8DFE803F0161B161B090F602A01
:100D100044D0802A3ED0BDE8F081D0F805102148AB
:100D2000BDE8F041D2E7D0F8052051421E48BDE8A9
:100D3000F041CBE7B0F80720B0F80510F6E7B0F9BE
:100D40000720B0F90510F1E746790024174D18483F
:100D500005EBC605FFF704FF012395F87072A74263
:100D600002D8BDE8F04103E7D5F86C624FEA840889
:100D700056F824204AB113B90E48FFF7F1FE56F891
:100D800008100D48FFF758FF00230134E7E74179C9
:100D90000A48C5E7827941790948C8E70948BDE8AA
:100DA000F04193E7CF290608E52906083C4A0508E3
:100DB000FC290608502C0608423F06080D2A0608A2
:100DC0001E2A0608352A06082DE9F04385B0224E72
:100DD000FCF712FD0269838900250188044602920E
:100DE0008268DFF8888001924288DFF884901B4F88
:100DF000009242681A48FFF769FF15B91948FFF7D2
:100E0000CFFED8F800309D4212DA3378052B20D877
:100E100009EB8303D3F83424B388294601353846D7
:100E20000093063636F8043CFFF750FF062DE4D158
:100E30003AF0C8FB4288838864689B1A03FB044429
:100E4000FCF76CFD02460848214605B0BDE8F043BA
:100E50003CE70022E0E700BFA05A0120B72A0608BD
:100E60004D2A0608AB2A0608C62A06088029012052
:100E70003C4A05080249034801F521610EC925E7EE
:100E80000070F01FE32A060870B50022124C134DC3
:100E9000134E94F8033503F0010302B170BD002B2B
:100EA000FCD001212846FFF711FF752021F074FEC8
:100EB00001463046FFF70AFF1A2021F06DFE014679
:100EC0000848FFF703FF1B2021F066FE0146064895
:100ED000FFF7FCFE0122DCE778500120F72A060824
:100EE000032B0608162B0608292B0608BD4BBE4906
:100EF0001A68BE4BBE482DE9F047BE4C90B0BE4DBF
:100F00004FF00008BD4F4646B2FBF3F2FFF794FEE8
:100F1000B4F84C2A4FF47A730A20B2FBF3F103FBC6
:100F20001122B4F94E3A92B2B2FBF0F2B448FFF794
:100F3000CDFEB44AB449B548FFF77EFEFFF718FE70
:100F4000A17CB34A05EB8101B24BB348D31AD1F867
:100F50004C142288FFF7BAFEFFF70AFEAF48FFF7EE
:100F6000FFFD94F8501AAE48FFF766FEAD48FFF754
:100F7000F7FDB4F8522A94F8541A92B2AA48FFF72F
:100F80005BFEFFF7F5FDA949A948FFF755FEDFF81D
:100F9000149394F8FF3403F00103B8F1000F00F04C
:100FA000EA80002E40F01B81A248FFF7F9FDA24F16
:100FB0000126D4F85C8ADFF8F09207F1180A0123C1
:100FC000B34013EA080F15D019F8062057F8263059
:100FD0005AF8261053F822209848FFF72DFE012ECC
:100FE00006D1864B93F89D1511B19548FFF724FE65
:100FF000FFF7BEFD0136062EE1D19248FFF7B0FDA6
:10100000D4F800361B0640F1828194F87C3A032B19
:101010008CBF8D488D48FFF7A3FD94F8B035022BA7
:1010200040F044818A48FFF79BFD94F87C3A042BFA
:1010300000F264818748FFF793FD94F88C3A002B07
:1010400000F0638105EBC303D3F828158248FFF74E
:10105000F3FDFFF78DFD94F8943AD4F8906A05EB10
:1010600083037E48D3F85C15FFF7E6FD26B1327A9C
:10107000717A7B48FFF7E0FDFFF77AFDFCF7BCFBD8
:10108000016921B182687748120DFFF71FFEFFF753
:101090006FFD754B754819684FF47A73B1FBF3F126
:1010A000FFF7CAFD05A8FEF7BDFB38B105A908A8E2
:1010B0003FF04EFD08A96E48FFF7BEFDFFF758FD53
:1010C000D4F8208BB8F1000F00F0258107EE908A4C
:1010D000DFED686AB8EEE77AC6EE877AFDEEE77A6A
:1010E00017EE903A644F97F8200130B1634A0393AA
:1010F00092ED050A41F022FA039BD4F8A06A5EB192
:1011000007EE906ADFED5B6AF8EEE77A86EEA77A83
:10111000FDEEC77A17EE906A384AB2F8EC154246EF
:101120006429CDE90006A8BF64215548FFF7CEFD2C
:10113000B7F8242164235348534EB2FBF3F103FB69
:10114000112297F8353105EB830592B2D5F8703549
:101150000125009397F83431FFF7B8FD4B48FFF7AE
:10116000FFFCD4F8FC48002C40F0D780FFF700FDCE
:1011700010B0BDE8F087002B3FF413AF16B148461E
:10118000FFF7EEFC01214248FFF756FD94F8583A6C
:101190003D4805EB8303D3F85414FFF74DFD97F852
:1011A000CE33DA0702D53B48FFF746FD97F81831F2
:1011B000032B09D03848FFF73FFD97F81831012B72
:1011C00002D13648FFF738FDFB6C01265B7BB04649
:1011D000B3427FF6DEAE3248FFF72EFDD7E6FFF7CB
:1011E000C7FCE4E66C1C0120442B060840420F00BB
:1011F0004E2B0608785001203C4A05089C1E002012
:10120000602B06080000012000080000822B060861
:101210000080000800400008942B0608AB2B06084D
:10122000BD2B0608C52B0608C72B0608DB2B0608B6
:10123000E02B0608FF2B0608F04E05082F42060893
:10124000042C0608082C06080E2C06081A2C060882
:101250002A2C0608604406086E2C06088A2C06080C
:10126000932C06089D2C0608141C0120B82C060897
:10127000D22C0608002474497061012078030120F3
:10128000E52C06082B2D06087A2C0608502D06089A
:10129000E52B0608303F0608EA2B0608F22B060865
:1012A000F72B0608502C060884030120022011F0B9
:1012B00075FA064608B92048B5E690F9040039F0F9
:1012C000B9F907462EF0D4F905EB80003946D0F87D
:1012D000E4241A48FFF7B0FC94F8B335012B04D18D
:1012E0001748FFF73DFC17489DE6B379164805EB14
:1012F0008303D3F8E414FFF79FFCF4E794F8B235C6
:101300000BB9124897E6124895E612499EE6124834
:10131000FFF726FC9DE64346E4E694FAA4F0B0FA13
:1013200080F005FA00F024EA00040AF05DFD0146B1
:101330003046FFF781FC16E7302C06083A2C0608E9
:101340004A2C06084F2C060880370608532C06083E
:10135000632C06083C2B06087E2C06082DE9F04F6E
:10136000DFF86C8199B098F80730002B00F093807B
:101370004E4800254E4EDFF85CB1FFF711FC2F46BA
:10138000DFF85491DFF854A10BA9E8B215F09EFEE6
:101390009DF83430002B53D0139C54B107EE904A83
:1013A0009FED440AF8EE677A80EE270A41F0C6F80E
:1013B00004460B9A29465846FFF73EFC109A002A2D
:1013C0006BD002FB04F04FF47A73B0FBF3F3099394
:1013D000DDF848C0BCF1000F61D00CFB04F142F213
:1013E0001073B1FBF3F1082D98F8073018BF7F1880
:1013F000002B56D017984FF47A7E0A230790159841
:101400000690169805901198B0FBFEFECDF810E0FE
:101410000998B1FBF3FE03FB1E11CDE902E1099926
:10142000B1FBF3F103FB1100BCFBF3F3CDE90010BA
:1014300021465046FFF74AFC0023B362C6E90D334C
:10144000013540361E2D9FD198F8073003B31A4C52
:101450004FF47A731948D4E94E12B1FBF3F3D20872
:10146000D4F84011FFF732FC0A22154897FBF2F13D
:1014700002FB1172FFF72AFC124B1B78432B04D19D
:101480001148D4E95121FFF721FC0023C4F8403171
:1014900019B0BDE8F08F0D486BE7099298E76146F7
:1014A000A1E721464846FFF711FCC5E7662D06086F
:1014B000105B01208096184B706101200D2E0608EC
:1014C0002D2E0608B1280120512E0608C42D06082D
:1014D00078500120CE2D0608DE3E0608DD2D0608D8
:1014E000234870B5FFF73CFB224B93F82031002BCB
:1014F00038D0214B93ED050A41F020F801461F48F2
:10150000FFF7E4FB1E4C1F48FFF72AFB1E4B94F825
:101510003D051E4A00280CBF10461846FFF740FB49
:1015200094F83D3513B31A4C1A48B4F88216FFF7F5
:1015300083FB194E94F88006184D00280CBF3046E6
:101540002846FFF72DFBB4F884161548FFF774FB07
:1015500094F8810600280CBF30462846BDE870404C
:10156000FFF71EBB0F48FFF71BFBCBE770BD00BFAB
:101570008B2E06087061012078030120A52E060835
:1015800078500120B42E06084A2A0608FA490608AF
:101590009C1E0020C52E0608842E06087B2E0608F9
:1015A000EC2E0608AA2E06080EB403B503AA52F8BC
:1015B000041B0192FDF794FE064BD3F8242A1AB9B6
:1015C0000549986DFDF7DEF902B05DF804EB03B054
:1015D000704700BF78500120103506082DE9F0470C
:1015E00098460B7981460F4603F0E0051646402DDC
:1015F00032D10024634DDFF8A881DFF8B09116E006
:101600003B7903F00703013B042B04D8DFE803F028
:1016100014171A1D2100315D5A48FFF70DFB7B7925
:10162000013BA34202DD4846FFF79AFA01347B7979
:10163000A342E5DCBDE8F08731572846EDE736F8F0
:101640001410FAE736F91410F7E756F8241040465C
:10165000E3E756F82410F0E703F00703052B57D80B
:10166000DFE803F0031F27292C3E3478602D55D086
:101670002CD8002D75D1B7F80550B7F80760214672
:101680004048FFF7D9FAAC4239DBB44237DCB8F155
:10169000000FCFD0324629463B48BDE8F047FFF760
:1016A000CBBA96F90040602D38D00FD8002D58D114
:1016B00051E03488DAE7B6F90040F4E7D6F800A044
:1016C000202D54464DD034D9602D27D0802DB1D156
:1016D00032782E4B2E48002A14BF3146194635E089
:1016E000202D34683DD0EFD821462648FFF7A4FAD4
:1016F000D7F80510A14202DB4B42A34221DDFFF7E0
:1017000037FA23463A6848462249BDE8F0474BE796
:10171000202D25D01ED9602DD8D100247B7944FA04
:1017200003F3DB07BDE8F0474CBF1B481B48FFF73E
:1017300083BA51461A48FFF77FFAD7F805108A4551
:10174000DDD8B8F1000F3FF475AF1648BDE8F0479B
:10175000FFF772BA0024B7F90550B7F907608EE7B2
:1017600000247A79104B03EBC20393F87022A24253
:10177000C5DDD3F86C3253F82400BDE8F047FFF71D
:10178000EFB900BFF9290608723806085145060866
:10179000423F0608122F06084A2A0608FA49060898
:1017A000E22906080C2F06083C4A0508C52B060846
:1017B00070B5164605460C460846FDF7F3F8334665
:1017C000024621462846BDE8704007E70EB403B53F
:1017D00003AA52F8041B0192FDF782FD044B054950
:1017E000986DFDF7CFF802B05DF804EB03B07047D9
:1017F00078500120103506080049E7E72C2F06082D
:10180000F8B50C4606460846FDF740FF2021054680
:10181000204641F0DAFB044618B93046BDE8F840EE
:10182000EAE7114F0134114E3B7832789A4201D0E9
:10183000FCF76AF90E4B20461D603FF0D7FA0122F3
:1018400001462046FCF7FEF83B7832789A4201D0F8
:10185000FCF75AF920463FF0C9FA2A4601460548E6
:10186000BDE8F840FFF732BAD81B01208B290120D0
:10187000D41B0120432F06082DE9F0410D4688B006
:1018800006460846FDF702FF20210446284641F09F
:101890009CFB20B9304608B0BDE8F041ACE7FDF74D
:1018A000F5FE2246054601460F48FFF70FFA85B1BF
:1018B000202D2A466946204628BF2022E846FCF70C
:1018C0006BF900270646B74208DBAD1B3444002EF7
:1018D000EDD1FFF74DF908B0BDE8F08118F8010B24
:1018E0000137FFF787F9EEE7592F060810B50446D0
:1018F0000748FFF755F9FCF77FF920B10548BDE827
:101900001040FFF74DB920460349BDE810405DE7A0
:10191000712F06087B2F0608832F0608154BD3F876
:101920004C312DE9F041044688B0F3B11A6804A99E
:101930001846D56A6A46A847064688B104AC6D4683
:101940000027DFF83C80013735F8022B34F8021B02
:101950004046FFF7BBF9BE42F5DC08B0BDE8F081B8
:1019600005492046FFF732FFF7E7044908B0BDE814
:10197000F0412BE770610120A42F0608BC2F060858
:101980008A2F060870B5054608460C463FF02EFA29
:10199000024668B10D2804D12146084841F0EEFB0B
:1019A00030B12846054B064A0649BDE870400DE7B0
:1019B00002490548BDE87040FFF788B9C32F060803
:1019C000D12F0608DC2F06080630060870B505463C
:1019D00008460C463FF00AFA024668B1042804D1D2
:1019E0002146084841F0CAFB30B12846054B064A5B
:1019F0000649BDE87040E9E602490548BDE8704087
:101A0000FFF764B91430060819300608DC2F060801
:101A1000293006082DE9F04307469BB008460C46DE
:101A20003FF0E4F906462022002101A841F0B6FA71
:101A30002EB3402E07D0402332463A4938461BB0D9
:101A4000BDE8F043C2E601AD04F140084FF00009E3
:101A500002222146684641F0A3FB0023102209A977
:101A600068468DF80290FDF787FD099B0DF1020293
:101A7000934223D1023405F8010BA045E8D109AC0B
:101A800041220021284D204641F088FA002E3DD009
:101A900095F85061D6B1202205F2511101A841F00C
:101AA000D1FB98B105F251112046FDF7ABFC23465E
:101AB0001E4A38461E49FFF789FE04E01A78384668
:101AC0001C49FFF783FE1BB0BDE8F0831A4B93F867
:101AD0003430DBB9D6B901AB184E1A46083603CA02
:101AE000A24246F8080C46F8041C1346F5D101231F
:101AF0002046124985F87131FDF784FC1048FFF744
:101B000055F821460F48FFF7E1F8DCE795F8713109
:101B10001BB995F85031002BF3D008492046FDF74A
:101B200071FCEEE73C300608706101207A3006084F
:101B3000DC2F06085E30060878500120C1620120C3
:101B400084300608933006082DE9F74FDFF820812E
:101B5000834608460C463FF049F9D8F8AC7506466E
:101B600028B1024633492046FDF7CAFC80B9394600
:101B7000314838F0E5FC3149314821EA070138F0B5
:101B8000DFFC3049304803B0BDE8F04F38F0D8BC36
:101B900023782D2B23D10134013E4FF0010A2B4B2A
:101BA0004FF000094FF0FF3553F8041B51B1324696
:101BB00020460193FDF7A4FC0028019B0ABF4D4677
:101BC0000021012109F10109A1B9B9F11D0FEBD1E2
:101BD00022461F49584603B0BDE8F04FF6E54FF0E6
:101BE000000ADCE73B431B49C8F8AC351A4B12E04E
:101BF0001A4913E00123114AAB401A40002AF7D0DA
:101C000007EA0302BAF1000FECD027EA03031449F4
:101C1000C8F8AC35134B002A18BF1946124B1348AD
:101C200003EB8503D3F8842503B0BDE8F04FFFF73D
:101C30004DB800BFC92D0608CB300608BCD45518D6
:101C4000D5300608432BAAE7E1300608C04F050847
:101C5000EF300608C3300608BC300608A03006087E
:101C6000AC300608B33006083C4A0508B53706080C
:101C7000785001202DE9F74F019008460E4617468F
:101C800098463FF0B3F80446E8B93F4D3F48FEF7A9
:101C9000D3FF20460DF0A6FF3B68184206D0204631
:101CA0000DF0B2FF01462846FEF7C6FF0134172C9F
:101CB000EFD13B6813B93648FEF752FF03B0BDE8D9
:101CC000F04FFEF755BF024632493046FDF718FC8B
:101CD0000546A8B92C46304D3048FEF741FF204656
:101CE0000DF080FF10EA080F06D020460DF08CFFA3
:101CF00001462846FEF7A0FF0134182CEFD1DDE79E
:101D000033782D2B29D10136013C01254FF00009F4
:101D100048F4000B48460DF077FF22468246014604
:101D20003046FDF7EDFB18BB48460DF05BFF1BEAA4
:101D3000000F1DD09DB1B9F1170F02D03B6840EAEA
:101D400003081748C7F80080FEF70AFF51461248FB
:101D500003B0BDE8F04FFEF7B9BF0025D6E7B9F1F3
:101D6000170F02D03D6825EA00050E483D60EBE7FD
:101D700009F10109B9F1180FCCD132460A4901988D
:101D800003B0BDE8F04F21E5792C060800310608C4
:101D90000A310608C92D06087A2C060811310608F2
:101DA000B3300608C3300608EF30060840F20223BD
:101DB000004A5FE77C570120014B024A5AE700BF07
:101DC000FFFF7F007457012010B50446012020F06A
:101DD00035FA20B920460449BDE81040F6E403482E
:101DE000BDE81040FEF772BF1C3106082B31060813
:101DF000064B10B50446D3F874012DF0B1FB20B9A1
:101E000020460349BDE81040E0E410BD70610120A8
:101E10003631060870B5054608461646FDF736FC0D
:101E20000D4B041E93F8F4230EDB944205DA214691
:101E30000A48FEF74BFF204670BD2EB1FF2C03D1A0
:101E40000748FEF743FFF6E7013A064928464FF0F8
:101E5000FF34FFF7BBFCEEE79C1E00204C31060868
:101E60005D310608703106082DE9F04F074691B044
:101E700082480E46824DFEF729FF00238149402407
:101E8000062285F87C313046012391F8F413C5F819
:101E900078D185F87D4106F015FD0A20FBF7F6F8AC
:101EA00095F87C310C2BDAB240F2E4809DF80C609E
:101EB000FE2E2CD0FF2E15BF0F2415240025012542
:101EC000944240F0D780611E6846C9B232F016FED7
:101ED00004F140030DEB030414F8413C834240F04D
:101EE000C4806A1E9DF80D30012A12D903F01F0725
:101EF0005C0961376448FEF733FE022D39D0013C9E
:101F0000042C34D8DFE804F00B2D2F3331000225E8
:101F1000D6E79DF80E701E469DF80F40EAE75B4835
:101F20006C464FF00008DFF8BC91FEF739FEDFF891
:101F3000B8A1DFF8B8B15648FEF712FE08F1010863
:101F400014F8011B4846FEF777FEB8F10C0F16D0C7
:101F50000AFB08F3B3F1553FF0D85846FEF700FEF0
:101F6000ECE74C48DCE74C48DAE74C48D8E74C480B
:101F7000D6E700230DF11F008DF83F30D0E7FEF7C4
:101F8000F7FD022D3AD064223B464648B6FBF2F1FB
:101F900002FB1162C9B2D2B2FEF798FE85F00103CE
:101FA0005B42DBB2012B59D83F4A404B9DF81010E1
:101FB0003F4800290CBF114619463E4EFEF786FEEB
:101FC0009DF811103C4B3D4800290CBF3146194685
:101FD000FEF77CFE022D41D19DF812403848FEF7F5
:101FE000BFFD8CB1FF2C1FD00A233648B4FBF3F1A0
:101FF00003FB1142D2B2FEF769FE08E03A463146D1
:102000003148FEF763FECFE73046FEF7C9FD9DF885
:1020100013402E48FEF7A4FD44B1FF2C21D02146E9
:102020002B48FEF753FE04E02A48EEE72148FEF76E
:10203000B7FD0DF1130500241E4E1F4FDFF89480ED
:1020400015F8013F7BB1FF2B14BF3A4642462146AB
:1020500001342148FEF73AFE042CF1D111B0BDE85D
:10206000F08F1C48E3E73246F1E71C493846FFF79A
:10207000ADFBF3E71A48FEF793FDEFE7B63106082C
:10208000706101209C1E0020C7310608D23106086D
:10209000F8310608D9310608E1310608E9310608A9
:1020A0003C2B06080A3206089F31060896310608BE
:1020B00041320608A631060848410608583206088B
:1020C0005F32060873320608263206087B3206089D
:1020D000F9290608AA3106088B3206089632060846
:1020E000A632060859290608ABAAAAAA514506082D
:1020F0002DE9F84307460C46DFF8A49020463EF051
:1021000075FE064660B91E4B1E4893F814251E4BFB
:1021100003EB8203D3F8F415BDE8F843FEF7D6BD10
:10212000024649462046FDF7EBF960B1DFF86080D2
:10213000002558F8041BB1B9224638461349BDE8BA
:10214000F843FFF743BB124C124D1348FEF708FD4E
:1021500054F8041B19B12846FEF76EFDF8E7BDE8F8
:10216000F843FEF705BD324620460135FDF7C8F9B4
:102170000028DED1024B094C83F81455BEE700BF9E
:1021800078500120AF3206083C4A0508EF300608B7
:10219000345005087A2C060811310608984A0608BA
:1021A000C92D060838B50D460446052219492846AA
:1021B000FDF7A6F968B9184B93F85C2022B9012104
:1021C00083F85D2083F85C101448BDE83840FEF7C2
:1021D000E7BC032212492846FDF792F9A0B90E4D3B
:1021E00095F85C3063B195F85D304BB10D492046F0
:1021F000FFF7ECFA002385F85C3085F85D3038BDD8
:102200000948FEF7CDFCF5E720460849BDE838400F
:10221000FFF7DCBA9F40060878500120B932060863
:10222000F1410608CF320608063306081A330608BD
:1022300070B5194C054694F85C307BB194F85D306C
:1022400063B11649FFF7C2FA28461549FFF7BEFAEF
:10225000002084F85C0084F85D0070BD114B93F899
:102260007121B2B193F850219AB903F2511203F5DA
:10227000C07503F271161068083252F8041C2C461F
:10228000B24203C42546F6D1012283F8BB2109F0EE
:1022900067FA0120E1E700BF78500120CF3206083D
:1022A000293306087061012008B5034610460AB9B3
:1022B000002008BDDB0601D50029FAD0FEF776FC28
:1022C000F6E7F8B50D4E054696F8343093B9F8BDEB
:1022D00025B12388C3F30B039D4204D0A288D4E91F
:1022E000020140F003FE1C34BC42F1D3002386F807
:1022F0003430ECE7024C034FF6E700BF7850012082
:1023000028870608049006082DE9F04F164685B088
:10231000334C1A464FF00009A246CDE901010021D5
:102320003046FFF7C1FF06F0100300900393FEF75D
:10233000FBFB2379029A03F01803934203D0002A8F
:1023400044D1182B42D14FF00D0B0BFB09A3B3F86E
:10235000090033F015FE80462046FCF716FA0746C2
:10236000D8E90221024401442046FCF7C7F980F075
:1023700001010546009AC9B23046FFF795FF039B5D
:10238000009003B115BB0BFB09FBB3065AF80BB069
:102390000ED56DB959461348FEF74EFCD8F8082003
:1023A0002B4621463A440198FFF718F9FEF7E0FB67
:1023B00059460D48FEF740FCD8F80C200023214672
:1023C0003A440198FFF70AF9FEF7D2FB09F1010937
:1023D00040F262230D349945A9D105B0BDE8F08FD4
:1023E000A862050847330608483306080149FFF785
:1023F000EDB900BF5233060838B50C4605461549FD
:102400002046FCF76BF830B9FEF764FB1248BDE8D4
:102410003840FEF7C5BB11492046FCF75FF8A0B96C
:102420000F4B83F8C90183F8D10183F8B30283F815
:10243000BB0283F89D0383F8A50383F8870483F820
:102440008F0483F801050748E1E72846BDE83840D6
:10245000CCE700BF613306086733060882330608FD
:10246000785001208A3306082DE9FF4707460846C1
:102470000D463EF0BBFC082846D105F1FF3801AE01
:10248000073531464246B14612F8010FFDF732F8E2
:1024900001F8010BAA42F7D10023DFF880A08DF8E4
:1024A0000C30A84518D11C4948461FF059FE1A485F
:1024B00008231A4910F8012B013B11F8014B02F1D6
:1024C00010026A4402F80C4CF4D101A914488DF8AA
:1024D0000C30FEF7FBFB14E018F8010FFDF70AF8CB
:1024E0000446014606F8010B504640F06EFD28B147
:1024F0002146304640F069FD0028D2D03846FFF72B
:1025000075FF04B0BDE8F0870028D0D0384604B08D
:10251000BDE8F047FFF770B99455012094C805084D
:10252000A633060807B5009313460A460249FFF78B
:102530004DF903B05DF804FBAD33060820B1007817
:10254000B0FA80F040097047012070472DE9F74F3D
:1025500081460846FFF7F2FF0E46054670B100249B
:1025600001A92046013438F07BF801464846FFF7C0
:10257000EDFF122CF4D103B0BDE8F08F0846FDF753
:1025800085F8C4B2112C71D83C4D701CFCF763FA6D
:102590003B4E05EB44088346670098F8BCA1B8B9E8
:1025A000AAF102014B424B413D4495F8BC21B25C7B
:1025B000002B54D095F8BD31192040F2EE2100FBDC
:1025C000031321462F4803B0BDE8F04FFEF77EBB52
:1025D0000178304640F0F9FC80B1032C2A49A0EB89
:1025E000060394BF0022012202EB42020A4452FA7F
:1025F00083F393F868A6BAF1030F04D1484603B0F9
:10260000BDE8F04FF2E65846FCF725FAF0B1BAF112
:10261000020FF3D1FDF73AF840F6CA0380B29842B0
:10262000A8BF184640F2EE239842B8BF18461923B7
:10263000A0F2EE20B0FBF3F088F8BD01AAF102028F
:1026400053425341EA1982F8BCA1ADE7BAF1020F37
:10265000F4D1484603B0BDE8F04FFFF7CDB82146AE
:102660000A4803B0BDE8F04FFEF730BB11232A46FD
:102670000749484603B0BDE8F04F53E770610120B9
:10268000A4CA0508C63306083C4A0508D63306081E
:10269000E33306082DE9F04F0346A1B00846FFF7E3
:1026A0004DFF054628B1184621B0BDE8F04FFFF7B1
:1026B000A3B8FF23DFF8C09207464FF0FF388DF82C
:1026C0002830D9F874310B9093F83820ADF83000E9
:1026D0000D908DF838200F90ADF8400011930991BE
:1026E000CDE90500934909A840F00EFC044618BB4B
:1026F00001460AAC904F0B0190481A57002310F97D
:10270000016BB24240F0D2804E1C104637F092FF6F
:10271000024631463846FEF7D9FA022E4FF0010143
:10272000E9D19DF938A09DF92830534540F0C58086
:102730008348FEF7CBFA4DE02378002BD2D0032F4D
:10274000D4BF00260126062F00F2A980DFE807F09B
:102750000447509104475000042F10D07949204677
:10276000FCF7F2FE58B14FF4806010F017F8002823
:1027700000F0B58190F90400012306930AE0724944
:102780002046FBF7ABFE70B9D9F8743193F93800E5
:10279000042F22D0119B119320AB03EB061606F8F1
:1027A000580C01379EE7204637F03AFE0028EFDA52
:1027B00001230A2212A92046FCF7DEFE40B20028BF
:1027C00003DB129B1B78002BE2D02246711C5F4872
:1027D000FEF77CFA21B0BDE8F08F0023DBE720464E
:1027E000FCF754FF20AB03EB061646F8540CD8E771
:1027F00057492046FCF7A8FEB0F1000A554920468B
:1028000018BF4FF0010AFCF79FFE08B14AF0020A18
:102810003301DFF868C1079320AB03EB0616BCE871
:102820000F0006F850AC12AE0DF1480A0FC6BCE816
:102830000F000FC6BCE80F000FC69CE8030086E837
:1028400003000026B346DAF80010204640F0E4FC0E
:1028500010B19AF804301E430BF1010B0AF1080A7B
:10286000BBF1070FEFD1079B80336B4403F84F6C2C
:1028700097E739492046FBF731FEA0B1374920469A
:10288000FBF72CFE00288CD02046FCF7FFFE032827
:10289000804686D901463248FEF718FA9AE7224662
:1028A0000821304894E7012305937AE70133072B89
:1028B0007FF425AF01312C488AE70B9B1BB9AAF1A5
:1028C00014025542554100235F1CE368002B62D17E
:1028D00094F900B058460DF0D9F9D4F8049018B125
:1028E0000668002E40F08B80B9F1000F237A14BFE8
:1028F0004E464FF46146666023B91C48FEF7E6F980
:1029000003232372627A2AB1394619480792FEF7E7
:10291000DDF9079A02925846237ACDE90063002335
:102920001A46194611F04AFEE06048BB3946114884
:10293000B2E700BF8A3806086D340608E45005087F
:102940008A340608063406081134060815340608C9
:102950003034060875410608333406080C31060881
:10296000393406085134060878340608A3340608BA
:10297000BE340608D934060870610120AC50050841
:1029800058493346584A5948B9F1000F18BF0A460A
:102990003946FEF751F9022F04F110044FF00103FC
:1029A00092D1119E0D9F4DB15148FEF7F9F8336851
:1029B0001B6A1BB13A464F4930469847059B002B8E
:1029C00050D04D49474BBAF1140F18BF19464B4828
:1029D000FEF77CF9BAF1140F09D1059B002B43D007
:1029E0003368DB691BB10022454930469847069B96
:1029F000002B43D100223146384637F029FDE660EE
:102A0000B9F1000F2CD04946304603F031FA3D4A67
:102A1000B36839463C48FEF759F994F80890B9F183
:102A2000000F0CD03279914509D04B4639463748D2
:102A3000FEF74CF93368494630469B699847637AFC
:102A400023B1727939463248FEF740F9F36A002B18
:102A5000A1D039462F48FEF739F90023F3629AE7EF
:102A6000204AD5E71F49B2E7B8F1000FBFDB336852
:102A7000DB69002BBBD042462749B6E7DFF89C90C4
:102A80000025DFF89CA04FF0030B06F0E1FB0520CA
:102A9000FAF7FCFA9AF8F433AB42ABD919F8014FC4
:102AA000C4B1204607F07AFF804698B12046F7F778
:102AB00083FF0446EBB210B180F806B0C371204624
:102AC0000121F7F779FC98F806302046DB0703D59B
:102AD000F7F72EF80135DDE7F7F724F8FAE74FF0BE
:102AE000FF3049E6984A0608EB330608F534060835
:102AF000AB350608715E0108F9330608D4350608BF
:102B00006FEA0008F433060813350608383506085E
:102B10005B35060892350608F5E700081324012006
:102B20009C1E00202DE9F74F05460846FFF706FDDD
:102B30000B46044618B9334A92F8E07127B9284683
:102B400003B0BDE8F04F51E42646DFF8CC90DFF843
:102B5000CCA001AA2C49184640F003FA10B906F09F
:102B600083FB08E056B9012201462846FFF752F9D7
:102B7000421C04461BD103B0BDE8F08FFCF786FD74
:102B80002F28834637D80FB106F062FBBBF1060F42
:102B900014D01E4901235FFA8BF291F8F413E0B2CE
:102BA00005F090FE002759464846FEF78FF801AA27
:102BB00015490020013640F0D4F9CFE7DAF80036A5
:102BC0001B0114D5FF2C0ED0E1B22846FFF74CF9BB
:102BD000E8E701372846FFF747F9F9B298F8F423F8
:102BE0008A42F6D8DEE70027DFF82080F5E70848BC
:102BF000FDF7D6FFD6E72F2206492846FEF7E6FD69
:102C0000D5E700BF706101208A3806089C1E0020AD
:102C10001C31060808360608F735060878500120EA
:102C20002DE9F74307460846FFF788FC0B460446A4
:102C300028B1384603B0BDE8F043FEF7DDBD01AA78
:102C40002E491846264640F08CF9A0460546DFF886
:102C5000AC9065B92A4B3246A1B2D3F8740139F071
:102C600027FB68BB27493846FEF7B0FD28E0B8F1DE
:102C7000000F06D0B8F1010F25D03846FEF7BCFD95
:102C80001EE028463EF0B2F81F4906460246284696
:102C9000FCF736FC50B332461C492846FCF730FCA2
:102CA00030B332461A492846FCF72AFC10B33246A4
:102CB00018492846FCF724FCF0B13846FFF796FB8C
:102CC00003B0BDE8F083B31E294638465A425A4144
:102CD000FFF7A0F8421C0446F2D001AA49460020A2
:102CE00008F1010840F03DF90546B2E74646F4E731
:102CF0000126F2E70226F0E70426EEE78A38060806
:102D00007061012034360608283606082B3606087E
:102D10002E360608313606082DE9F7438046084668
:102D2000FFF70CFC0B46054628B14046FEF764FD54
:102D300003B0BDE8F08301AA2D4918462F4640F0A4
:102D400010F92E460446DFF8A8907CB9022DECD18C
:102D5000A7F57A73B3F57A7F21D94FF4FA634FF46C
:102D60007A7224494046FFF7DDFBE1E74DB1012DC2
:102D700010D001AA49460020013540F0F2F804467F
:102D8000E3E7012221464046FFF744F8431C06468C
:102D9000EFD1CDE72046FCF779FC0746E9E7164D71
:102DA000B8B2D5F890365B689847FCEEC07AFF2E33
:102DB00017EE902A0BD195F8F413B6EEC00A0F4B1C
:102DC000A14210DC11460E48FDF780FFB0E70D4B25
:102DD00031460D48B6EEC00A03EB860383ED790A4F
:102DE000FDF774FFA4E70134A3EC010AE8E700BF94
:102DF0008A380608423706089C1E002054630120CA
:102E00005F3606087061012052360608F8B507469D
:102E10000846FFF793FBC8B11F4B9E690136304649
:102E200034460CF0F1FE0546F0B90134182CA8BF69
:102E3000002420460CF0E8FE0546A8B9B442F4D1BF
:102E400038461649BDE8F840FEF7C0BC0846FCF716
:102E50001DFC04460CF0D8FE054628B92146104852
:102E6000BDE8F840FDF732BF0B4B9C6109F080F8DC
:102E70002A4621460B48FDF729FF172C09D80A4B93
:102E80000C2202FB043393F8B006BDE8F84008F0CA
:102E9000C5BF0020F9E700BF780301206E360608A1
:102EA00082360608983606083C4A050838B50446B6
:102EB000114D0846FFF742FB68B1104B93F9001023
:102EC0004B1C06D10E4B19790E48BDE83840FDF772
:102ED000FDBEC9B2F8E70846FCF7D8FB032804D8C2
:102EE000C0B2FDF7EFFA2946E3E720460322064980
:102EF000BDE83840FEF76ABC984A0608780301200E
:102F000078500120B1360608C136060838B50446A7
:102F1000114D0846FFF712FB68B1104B93F90110F1
:102F20004B1C06D10E4B59790E48BDE83840FDF7D1
:102F3000CDBEC9B2F8E70846FCF7A8FB032804D8C1
:102F4000C0B215F077F82946E3E720460322064988
:102F5000BDE83840FEF73ABC984A060878030120DD
:102F600078500120AD360608BC360608444B2DE9E2
:102F7000F74FDFF8249105461A79009189F800206F
:102F80005A7993F8343089F801200BB905F062F9C9
:102F900000263C4C33F02EF8B0460D23394A0099F8
:102FA000734352F803A05046FCF7CEFA002841D0F4
:102FB000B8F1000F01DDFDF7DBFD51463248FDF7AA
:102FC0003BFE002221462846FEF7F2FBFDF7D0FD2E
:102FD000237903F01803082B45D0102B48D0204646
:102FE000FDF783FE0D22274B02FB0633B3F80900E1
:102FF00032F0C6FF8346D8B12046FBF7C6FB074632
:10300000DBE90221024401442046FBF777FB78B953
:10301000514601901D48FDF70FFEDBF80810019A9C
:1030200028461346CA192146FEF7D8FAFDF7A0FD37
:1030300008F10108013640F262230D349E42ACD102
:103040000020FFF73EF9FF2389F8003089F80130AE
:10305000B8F1000F11D1009A28460D4903B0BDE820
:10306000F04FFEF7B3BB0B492846FFF71FFFB6E74B
:1030700008492846FFF74AFFB1E703B0BDE8F08FE3
:1030800078500120A86205084C330608DC36060893
:10309000EF300608984A0608780301202DE9F74F1B
:1030A000804608460F463DF0A1FE044620B10128A7
:1030B00024D13B782A2B21D1A94E00254FF00D0AAF
:1030C000A84FB14604F00104A748FDF769FD0AFBCB
:1030D00005F33846013559F80310FDF7ADFD3146CB
:1030E00022464046FEF764FB0D36FDF741FD40F2F7
:1030F00062239D42EBD103B0BDE8F08F3D213846FD
:103100003FF063FF002800F0248103469A4613F83D
:10311000012D202AFAD0AAEB070A0130054610F843
:10312000013B202BFAD05FFA8AFA4FF00009DFF852
:1031300030B20D235246384603FB09F35BF8031007
:103140000BEB03040091FCF7DBF9064670BB00991A
:1031500008463DF04BFE824528D1277907F0E00173
:10316000402900F08A8012D871B366797F4A00271F
:1031700002EBC606BA463B4696F870220092009AC9
:10318000BA4202D9BAF1000F63D02BB12DE0602909
:10319000ECD0802900F0A58040467549FEF716FB6B
:1031A000204603B0BDE8F04FFDF79FBD09F10109CE
:1031B00040F262239945BCD13A466E49404603B07D
:1031C000BDE8F04FFEF702BB07F00703042B1CD14C
:1031D0000B460A222846FCF7CFF9D4F80530014601
:1031E0008342D9D32046FBF7F3FB0D23624803FB50
:1031F00009F95BF80910FDF71FFD00222146404642
:1032000003B0BDE8F04FFEF7D3BA052B0DD1012373
:103210000A222846FCF7B0F9D4F80530014683426B
:10322000BADB5B428342B7DCDCE72846FCF72EFAC8
:1032300017F0050F014607D1B4F80520B4F80730A0
:103240009142A9DB9942EEE7B4F90520B4F90730C1
:10325000F6E7D6F86C1251F8270060B129460193C1
:10326000FBF73CF9019B30B94FF0010A3946204683
:10327000FBF7AEFB5346013781E707F00707637999
:10328000013F0093009BB342AFDDAA4615F8013B16
:10329000202BFAD02046FBF785FB0546042F04D8E7
:1032A000DFE807F0030E0E141D005046FCF7EEF9A0
:1032B000A8552C2150463FF088FE0136451CE1E719
:1032C0005046FCF7E3F925F81600F2E700230A223E
:1032D00000215046FCF750F945F82600E9E70123A4
:1032E000F5E728463DF082FDE379064694F805A00F
:1032F000DB07A7790AD52046FBF754FB0378014684
:1033000023B1324628463FF039FFE0B9DEB1B7427B
:1033100019D32046FBF746FB3A4600213FF03EFE1C
:10332000B2453FF662AF3246144928463FF026FFC9
:1033300000283FF45AAF2046FBF734FB32462946BB
:103340003FF0D4FD51E73A460D494046FEF73EFABC
:1033500022E73946404603B0BDE8F04F06E600BF1D
:10336000A86205084C330608EC3606083C4A0508F6
:103370003A370608EF3006082F3706085145060889
:10338000FF3606082DE9F04F914687B00C461A46E5
:10339000002180464D46FEF787FF00270646B9F11B
:1033A000000F63D02946062220463FF04BFF00283D
:1033B0003246404613BF012100214FF0010A4FF071
:1033C000000AFEF771FF0646287811F019FE8346C1
:1033D000F8B1687911F014FE4FF461714FF0190CD7
:1033E000AB78EA789BF805E01CFB03131CFB021288
:1033F00095F801B0297900B14079CDE90410CDE903
:10340000023251463B461A4A4046CDE900EBFDF7F1
:10341000FBFB207811F0F4FD8346F8B1607911F0E0
:10342000EFFD4FF461714FF0190CA378E2789BF82F
:1034300005E01CFB03131CFB021294F801B0217978
:1034400000B14079CDE90410CDE9023251463B4646
:10345000074A4046CDE900EBFDF78EFB0137063405
:103460000635142F9BD107B0BDE8F08FCA46D0E7D0
:10347000483706082DE9F041054686B008460F4654
:10348000FFF75CF8064638B100235B4901201A4675
:1034900006B0BDE8F04175E70846FCF7F7F81328D9
:1034A000044600F3A08006258DF81760534E45436F
:1034B000781CFBF7D0FA074660B1FCF7E7F8C0B21A
:1034C00011F0B8FD30B17319027983F86426012335
:1034D0008DF817303846FBF7BEFA074668B1FCF79F
:1034E000D5F80D2809D8062303FB046383F8650685
:1034F0009DF8173001338DF81730DFF8FC80A91CD8
:103500000DF1170238464144FCF7C4F8FBF7A3FA63
:10351000074668B1FCF7BAF8012809D89DF81730BA
:103520000622013302FB04628DF8173082F8680628
:103530003846FBF790FA80B1FCF7A8F8C0B211F05A
:1035400079FD50B19DF817300622017902FB046223
:10355000013382F869168DF817309DF8172006237D
:10356000042A2FD103FB04630022A3F86826062552
:1035700019F054F805FB046595F8640611F040FD58
:1035800095F8671695F8667619234FF461728046B0
:1035900095F8690613FB012613FB072711F030FD90
:1035A0004379214698F80520039395F86836144826
:1035B0000097CDE9016395F86536FDF787FB06B006
:1035C000BDE8F081052A05D103FB0463002283F8DE
:1035D0006926CCE7062ACAD0002308EB050248F882
:1035E00005309380C3E7132332460649284606B0C8
:1035F000BDE8F041FEF796BFDC560120785001206F
:1036000048370608613706082DE9F04F904689B023
:103610001A460C46002181464546FEF745FE3A4EC5
:1036200008F154030746DFF8E4B0079394F9040067
:103630000CF02CFB00285CD0B8F1000F61D02946BB
:103640000C2220463FF0FEFD00283A46484613BFB4
:10365000012100214FF0010A4FF0000AFEF724FE7D
:10366000074695F9040036F0E5FFEA79034651462E
:1036700006EB82024846D2F8E42404922A7A06EB4A
:103680008202D2F8E4240392AA7906EB8202D2F8ED
:10369000E42402926A7906EB8202D2F8E4240192D1
:1036A0002A6800925A46FDF7AFFA94F9040036F002
:1036B000C1FFE2790346514606EB82024846D2F842
:1036C000E4240492227A06EB8202D2F8E4240392E4
:1036D000A27906EB8202D2F8E4240292627906EB28
:1036E0008202D2F8E4240192226800925A46FDF741
:1036F00043FA0C35079B0C34AB4297D109B0BDE8B7
:10370000F08FC246D1E700BF3C4A0508673706087C
:103710002DE9F04F80468DB00846FEF70FFF0546B5
:1037200038B10023624901201A460DB0BDE8F04FC0
:103730006AE709AF099007915E49C7E9010007A848
:103740003FF0E2FB064636F06BFE431C04460CD10C
:103750002B460A2208A93046FBF70EFF089B1B7870
:103760001BB9C4B2132C15D944B2A31CDBB2012B74
:103770000AD94F4E002396F90420A24200F08C8013
:1037800001330C36072BF6D14046FEF72FFE0DB065
:10379000BDE8F08F333464B2E7E7002302250A2244
:1037A0001946FBF7E9FE09904FF0000BDFF8049192
:1037B000DFF808A1494607A83FF0A6FB20B3FBF7B6
:1037C00065FF3D4A002352F8041B884222D1DBB238
:1037D0000AEB8302D2F8E424904215D1BBF1020F28
:1037E00022D0BBF1030F24D05A1EBBF1010FD2B27D
:1037F00015D00B2A03D88DF829300135EDB20BF125
:10380000010BBBF1040FD5D1052D18D84046FDF7AB
:10381000F3FFBCE70133102BD5D10023D8E7052AED
:10382000EDD88DF82A30E8E7092BE8D88DF82C3050
:10383000E3E79A1E0D2AE2D88DF82B30DDE797E8F2
:10384000070086E80700204636F0F4FE1B4A9DF884
:103850002B10034602EB8101D1F8E41404919DF88A
:103860002C1002EB8101D1F8E41403919DF82A1089
:1038700002EB8101D1F8E41402919DF8291002EBCA
:1038800081020021D2F8E42408460192099A0092AC
:103890000B4AFDF771F97AE7064907A88DF8284029
:1038A0003FF032FB00287FF478AF01257CE700BFB2
:1038B000C85501208A380608204F05083C4A0508EB
:1038C000673706082DE9F04F90468BB000264FF081
:1038D000190A45464FF461790C461A4600210746FD
:1038E000FEF7E2FC0990B8F1000F49D029460A2200
:1038F00020463FF0A7FC0028099A384613BF012153
:1039000000214FF0010B4FF0000BFEF7CDFC2A8990
:103910000990334606925946EA88384605922A7934
:103920000492EA780392AA781AFB029202926A78C9
:103930001AFB029201922A780092124AFDF764F96A
:10394000228933460136594606923846E2880A35BE
:10395000059222790492E2780392A2781AFB0292ED
:10396000029262781AFB0292019214F80A2B0092DA
:10397000044AFDF701F91E2EB5D10BB0BDE8F08F5A
:10398000C346DDE7843706082DE9F04380468BB057
:1039900008460F46FEF7D2FD044638B100235E49C3
:1039A00001201A460BB0BDE8F0438BE70846FBF751
:1039B0006DFE1D28054600F3A5800A268DF82740D8
:1039C0004643781CFBF747F810B101238DF82730E8
:1039D000FBF741F8514C074668B1FBF757FE0D283D
:1039E00009D80A2303FB054383F804029DF8273016
:1039F00001338DF82730DFF82091711C0DF127027B
:103A000038464944FBF746FEFBF725F8074668B100
:103A1000FBF73CFE232809D89DF827300A22013302
:103A200002FB05428DF8273082F807023846FBF783
:103A300012F8074668B1FBF729FE0D2809D89DF852
:103A400027300A22013302FB05428DF8273082F825
:103A500008029DF82730062B0CD0002309EB060244
:103A6000404649F80630536013810BB0BDE8F0437F
:103A7000FDF7C2BE0A260023384606FB0546A6F817
:103A80000A32A6F80C32FAF7E6FF074618B1FBF740
:103A9000FDFDA6F80A023846FAF7DDFF30B1FBF764
:103AA000F5FD0A2303FB0543A3F80C021C4B4FF062
:103AB000FF324FF461705A600A2303FB0542B2F8EB
:103AC0000C320693B2F80A32059392F80832049346
:103AD00092F807320393192392F8061213FB01019F
:103AE000029192F8051213FB01030021019308468D
:103AF00092F804320B4A00932B46FDF73DF80BB0C9
:103B0000BDE8F0831D232246074940460BB0BDE8BF
:103B1000F043FEF707BD00BF746301207061012010
:103B20007803012084370608613706082DE9F04F35
:103B3000804691461E460C4615460027DFF81CA11C
:103B40002DED088B95B094ED008AB5EE408AF1EE2C
:103B500010FA7BD0D4ED019A94ED029AD4ED038A49
:103B6000B9F1000F49D0D5ED00BA95ED01BAB4EE28
:103B70006B8AD5ED02AA95ED03AAF1EE10FA6AD18F
:103B8000F4EE4B9AF1EE10FA65D1B4EE6A9AF1EECA
:103B900010FA60D1F4EE4A8AF1EE10FA0CBF01215E
:103BA000002132468B46404681F00101FEF77CFB46
:103BB000B0EE6B0A064611A8FAF770FEB0EE4B0A9B
:103BC00007900EA8FAF76AFEB0EE6A0A06900BA8F4
:103BD000FAF764FEB0EE4A0A059008A8FAF75EFE0E
:103BE0000599069A079B0390404602915946019217
:103BF000524600933B46FDF707F8B0EE480A11A87D
:103C0000FAF74CFEB0EE690A83460EA8FAF746FEB4
:103C1000B0EE490A06900BA8FAF740FEB0EE680A2B
:103C2000059008A8FAF73AFE069B059A0021039032
:103C300040460292524610341035CDE900B33B465F
:103C40000137FCF799FF082F7FF47DAF15B0BDEC6D
:103C5000088BBDE8F08F0021A3E700BFA737060857
:103C60002DE9F14F06460C46DFF8A8B12046FEF7D5
:103C700065FC074638B100235E4901201A4601B0B1
:103C8000BDE8F04F52E705225B492046FBF738FCC0
:103C9000A0B95A4B0022C3F83023C3F84023C3F81D
:103CA0005023C3F86023C3F87023C3F88023C3F8FC
:103CB0009023C3F8A02301B0BDE8F08F0422594639
:103CC0002046FBF71DFC05462046002D45D1FAF79E
:103CD000C2FE07460028EED03DF088F8DFF838A194
:103CE0005FFA80F85AF8049BB9F1000F07D1224619
:103CF0004349304601B0BDE8F04FFDF767BD42468D
:103D0000494638460135FBF7FBFB84460028E9D1DC
:103D1000384A034600211746013342F8101B082B8E
:103D2000FAD1384B03EBC505D5F880E0BEF1000FA2
:103D300005D149463448354CFCF7C8FF96E795F85D
:103D40007C50AC45F5DA0EEB0C1307EB0C140CF1C0
:103D5000010C0FCB84E80F00F3E7FBF797FC072873
:103D600005463DD82046FAF776FE074658B3FAF7DF
:103D7000D9FB224B012403EB051383EDCC0A384613
:103D8000FAF769FE074638B1FAF7CCFB1B4B013452
:103D900003EB051383EDCD0A3846FAF75CFE0746C0
:103DA00038B1FAF7BFFB154B013403EB051383ED74
:103DB000CE0A3846FAF74FFE38B9304601B0BDE8B2
:103DC000F04FFDF719BD0446D9E7FAF7ABFB0B4BF3
:103DD000032C03EB051383EDCF0A3FF44CAFECE764
:103DE00007233A460A49304601B0BDE8F04FFEF7D6
:103DF00099BB00BFA0640120333406087061012024
:103E0000EF3006083C4A0508C0370608984A0608FD
:103E100061370608BB370608345005082DE9F74F0F
:103E200092460C461A46002181465646FEF73CFA59
:103E300000258046DFF864B0BAF1000F2CD031467F
:103E4000042220463FF0FEF900284246484613BFB0
:103E50000121002101270027FEF726FA73888046FA
:103E60005A46019339463AF82530484600932B4686
:103E7000FCF7CAFE63885A46394648460193043621
:103E800034F8043B00932B460135FCF775FE042DF6
:103E9000D2D103B0BDE8F08F5746EBE7CA3706082A
:103EA0002DE9F34105460846FEF748FB0C46074658
:103EB00038B10023334901201A4602B0BDE8F04171
:103EC000ACE731492046FAF709FB70B904222D4BC3
:103ED0004FF47A704FF4FA61013A1880598003F177
:103EE0000403F9D102B0BDE8F0812046FBF7CEFB18
:103EF0000328064641D82046FAF7ADFD074698B19B
:103F0000FBF7C4FB4FF0010804463846FAF7A3FD5F
:103F100020B1FBF7BBFBB8F1000F09D1284602B076
:103F2000BDE8F041FDF768BC40F2EE248046ECE7C6
:103F3000A4F2EE2240F2DC539A4203D8A0F2EE2221
:103F40009A420AD940F6CA0340F2EE220F492846A7
:103F500002B0BDE8F041FEF7E5BA0D4B00210D4A75
:103F600003EB8603A3F8B043A3F8B2033346CDE9CD
:103F700000400846FCF700FEB4E703233A46064932
:103F8000E5E700BF2065012033340608DB3706086B
:103F900070610120CA370608E33306082DE9F04FA7
:103FA0008FB08946174600211A4606460024FEF7C0
:103FB0007BF90DF1240B0546DFF86CA059F824803D
:103FC000594602A8CDF8088036F0E4FA4FB357F806
:103FD00024302A4630469845039313BF012100211F
:103FE0004FF001084FF00008FEF75EF904A90546FE
:103FF00003A836F0CFFA04A9234652460091304672
:104000004146FCF701FE2346013452464146304604
:10401000CDF800B0FCF7B0FD202CCFD10FB0BDE83B
:10402000F08FB846EFE700BFE9370608F0B507465E
:1040300089B008460E46FEF781FA054638B10023DE
:10404000194901201A4609B0BDE8F040A6E7084624
:10405000FBF71CFB1F2804461DD83046FAF7FBFC73
:10406000014620462BF06CFC78B103AE0E48314679
:1040700000EB840036F08EFA23460C4A2946284687
:104080000096FCF779FD09B0F0BD384609B0BDE8EF
:10409000F040FEF7ABB91F232A460549384609B060
:1040A000BDE8F040FEF73EBA30650120E93706086A
:1040B000613706082DE9F04F924685B00C461A4646
:1040C000002181465546FEF7EFF800268046DFF8CE
:1040D0006CB0BAF1000F2FD02946042220463FF0E1
:1040E000B1F800284246484613BF012100210127AC
:1040F0000027FEF7D9F8EB7880465A4602933946F6
:10410000AB78484601932B8800933346FCF77CFD3F
:10411000E3785A463946484602930435A37801931A
:1041200034F8043B009333460136FCF725FD102E8E
:10413000CFD105B0BDE8F08F5746E9E7F337060861
:10414000F0B5074685B008460E46FEF7F7F9054676
:1041500038B100231C4901201A4605B0BDE8F040E3
:10416000A8E70846FBF792FA0F28044623DC3046FE
:10417000FAF771FC014620462BF0BCFCA8B104F113
:104180002002124B2946284603EB820393F8C323EF
:10419000029293F8C2230192B3F8C0330C4A009301
:1041A0002346FCF7E9FC05B0F0BD384605B0BDE894
:1041B000F040FEF71BB90F232A460649384605B0E2
:1041C000BDE8F040FEF7AEB9B06501207061012096
:1041D000F3370608613706082DE9F04F85B014461D
:1041E0001A46054602910021FEF75EF84FF00008DE
:1041F000064606234FF0000903FB08F7C037029B71
:1042000013F807B0002C7AD0E35D324628469B4570
:10421000039313BF012100214FF0010A4FF0000A60
:10422000FEF742F8039B0646374A51462846CDE939
:1042300000934346FCF7E8FC4346334A5146284680
:104240000137CDE9009B09F10109FCF795FCB9F1B3
:10425000060FD4D108F10108B8F1060FC9D1E4273F
:10426000029BA7F1E40913F807A0002C49D014F829
:1042700007B032462846DA450DBF4FF001084FF02F
:10428000000801210021FEF70FF8062306461E4A0A
:1042900041462846CDE9009BFCF7B6FC01370623D2
:1042A000194A41462846CDE9009AFCF765FCEF2FF4
:1042B000D6D1029B93F8EF70ACB194F8EF80324600
:1042C0002846474513BF0121002101240024FDF7A2
:1042D000EBFF00230C4A2146009328460723CDF824
:1042E0000480FCF791FC0023074A214628460093EE
:1042F00007230197FCF740FC05B0BDE8F08FA2460C
:104300009AE7A046CAE700BF05380608F0B505469B
:1043100085B008460B46FEF711F9044638B1002374
:104320001B4901201A4605B0BDE8F04054E701AE34
:10433000184F6A46174918463EF013FE88B1032C01
:1043400004D12846FDF758FA05B0F0BDFBF79EF9F9
:104350006A4646F8040B3946002001343EF001FE5F
:10436000ECE7032CEDD1039FDDE901463A463146E7
:10437000E0B22BF0F9FB18B92846FEF737F8E3E76F
:104380003B46324621460448FCF7A0FCDCE700BF70
:10439000306501208A380608053806082DE9F04FF7
:1043A0000E46154689B01A4600210446B046FDF770
:1043B0007BFF2F4681464FF0000B002D7AD0394607
:1043C0000C2240463EF03EFF00284A46204613BFDE
:1043D000012100214FF0010A4FF0000AFDF764FFB0
:1043E00097F90B2081465B460492514697F90A20C3
:1043F00020460392B7F908200292B7F906200192ED
:10440000B7F904200092364AFCF7FEFB98F90B201E
:104410005B460BF1010B51460492204698F90A20A5
:104420000C3708F10C08039238F9042C029238F981
:10443000062C019238F9082C0092294AFCF79CFBC3
:10444000BBF1080FB9D14FF0000BDFF898800C23B7
:1044500003FB0BF985B3002755F80900012356F833
:10446000092003FA07FA42403AEA020214BF194649
:10447000002110EA0A0F07D05B464246204600970B
:104480000791FCF7C1FB079956F809201AEA020FB9
:1044900005D05B46424620460097FCF76DFB01378E
:1044A0000E2FD9D10BF1010BBBF1080FCFD109B001
:1044B000BDE8F08FAA46A9E72F46012356F8091058
:1044C00003FA07F20A4206D05B4642460121204623
:1044D0000097FCF751FB01370E2FEED1E2E700BF4A
:1044E0001938060831380608F0B506468BB008467C
:1044F0000D46FEF723F8044620B300233D49012072
:104500001A460BB0BDE8F04048E72D2903D0A1F1D1
:104510003003092B49D8052C05DD30460BB0BDE82A
:10452000F040FDF769B92846FBF7B0F80AAB621C0A
:1045300003EB440424F80C0C15F8013F303B092B25
:10454000FAD9144629780029DFD1062CE5D1BDF827
:104550001C20BDF91C30072ADFD8BDF91E50A5F577
:10456000FA7292B2B2F5FA6F18D8BDF92070A7F5B9
:10457000FA7292B2B2F5FA6F10D8BDF922C0654551
:104580000CDC67450ADBBDF924E00EF1640292B24F
:10459000C82A03D8BDF92640112C11DD1649304632
:1045A0000BB0BDE8F040FDF711B9202902D101356B
:1045B0002246C6E730460BB0BDE8F040FDF716BF17
:1045C0000C200E4A64B200FB03220846A2F8B45441
:1045D000A2F8B674A2F8B8C482F8BAE482F8BB4470
:1045E000074A0095CDE903E4CDE9017CFCF7C4FA64
:1045F0000BB0F0BD2066012046380608706101202E
:10460000193806082DE9F04F89468DB0164600216D
:104610001A4607460024FDF747FEDFF8DCA00546F2
:10462000C4EBC40309EB030259F80300918840F37B
:10463000074892790890ADF824108DF82620B8F13B
:10464000000F53D0002E54D0F218F058918893796F
:1046500007220A9008A8ADF82C100AA98DF82E3070
:104660003EF0F0FD00282A46384613BF0121002104
:104670004FF0010B4FF0000BFDF716FE9DF82E30AA
:1046800005465246069359469DF92D303846059306
:104690009DF92C3004939DF82B3003939DF92A301B
:1046A00002939DF8293001939DF82830009323460A
:1046B000FCF7AAFA9DF8263052465946384606932A
:1046C0009DF9253005939DF9243004939DF82330FE
:1046D000CDE902839DF8213001939DF820300093AD
:1046E00023460134FCF748FA102C99D10DB0BDE8EF
:1046F000F08FB346DEE700BF5C3806082DE9F04FC7
:1047000006468BB00D46DFF8A08228463CF06EFBD3
:10471000034630B90246964901200BB0BDE8F04F80
:1047200070E7052293492846FAF7EAFE0446C8B91D
:10473000914D0146702205F5A2603EF02FFCC5F8B0
:10474000B044C5F8BC44C5F8C844C5F8D444C5F85D
:10475000E044C5F8EC44C5F8F844C5F804450BB08E
:10476000BDE8F08F042241462846FAF7C9FE044608
:1047700030BB2846FAF76FF981460028EFD03CF0AD
:1047800035FBDFF828B282465BF8047B3FB92A4646
:104790007A4930460BB0BDE8F04FFDF717B85246E6
:1047A00039464846FAF7ACFE40B92046744D1CF035
:1047B00069FC39467348FCF789FAA6E70134E3E758
:1047C000072271492846FAF79BFE074600287AD14E
:1047D000202128463EF0F9FB044670BB6B4D6C4827
:1047E000FCF72AFA214601342846FCF725FA0E2C5C
:1047F000F8D10025DFF8B891664FFCF7B9F9DFF87A
:10480000B4810C260024DFF8B0A129466E43484647
:10481000FCF712FA0123F2595F48A3400134134216
:104820000CBF41465146FCF707FA0E2CF2D1013578
:10483000FCF79EF9082DE4D191E702AC574D01AA8F
:1048400056493EF08EFB002848D0022F11D1029A23
:10485000072A07D8039C0D2C04D80378722B13D099
:104860006E2B25D0082300224D493046FDF75AFE15
:1048700075E7FAF70BFF01AA44F8040B294600205C
:1048800001373EF06EFBDEE70C233B4903FB0211D0
:104890000123D1F8B014A3400B4337490C2000FB8F
:1048A00002123949C2F8B0343046FFF727FF56E705
:1048B000314B0C20012100FB0233A140D3F8B0346E
:1048C00023EA0103E9E72846002402AD334F01AA99
:1048D00032493EF046FB80B1082C03D13046FCF74C
:1048E0008BFF3CE7FAF7D2FE01AA45F8040B3946E4
:1048F000002001343EF035FBEDE7082CEED1029BA1
:104900000F2B30D8DDF80CE0BEF1070F2BD8DDF807
:1049100010C0BCF10D0F26D8059F07F16402C82A0C
:1049200021D8069DFF2D1ED8079864281BD808990A
:10493000642918D8884216DA099C032C13D8C3EBD3
:10494000C3020D4B134483F8151583F810E50C4989
:1049500083F811C583F8127583F8135583F814058D
:1049600083F81645A0E70F493046FCF72FFFF6E61F
:10497000806601203334060870610120EF3006089C
:10498000984A0608C03706087938060881380608AC
:10499000433F060820660120863806088A38060844
:1049A0008C38060846380608BB3706083450050818
:1049B000F92906089B3D0608443806082DE9F04F02
:1049C0009246002689B04FF019095546B3464FF478
:1049D00061780C461A4600210746FDF765FC0790F2
:1049E000BAF1000F27D02946062220463EF02AFCC5
:1049F0000028079A384613BF012100214FF0010B10
:104A00004FF0000BFDF750FC6A790790334619FB15
:104A100002825946384605922A7919FB028204928D
:104A2000EA780392AA7802926A7801922A78009230
:104A3000104AFCF7E9F8627933460136594619FB0A
:104A40000282384606350592227919FB02820492C9
:104A5000E2780392A27802926278019214F8062B0F
:104A60000092044AFCF788F80A2EB9D109B0BDE8D3
:104A7000F08F00BF923806082DE9F04F074689B045
:104A800008468B46FDF75AFD044638B100235449C9
:104A900001201A4609B0BDE8F04F8FE7514B084698
:104AA00093F888A793F8899793F87288FAF7EEFD40
:104AB0000928054600F38B8006268DF81F404A4CD6
:104AC00046430BF10100F9F7C6FF834648B1FAF7F8
:104AD000DDFD0D2805D8A31983F8800501238DF885
:104AE0001F305846F9F7B7FF834668B1FAF7CEFD95
:104AF000504509D8062303FB054383F881059DF83B
:104B00001F3001338DF81F305846F9F7A4FF824655
:104B100068B1FAF7BBFD484509D8062303FB0543F6
:104B200083F882059DF81F3001338DF81F30504601
:104B3000F9F791FF814668B1FAF7A8FD804509D3DE
:104B4000062303FB054383F883059DF81F300133DB
:104B50008DF81F30DFF88880311D0DF11F024846A7
:104B60004144FAF797FD9DF81F30062B0BD0002328
:104B700008EB0602384648F80630938009B0BDE8D5
:104B8000F04FFCF739BE03FB05424FF46170192367
:104B900092F8851513FB0101059192F8841513FB1A
:104BA000010300210493084692F88335039392F899
:104BB0008235029392F88135019392F880350B4A41
:104BC00000932B46FBF7D8FF09B0BDE8F08F09230F
:104BD00022460749384609B0BDE8F04FFDF7A2BCB0
:104BE000F06601207850012070610120923806089B
:104BF000613706082DE9F04F14468BB00F461A4670
:104C000000210646FDF750FB0546002C00F0D7803A
:104C100022783B789A42024630460DBF4FF0010899
:104C20004FF0000801210021FDF73EFB23780546E7
:104C30009B4A41463046FBF7E7FF3B784146984A9E
:104C40003046FBF799FF002C00F0BB8062783046BD
:104C50007B789A422A460DBF4FF001084FF00008BA
:104C600001210021FDF720FB637805468D4A41466E
:104C70003046FBF7C9FF7B7841468A4A3046FBF74E
:104C80007BFF07F1C90307F1020A04F1CA0B059380
:104C9000A31C4FF000090693822307933B784B45F2
:104CA00000F39180002C00F0F58097F8EA30304650
:104CB00094F8EA209A422A460DBF4FF001084FF0BF
:104CC000000801210021FDF7EFFA94F8EA300546CB
:104CD000754A41463046FBF797FF97F8EA30414660
:104CE000714A3046FBF748FF002C00F0D58004F1F4
:104CF000EA0307F1EA0204F1FA014FF0010833F880
:104D000002CF32F8020F844518BF4FF000089942D5
:104D1000F5D188F001012A463046C9B2FDF7C4FA40
:104D20000821054604F1EC00FAF74CFB5F4A034604
:104D300041463046FBF768FF97F8EA1007F1EC00B0
:104D4000FAF740FB594A034641463046FBF714FF49
:104D5000002C00F0A3804FF0FC094FF0010807EB96
:104D6000090104EB0900F9F7B9FB09F1040900286E
:104D700018BF4FF00008B9F58E7FF0D188F001011F
:104D80002A463046C9B2FDF78FFA082104F1FC002B
:104D9000F9F773FE464A034641463046FBF734FFB7
:104DA00097F8EA1007F1FC00F9F767FE404A03465E
:104DB000414630460BB0BDE8F04FFBF7DDBEA046E4
:104DC0003BE7A04657E7079BFB180993002C5FD0F1
:104DD000079B0998E31819460893F9F77FFB059B91
:104DE0005A789BF800309A424FD1B0FA80F84FEAD7
:104DF0005818069AAAF102030AF10E01023A33F892
:104E000002CF32F8020F844518BF4FF000088B42E2
:104E1000F5D188F001012A463046C9B2FDF744FABF
:104E20006278069905469BF81800FAF79DFA0290F9
:104E30009BF8003041461F4A30460193089B00937F
:104E400009F10103FBF7E0FE059B51467A7809F171
:104E50000109587E0AF1100AFAF786FA059A0290BB
:104E6000414612F8013F30460BF1010B0193099BBB
:104E7000059200934B460F4AFBF77EFE069B1033CC
:104E80000693079B0933079308E74FF00008B0E744
:104E9000A046D9E7A04620E7A0464DE7A0467FE719
:104EA000AB380608BD380608EB3806080339060893
:104EB0001A390608D23806082DE9F04F8FB004469B
:104EC0000846B24902AA3EF04CF8054640B90346EE
:104ED0000246AF494120FFF78DFE0FB0BDE8F08FCD
:104EE000AC49F9F7FBFA064628BB02AAA7493EF0EF
:104EF00038F8FAF7CBFB0828054606D908233246CE
:104F0000A5492046FDF70EFBE7E7A44C94F8883747
:104F100083420CDC84F88857DFE731460136384697
:104F200024F0C0F994F88837B342F6DCF2E706467D
:104F300004F5F167F6E79A492846F9F7CFFA0646ED
:104F4000E0B902AA91493EF00CF8FAF79FFB082855
:104F5000054603D9082332469249D2E78F4C94F88C
:104F60008937834202DC84F88957B6E73046013638
:104F7000294635F02DFA082EF8D1F4E78A4928465B
:104F8000F9F7ACFA064600BB02AA80493DF0E9FFFA
:104F90000028A2D0FAF77AFB0828054603D908238F
:104FA00032468249ADE77D4C94F87238834209DD80
:104FB000014604F5F16024F0BBF9294604F5F160DF
:104FC00024F0C4F984F8725887E779492846F9F73C
:104FD00085FA064618BB06AD704BDFF8B091014666
:104FE000A8461022284693F872783DF0D7FFBE42BB
:104FF00002AA80F20A81494600203DF0B2FF10B9B2
:105000003A466C490AE1FAF741FB013628F8020BEF
:10501000EDE7694C95E80F0084E80F005DE767490C
:105020002846F9F75BFA0646C0BB5C4B06ADDFF8D5
:105030005C9193F87278BE4202AA80F2F3804946EE
:1050400000203DF08EFF014610B93A465C49E5E08C
:10505000AA464FF00008032228463EF0A1F8284651
:105060003BF0C4FE404502D801360435E3E79AF828
:10507000000008F10108FAF73DFA0AF8010BEEE723
:10508000B60004464F4DB4423FF427AF06AB281993
:1050900003221919043424F0EFF8F4E74A492846AA
:1050A000F9F71CFA0746002840F0AC80DFF8EC80E6
:1050B00002AA364998F888673DF053FF00283FF46C
:1050C0000CAFFAF7E3FA451E01D4AE4203DC3346D7
:1050D00001223E4915E72D4902AA00203DF041FF7B
:1050E000014600283FF4F9AE00260DF10C09082214
:1050F00003A88DF814603EF053F803A83BF076FE49
:10510000B0421BD802AA214900203DF02AFF002806
:105110003FF4E3AE0026037898F889A7B1460193DF
:10512000564502AA19494FF0000080F285803DF0F3
:1051300018FF834650B9524625496FE099F80000A0
:105140000136FAF7D7F909F8010BD6E7A6B99BF8AB
:105150000030303B092B0FD91E49F9F7BFF938B1A0
:105160001D495846F9F7BAF970B15A461B4955E03E
:105170004FF001094FF0FF365846FAF787FA00283A
:1051800030DA5A46164949E0B146F3E78A3806084C
:1051900000580120313906083739060878500120B7
:1051A000423906084B390608593906086539060898
:1051B00077390608663A0608EC580120A139060836
:1051C000863A0608FC580120CB390608D039060873
:1051D000A63A060843290608DC390608E33906081A
:1051E000183A06080EAB03EB4603013623F8200CF1
:1051F00096E752461F4911E033F8022B013724F895
:10520000022F30E02A461C4908E01C4900203DF0EE
:10521000A8FE00283FF4FDAE3A4619492046FCF7A7
:10522000D5FA5AE6154900203DF09BFE00283FF4D0
:1052300027AF3A461349F1E73DF093FE0028D8D155
:1052400005EBC500104C082203A98230204404EB72
:10525000051424F011F80198FAF74CF908EB05034E
:1052600083F8520806ABBE42C6DC454485F86A980E
:1052700033E600BF2D3A0608503A06088A38060879
:1052800083390608AD390608005801202DE9F04F92
:105290000F46904689B0002187EA08080646139A0F
:1052A00000250393FDF700F8DFF884906FEA080308
:1052B0000446069328460AF095FC129B184230D00B
:1052C000069BDFF870B0034014BF4FF0010A4FF0A7
:1052D000000A049310EA070328460CBF4A465A46C0
:1052E000059307920AF090FC039B8046079A51466B
:1052F00000903046FBF788FC049B22463046B3FA08
:1053000083F14909FCF7D0FF059A0446039B002A64
:105310000CBF5A464A4651463046CDF80080FBF74E
:105320002BFC0135172DC5D109B0BDE8F08F00BFAA
:10533000CB3A0608B537060870B504460E4608464F
:105340003BF054FD3146054602462046FAF7D8F8B0
:1053500068B9635D1846FAF7B7F800B933B9013593
:105360002C44204601340378202BFAD070BD002055
:10537000FCE708B504460948FBF7F2FBFBF7D4FB52
:10538000074BD3F874010FF0F9F803F0CBFE012CB2
:1053900001D136F01FFBF6F7C9FB00BFD23A060871
:1053A0007061012010B5044608460B46FDF7C6F8AB
:1053B00028B9032208491846FAF7A2F828B907487D
:1053C000FBF7F4FB0120FFF7D4FF20460449BDE8BA
:1053D0001040FCF7FBB900BFDE3A0608E23A0608C7
:1053E0001A3306082DE9F74F4FF0000B064601AAC5
:1053F00008462E495D463DF0B4FD01270446DFF81E
:10540000BC80DFF8BC90DFF8A4A01CBBBBF1000F90
:1054100028D1274C002D44D029462648FBF756FCBE
:1054200094F834300BB902F015FF30F0E3FD00239F
:1054300084F85D30FBF74EFB15B12846FCF741FFC1
:105440009FB13046FCF7F4FE78B1FBF7C1F90020BC
:10545000FFF78FFFBBF1000F0AD02046FAF716F9CD
:1054600085B2C5B93046FCF7C1FF03B0BDE8F08F87
:1054700041462046FAF768F880B949462046FAF7CF
:1054800063F80028EED05F4601AA514600203DF0A7
:1054900068FD0446B9E74FF0000BF5E74FF0010B4C
:1054A000F2E70548FBF782FBBFE700BF8A38060832
:1054B000785001200D3B0608303B0608043B0608E7
:1054C000D640060810B50C46FCF7B2FE78B1084B82
:1054D00001229A74FBF77CF90648FBF767FB064943
:1054E0002046F8F7FBFF10B10020FFF742FF10BD88
:1054F00078500120463B0608632906080329F0B5C9
:10550000054685B00C46164614D80B4F3970FBF78C
:105510002FFB0A492846FDF7C9FC2246084901A885
:10552000F9F70CFF01AB324608212846FCF7ECFEE8
:10553000FF233B7005B0F0BD78030120984A0608B0
:10554000B13606080329F0B5054685B00C46164667
:1055500014D80B4F7970FBF70BFB0A492846FDF76F
:10556000D5FC224608496846F9F7E8FE6B46324604
:1055700010212846FCF7C8FEFF237B7005B0F0BD64
:1055800078030120984A0608AD36060810B5114B7D
:1055900086B0114904460493104B11480393114BF4
:1055A000114A0293114B0193114B0093114BFBF7DE
:1055B00043FBFBF7DDFA10491048FBF787FB3CB1D2
:1055C0000F4A1049104806B0BDE81040FBF77EBBFB
:1055D00006B010BD8D3B0608573B0608923B0608F7
:1055E000623B06089D3B06084D3B0608A63B0608A5
:1055F000B23B060883500120BC3B0608C43B0608AA
:10560000C32F060814300608D53B06080120BDE765
:105610002DE9F04F3B4C89B00A4600210546FCF7C6
:1056200043FE059094F9000003F058FE814660881F
:1056300030F0A6FC344BD0F808B093F8347017B1B2
:105640005F46D0F80CB0A3790026012B38BF0123A8
:1056500006932279637906FB02331BF80380002F3F
:105660003AD0FB5C4345059A2846079313BF0121B6
:1056700000214FF0010A4FF0000AFCF715FE079BCE
:105680000136059053B303F00F021B09514628461B
:10569000403302921D4ACDE900634B46FBF7B4FA52
:1056A000B8F1000F24D008F00F034FEA1818174A7A
:1056B0005146029308F140032846CDE900634B466A
:1056C000FBF75AFA069BB342C3DC0834104BA342E3
:1056D000A8D109B0BDE8F08F3B46C3E7002FDFD06B
:1056E0004B460C4A514628460096FBF78DFAD7E701
:1056F0006B06E7D44B46074A514628460096FBF70F
:105700003BFADFE70C52050878500120023C0608FE
:105710000C530508183C060838B50B4D0C4605EB34
:10572000C00595F9D00703F0D9FD01460748FBF7FE
:1057300083FA95F8D63733B1611C0548C9B2BDE884
:105740003840FBF779BA38BD3C4A0508423F0608A5
:10575000F829060873B50E4610490546F8F7BEFE4F
:1057600018B93070012002B070BD2C78602C8CBF4D
:10577000613C413C082C0FD8013501230A2201A9C4
:105780002846F9F7F9FE019BAB4205D00F2803D854
:10579000013440EA0410E4E70020E4E7DD280608CD
:1057A0002DE9F04F724C8DB0DFF8D0910A4604F12C
:1057B000800A00218346FCF777FD03900025A37A39
:1057C00099F83460AB4200F3928010345445F5D11F
:1057D00040F216200DF1180A30F0D2FB0027002EFF
:1057E0004FF015024FF00001D0E90245504604BFCA
:1057F000254634463DF0D2FB2E78002E3ED0697807
:105800003046059104F0F8FB95F90290049009F1F7
:10581000010253425341002C00F0A680002205995A
:10582000A05CB04240F09C80224492F90280C145C5
:1058300040F0948052788A4208BF0123012203F08D
:1058400001030AF8072083F00101039A58460593E3
:10585000FCF72AFD059B039044B1464A3046049963
:10586000CDE900B24246F9F77BF9059B424A304642
:105870000499CDE900B24A46F9F772F901370335C8
:10588000152FB9D184B3564604F13F07DFF8E48001
:10589000DFF8E49016F801ABBAF1000F21D12078BF
:1058A000F8B194F9023001331BD0617804F0A4FB05
:1058B0000546039A01215846FCF7F6FC94F90220AC
:1058C0005346294603902078CDE900B8F9F748F906
:1058D000207853464FF0FF322946CDE900B9F9F759
:1058E0003FF90334BC42D5D10DB0BDE8F08FE0885C
:1058F00030F046FB002E627AD0E90231207A04BFF4
:105900001946334605FB00228F5623B39E56B742F5
:10591000039A5846049313BF012100214FF0010858
:105920004FF00008FCF7C0FC049B039043B1114BFF
:10593000324629462046CDE900B34346F9F7CCF874
:105940000D4B29463A4620460135CDE900B3434682
:10595000F9F7C2F833E74FF0FF36D8E700236DE7D9
:1059600003323F2A7FF45CAF4FF0FF386BE700BF94
:1059700094030120090C0108790B010878500120DB
:105980002DE9F04F80468BB008460D463BF02EFACD
:105990000246A8B3A3492846F9F7B2FD044678BBEE
:1059A000FBF7E6F8A04DA148A14EFBF7F9F8A14F8F
:1059B0001420DFF8C08234F01FFDE110304604F0FF
:1059C00007020131FBF738F995F81D9095F91C0095
:1059D000B9F1000F0DD003F081FC4A460146404664
:1059E000FBF774F901342435102CE6D10BB0BDE877
:1059F000F08F03F073FC01463846FBF767F9F1E7D7
:105A0000284605AA8C493DF0ACFA054620B9014666
:105A10004120FFF7C5FEE9E78849F8F75FFD20B9A7
:105A200087494046FBF7D2FEE0E7864E0827002470
:105A300031682846F8F752FD002808BF3446013F78
:105A400006F11006F4D154B97F492846F8F746FD0F
:105A500028B12A467D494046FBF7B8FEC6E700203C
:105A600005AA75498DF813003DF07BFA0646002C17
:105A70004ED000284AD0F9F709FE031E43DB2279F5
:105A8000062A3BD10121E26801FA03F010423AD024
:105A9000DBB247F6FE7040FA03F2D20733D59940E5
:105AA000013908403DF02AFC0546E088002730F027
:105AB00067FA6749039791F83410D0E90223002967
:105AC00018BF1A46217A637A05FB013302EB030AF9
:105AD00012F9039005AA584900203DF042FA834686
:105AE00000283ED101235B4994B39AF90020204657
:105AF000CDE900312946F8F7EFFF77E75D1E13B1D6
:105B0000A37A9D42D1DB32465349A4E7534EFAE7CC
:105B100068B10DF11301FFF71DFE28B19DF8135078
:105B20002846F4F749FF20B932464D4993E74B4EDA
:105B3000FAE72846A246F4F727F88146284604F0FB
:105B400047FA03902846254604F028FF0746C1E798
:105B5000CDE900314A4639469DF81300F9F700F8BF
:105B600044E73649F8F7BAFC064658BBACB1EDB28B
:105B70003C4F72B229462079F3F7E0FF00283FF44A
:105B800035AF028831460378384601360093C2F3B8
:105B90000323120BFBF79AF8EBE7324C72B27979D8
:105BA0003868F4F70DF800283FF420AF028831463A
:105BB0000378204601360093C2F30323120BFBF750
:105BC00085F8EBE728495846F8F788FC002853D0B9
:105BD0005846F9F75BFD064642B29CB1E9B220791E
:105BE000F3F7ACFF002849D1266829462046F8F78C
:105BF00021FE324603461D49CDF800B04046FBF772
:105C0000E5FDF3E679793868F3F7DAFFB0BB9DF884
:105C1000133017491A09CDF800B003F00F034032D2
:105C2000ECE700BF2C3C06087C000120313C060854
:105C3000473C06087A2C06088A380608C92D06084B
:105C4000583C060894030120EE4306086C3C060805
:105C500078500120790B01087B3C0608984A060819
:105C60008B3C06089D3C06080C310608BE3C060825
:105C7000E13C0608204206084FF0FF3606AF3046EA
:105C80003946F9F7D1FB08A94846F9F7CDFB4E454F
:105C90001CD076B274B18AF8006029462668204686
:105CA000F8F7C8FD08AB0246314613480097FBF7EA
:105CB0000DF89BE69DF81320039B11090F489E7079
:105CC00002F00F0208AB40310097F0E75CB12668A4
:105CD00029462046F8F7AEFD08AB02463146084893
:105CE000FAF7F4FF82E69DF8132008AB0548110986
:105CF00002F00F024031F3E7093D06082C3D06088B
:105D0000543D06086F3D0608224BB0F5FA6F1A683D
:105D10000346A8BF4FF4FA63B3F57A7FB8BF4FF4D8
:105D20007A73D20416D540F2DC52904215D040F27C
:105D3000DB5207EE903A9042F8EE677A1FD8DFED1B
:105D4000166A9FED167A77EEE67A9FED150AA7EEB2
:105D5000870A7047B0F57A7F02D89FED120A704724
:105D600007EE903ADFED106A9FED107AF8EE677A51
:105D70009FED0F0A77EEE67AA7EE870A7047DFED10
:105D80000D6A9FED0D7A77EEE67A9FED0C0AA7EE8D
:105D9000870A70477856012000007A44D62000C058
:105DA00000E082440000000000407A446610004099
:105DB0000000404200A0BB44D620004000008344C5
:105DC00009494FF4EB7200234FF01F0CC0F802108A
:105DD000C2800649064A0370A0F808C0C0F80A103D
:105DE0004382C0F80E2070474A01B400C2010E0180
:105DF00096004400704700BF00207047704700BF06
:105E00000020704701207047704700BF704700BFF7
:105E1000704700BF704700BF9FED010A704700BF89
:105E20000000000000207047064B1B78834206D913
:105E300000EB4000044B03EBC0035869704700209F
:105E4000704700BFA4070020E006002000EB4000E0
:105E5000024B03EBC003587C704700BFE0060020F4
:105E6000024B1878003818BF01207047A4070020A3
:105E700003681B6903B11847704700BF70B5094C30
:105E8000236873B10546002606E099681A681E73F8
:105E900021609047236823B15A681846AA1A002A3D
:105EA000F3DA70BD6C7901200B4B1A79D20700D55B
:105EB00070479A68002AFBD04FF47A7101FB02F216
:105EC0009042F5D3054A12781AB9054A91681269C9
:105ED0000A6000229A6070476C790120D467012023
:105EE000E867012008B5294B1B68DB041ED5B5EE19
:105EF000400AF1EE10FA26D0DFED257AB4EEE70A7B
:105F0000F1EE10FA1FD49FED237AB4EEC70AF1EE3A
:105F100010FA2AD870EE677A9FED1F7A9FED1F0A5C
:105F2000A7EE870A3CF00AFB80B208BDDFED187AC5
:105F3000B4EEE70AF1EE10FA0BDA9FED190A3CF025
:105F4000FDFA80B208BD9FED170A3CF0F7FA80B267
:105F500008BD70EE677A9FED147A9FED140AA7EEE4
:105F6000870A3CF0EBFA80B208BDDFED117ADFED75
:105F7000116A70EE677A9FED107AA7EEA67AB0EEFE
:105F8000470A3CF0DBFA80B208BD00BF785601201A
:105F90000000404200E0824466BEFFBE0060BB4499
:105FA00000007A440080BB4438DFFF3E00407A4462
:105FB0000000834466BEFF3E00A0BB446B4B1B78D1
:105FC0002DE9F04F87B0002B00F0CA80684D4FF0EC
:105FD00000086848A968FAF779FE69686648FAF720
:105FE00075FE664B6648D3E90031C91A654B1A68DD
:105FF000B1FBF2F2FAF76AFEFAF7BAFD6248FAF775
:10600000CFFD6248FAF7CCFD614B5FFA88F41B784C
:10601000A34221D85F4D00245F4EFAF7A9FD013459
:1060200055F8041F3046FAF707FE162CF7D15B4DE2
:106030000124594EFAF79CFD2B466968013430461D
:106040001B680435C91AFAF7F7FD162CF4D107B00E
:10605000BDE8F04FFAF78CBD514B14264FF03C0BC6
:10606000671C03EB840306FB045693ED000A3CF027
:1060700065FA96F81EA081B2B6F80E901AF0010FDC
:1060800080B20CBF2D2252221AF0020F0490454814
:106090000CBF2D2354231AF0040FB1FBFBF10CBFEE
:1060A0004FF02D0C4FF0560C1AF0080F05914FF0E1
:1060B00064010CBF4FF02D0E4FF0430E1AF0800F0D
:1060C00001FB09F10CBF4FF02D0A4FF0530ACDE947
:1060D00000CECDE902A13946FAF7AEFDB37FDB076A
:1060E0003AD55C23304A6343D118D05891ED010A68
:1060F00070B1B8EE400ADFED2D7A20EE270A07EEE8
:10610000900AF8EE677A80EE270A3CF017FA00B2A0
:10611000642290FBF2F102FB11022548FAF78CFD94
:106120001421244808F1010801FB075701FB04541E
:10613000F988628A0491218B02F00303920803918B
:10614000E18A0291A18B0191A18A009119214B430F
:10615000218AFAF7BBFD57E71748FAF701FDDFE799
:10616000164807B0BDE8F04FFAF71ABDA8010020A5
:10617000081D0020B93D0608C93D0608101E002074
:10618000E03D0608A02401200D3E0608693E0608F1
:1061900090220020B01D0020193F0608B41D0020E9
:1061A0008C530020C53E0608281A002000401C46DB
:1061B000E23E0608F73E0608EE3E06081D3F0608CA
:1061C0002DE9F84F002607460C461D4DB046DFF876
:1061D0007890DFF878A02046FCF7B0F9D5F800B049
:1061E00048B921465846F9F7AFF920B92146686801
:1061F000F9F7AAF980B15846FAF7B2FC696811B10B
:106200005046FAF719FDA96811B14846FAF714FD8E
:106210004FF00108FAF7ACFC013610353A2EDAD10E
:106220002046FCF78BF948B9B8F1000F06D1224699
:1062300038460449BDE8F84FFBF7C8BABDE8F88F07
:10624000A4810508453F06083F3F0608393F060878
:1062500070B5224C2378012B00D070BD204B1B68F9
:10626000002BFAD01F4D2B6828465B689847002802
:10627000F3D01D4B1D4E1A68338892889A421BD367
:106280001B490022284609684968EA622A6803FB1C
:1062900001F1D36898473AF0F5FC3388154A013389
:1062A00052683380002AD8D0116893884A69134213
:1062B00018BF1B048B6170BD0E4A00210E4B526843
:1062C0001B782170002AC8D0C3F34003918812685C
:1062D0001B0101FA03F3936170BD00BF8A290120FD
:1062E000DC1B0120E01B01208429012088290120DA
:1062F0007C2901201C1C0120281C0120144B1B7828
:10630000222B144B04D0187900F0010038F09DBE08
:10631000114AD96892F87422013A18BF012289B152
:10632000888810B40C6821695DF8044B08420B4959
:106330000CBF10B201204A800880187900F00100DB
:1063400038F083BE054910B24A800880DBE700BF01
:10635000B12801206C790120A0290120B428012056
:10636000F8B5BB4B1B6813F004022DED048B40F015
:10637000EB801546DFEDB78AB74C13F0200304D04D
:1063800094F8DC3013F0020377D122799FEDB39AB1
:1063900012F0010294F81C1140F08480002967D1AA
:1063A000D4ED487A9FEDAE6ADFEDAE6A67EE867A8D
:1063B00094ED4A7A38EEC77AE8EEA67A84ED497A07
:1063C000C4ED487A63B1012194F83021D4F8E0306B
:1063D0008A4284F81D11C4F82C3118BFC4F8243146
:1063E000A14B1E780D2E0BD1D4ED387A9FED9F7AFC
:1063F0009F4B67EE877AFDEEE77A17EE902A9A8038
:106400009FED940A9B483DF043F9B0EE408A84ED3D
:106410004E0AD4ED4F7A9FED980A78EE677A974846
:1064200084ED4F8A27EE800A3DF032F984ED530A5D
:106430003CF084F802B282EAE273A3EBE2739BB20F
:10644000092B7FD9002AACBF0A380A3005B20D2EBD
:10645000A4F8505161D0242E52D0382E05D1B0EE80
:10646000480A3CF06BF8824B9880BDEC048BF8BD79
:1064700084F81D2184F81C2192E7D4ED3B7AB4F80E
:10648000F030F8EEE77AC4ED387A002B40F09B80CC
:106490009FED729A2279012394F81C1112F00102E7
:1064A0003FF47CAF002900F0868094ED4A8A6E4A62
:1064B00078EEC89A94F81D711678002B49D0012FF8
:1064C00002D0002D40F09980002F40F0B0800D2EBA
:1064D00000F0B280002D00F0A78094F83031012B3D
:1064E00000F2A280B0EE690A6248F0EE698A3DF0DF
:1064F000CFF8B0EE408A84ED4E0A84ED490A88E771
:10650000DFED5F7A94ED490A20EE270A3CF016F899
:10651000574BBDEC048B5880F8BDDFED577A9FEDEB
:10652000580A69EE277A524C28EE800AFDEEE77A87
:1065300017EE903A23803CF001F8E5806080BDECD6
:10654000048BF8BD002582E7434C0125D4ED348A45
:1065500013E70D2E44D09FED3F9A002FBAD094F848
:106560003031002B5DD194ED4E0A002DBCD070EE81
:10657000687A94F83131DFED436A07EE103A77EE2E
:10658000887AB8EEC77AF0EEE77A67EE877AF4EEAB
:10659000E67AF1EE10FA03DD69EE266A86EEA79A36
:1065A000F7EE007A77EEC97A67EEA97AE9EE007A1B
:1065B000B0EE670A98E794ED488A012284ED4A8A92
:1065C00084F81C2173E707EE903ADFED2B6A9FED0C
:1065D0002E7AF8EEE77A86EEA79A89FE479A59E76F
:1065E000D4ED4E7A9FED1B9A9FED250A27EE800A87
:1065F0003BF0A4FF1E4B9880AFE7D4ED387A01231F
:1066000037EEE87A84F81D3137EE087A84ED4B7A5C
:1066100077EEC77A0D2EC4ED4E7AA0D194F81D7195
:10662000E2E7022B7FF456AF94ED4E0A5CE7D4ED1F
:10663000387A94ED4B7AEBE7DFED117A94ED4E0A60
:1066400020EE270A3BF07AFF094B988042E700BF13
:10665000D45A0120000000006C7901209A99993EDB
:10666000CDCC4C3FCDCC4C3EB12801200AD7233CA9
:10667000B4280120C07A01200000C842AC7A012071
:10668000CDCCCC3D00401C466666663F2DE9F84FF8
:10669000C14C2DED028BA36820469847002800F0DE
:1066A000B880B4F90E3004F14805A17D06EE903AA9
:1066B000B4F91030092907EE103AB4F91230F8EEA7
:1066C000E66A07EE903AB8EEC77AF8EEE77AC4EDDC
:1066D000126A84ED137AC4ED147A00F09E80DFF81C
:1066E000E89228461BF07AFEB9F82C30002B40F0D7
:1066F000A080AA4B1B685B0700F1C580D9F8283041
:106700000026D4ED135AB3F9022094ED127A06EE66
:10671000902AA34AD4ED147AF8EEE66A92F800B013
:10672000B3F90420B3F9003075EEE65A06EE902A6C
:1067300006EE103ADFF89482F8EEE66A994FB8EE6A
:10674000C66A994AC4ED135A77EEE67A37EE467A6E
:10675000C4ED147A84ED127AB4F84430B9F800A08C
:1067600007EE903A92F8D233B342B8EEE78A00F0DF
:106770008D80BAF1000F40F0CC8095ED007AD7ED16
:10678000007A87ED007A77EE677A67EE887AC5ED52
:10679000037A0136043508F10C080437032EDBD1E7
:1067A00094ED137ABBF1040FD4ED167A27EE077A35
:1067B000D4ED124A67EEA77A94ED155AD4ED145A27
:1067C000A4EEA47A94ED176AE5EE057AD4ED006A9A
:1067D000A5EEA57AE6EE067AB1EEC70AB1EEE77A43
:1067E00026EE800A84ED180A26EE878A84ED198A3F
:1067F0000CD1DFED6E8A6E4D20EE280A3BF09EFE36
:1068000028EE280AA8803BF099FE2881012384F80D
:106810006830BDEC028BBDE8F88FDFF8AC9104F175
:10682000200128461BF072FDB9F82C30002B3FF4F4
:1068300060AFD9F828C02946DFED5E6A00265E48C1
:10684000ACF102020CF10407B3F5C87F74D0D0EDAF
:10685000007AB8EEE77AD1ED007AE1EC016A77EEE2
:10686000877AFDEEE77AE0EC017A22F8026F974230
:10687000EAD1012B63D0013BA9F82C30474B1B68B0
:106880005B077FF53BAF33F021FC37E7BBF1040F2B
:1068900022D0BAF1000F29D195ED000AD7ED007A88
:1068A00087ED000A70EE677A27EE888A85ED038A05
:1068B000BBF1040F7FF46DAF3BF040FE9FED3F0A4C
:1068C000DFF8ECA028EE000AAAF802003BF036FE42
:1068D000354AAAF806005CE795ED000A3BF02EFE6B
:1068E000334B314A1880BAF1000FD5D095ED000A2C
:1068F00040463CF0CDFED7ED007A2B4A70EE677A29
:1069000085ED000A87ED000A27EE888A85ED038A67
:10691000CEE795ED000A40463CF0BAFED7ED007A8E
:10692000214A70EE677A85ED000A87ED000A67EE6E
:10693000887AC5ED037A2CE7B0EE667A8BE7204AB9
:10694000204FD2F86801B4F80C80C830DFF880E03E
:1069500087FB00BAC017D2E95812C0EBEA10C83161
:10696000C832A0EB0800ACF8040087FB0180C9170F
:10697000C1EBE011ACF8001087FB0217D217C2EB95
:10698000E712ACF80220CEF80A30AEF80E60F9F744
:106990004FFFB9F82C306EE71C24002078560120F8
:1069A000B1280120D87A01209C1E002000007A44E2
:1069B000B428012000000000CC7A01200AD7233C33
:1069C0006C7901201F85EB51E8230020EC23002087
:1069D000C05601202DE9F04FBD4C05462DED048B2E
:1069E00094F878718FB0022F28D110F081FF11F048
:1069F0008BFC2379DA0740F1D0800023B54E98460E
:106A000084F87831B44B1B78002B00F0AD803378DC
:106A1000472B07D104EB8703B04AD3F844339B11CB
:106A200022F8173004EB8808D8F8440380110FB01F
:106A3000BDEC048BBDE8F04F3CF05ABE0123A84AE0
:106A40009F4282F8203000F0838094F87931002B47
:106A500040F0308194F898310193002BCDD0002381
:106A600094F8992184F89831002A40F04D81002D46
:106A700000F00A8394F89A31002B00F02585164621
:106A80009FED988ADFF87092DFF87082DFF870A2CD
:106A90000CE09047032E3FDD013694F89AB109F1DE
:106AA0000409AAEC010A5E4580F2F982072ED8F8A3
:106AB0002C30D4F88021D4BF18F806B05FFA86FBDA
:106AC00089485946002BE4D09047B8F81A2004EBC7
:106AD0004B03F0EE406AB3F8E4319A4200F2DA82F6
:106AE00007EE903AB8F81C30B8EE677A07EE903AA5
:106AF000F8EE677A87FEC70A012303FA0BFBD8F882
:106B00002C301BEA030F03D0D4F80C321B05C1D480
:106B1000032EB6EEE60ABFDCB5EE400AF1EE10FA3F
:106B2000BAD0B9F8003007EE103AB9F80230B8EE32
:106B3000477A07EE903AF8EE677A30EE470A77EE3A
:106B4000C77A20EE080A80EE277A37EE080AA3E714
:106B500012F0D2F802235F4E984684F878315E4BEB
:106B60001B78002B7FF453AFC5F10105F5F7D4FE78
:106B700005443CF091FD04EB8703BA00D3F844339D
:106B8000B0EBA31F01D0830198118542224440F34A
:106B90009A80AD01C2F8445339E7544A0BA9DFF893
:106BA00064C102F1080612F8010F013104EB800301
:106BB000D3ED857AFDEEE77A17EE903AB3F5FA6FEA
:106BC000A8BF4FF4FA63B3F57A7FB8BF4FF47A7376
:106BD0000128A3F57A73C3EBC3134FEA4303ACFB5D
:106BE00003E34FEA9313A3F17F0308BF5B4296428E
:106BF00001F8013CD7D14FF0000C3D484FF0010E99
:106C0000664662468DF834C010F8013F0EFA02F174
:106C1000013204EB83033143D3ED857AFDEEE77A4D
:106C200017EE903AB3F5FA6FA8BF4FF4FA63B3F5D5
:106C30007A7FB8BF4FF47A73A3F57A73C3EBC313AB
:106C40005B00B3F5FA3F02DB4EB24FF0010C082AAD
:106C5000DAD1BCF1000F01D08DF83460254B93F8E8
:106C60007422D3F89812032A7FF4C7AE00293FF4A8
:106C7000C4AE0A7B002A7FF4C0AE01200873D3F8AB
:106C8000A832C3F8A8200BAA03F19001C3F89C20F6
:106C90000922C3F8A42040F20312A3F890201A6935
:106CA000824202D10BA8C3F8A000D2B2186836F015
:106CB000C7FDA2E6D4F8883104F5BE7098470023DA
:106CC00084F87931C6E6013BC2F844339FE600BF41
:106CD0006C790120B128012018240020B42801205B
:106CE0008C53002000007A44E87A0120438505088F
:106CF0004B850508A029012020650120945501201D
:106D0000087B0120D34D6210BE4E94F89B3196F85B
:106D100000C015B1013A84F89921D4F8A802D3B182
:106D2000D4F894E1BEF1000F08BFAE46002840F051
:106D300071829FEDB50A4FF448710246BCF13E0FD7
:106D4000C4F8A8E2A4F8AC1284EDAC0A00F08E837B
:106D5000AE4B187026E0002800F055822A1A4FF634
:106D6000DC709FEDAB7A9042A8BF1046B0F5487F2B
:106D7000B8BF4FF4487007EE900A81B2801AF8EE5F
:106D8000E77AB0FA80F087EE270A4009DFF87CE264
:106D9000BCF13E0FA4F8AC1284EDAC0A8EF80000F2
:106DA00000F02883BCF1270F03D13BF0C7FB994BC0
:106DB0001880DFF890B2DBF80030D80400F11682BA
:106DC00094F8B732022B00F0E582042B00F0B08279
:106DD000012B19D1D4F8BC32EB1A002B14DB44F68A
:106DE00020632B44C4F8BC3294F8EB3253B194F8CE
:106DF000E932052B00F27A83874A02EB43039B8C2E
:106E0000C3F38D03A4F8BA32D4F80C238349AB1A28
:106E10008B4239DC954239D007EE903A804B9FED9A
:106E2000816AF7EE006AF8EE677A93F828309FEDF2
:106E30007E7A9FED7E5A67EE867A06EE103AB4F8B7
:106E4000B822B8EEC66AB4F8BA3277EEE65A9A4279
:106E500037EE467A27EE057AE7EE256A27EE277A9F
:106E600087EE268A40F01C82DFF8DC81B8F900301A
:106E7000B8F902209A4240F03382B8F90430B8F9E8
:106E800006209A4240F01C82C4F80C53684B9D4285
:106E900000F2A48111F0E0F8814610F0A5FC2379FE
:106EA00094F828A313F0010396F800E000F0CE80D8
:106EB00000285B4BB8BF40425B7E5FFA80F84345D9
:106EC00040F29D81BAF1010F94F82A1302D00029F3
:106ED00040F0E18194F82B33B9F1000918BF4FF06D
:106EE0000109002B40F07C82BAF1010F14BF484623
:106EF00049F00100002800F00382474A82F8793205
:106F00004C4B82F838005878002874D094F82C0341
:106F1000002870D194F82D0300286CD194F82E032A
:106F2000002868D144480078CDE900E118F004FB5E
:106F3000404BDDE900E100285DD1DBF80000C2062E
:106F400000F1D682187941004B29A8BF4B2180451A
:106F5000C9B280F0EF828845C0F0D1823749DFEDB9
:106F6000387A91ED0B7AB0EEC77AB4EEE77AF1EEAB
:106F700010FA40F1C48291ED057AB0EEC77AB4EE12
:106F8000E77AF1EE10FA40F1BA8291ED117AB0EEA3
:106F9000C77AB4EEE77AF1EE10FA40F1B082D4F895
:106FA0003C1309B9C4F83C535988B8F14A0F4FF45F
:106FB0007A7C88BF4908D4E9CF030CFB01F11B1A86
:106FC0002B448B4202D9012184F82C13002800F0B5
:106FD000A282BEF11F0F07D14FF47A72B3FBF2F316
:106FE0000C4AD38001239380BAF1010F00F02A826A
:106FF0000123984604E5BEF11F0FF5D1054B002291
:107000005A60F1E7B128012000409C4490620120C1
:1070100000247449B42801208C53002090D0030030
:1070200094550120BD378636000080430000803B28
:10703000404B4C007C55012094670120A057002054
:107040000000C84278560120A80401200121BF4A4F
:10705000BF4882F87912016884F8293391F8361014
:1070600084F82B33003918BF0121BEF11F0F82F8BD
:10707000381001D1B74A5360BAF1020F00F005820F
:10708000002384F82833B3E7B34E94F89B3196F885
:1070900000C042E607EE902AB8EE670A2CE5D4F865
:1070A0000832DFF8E8E213F48073DEF800C00593DD
:1070B00094F89B3103F0010A18BF4FF0000A84F8DE
:1070C00010A2BBF1000F00F00F82B8F812200CF5EF
:1070D0009670A249002609EE102AB8F81A20DFF8A7
:1070E000B0920092B8EE499AB8F81C2009F148080D
:1070F000DFED9B8A0292CA789FED9A8A0490CDF8C0
:107100000CC0CDE906735F46DDF814B00595154651
:10711000CDE9081E944B03EB8600D0ED007ABAF15E
:10712000000F14D0BCEEE77A17EE103A98B2009B2D
:1071300098420CD3029B984209D8049BC8F80030AF
:10714000002D00F08180032E40DCAA4607E06DB3DD
:10715000032E3BDC032E00F04681F0EE497A013627
:10716000C7FEE87A08F10408C7FE887ABE42E9EC57
:10717000017ACFD1059DDDE90673DDE9081EDEF851
:107180000000BAF1000F63D00A69C860002A00F05D
:107190008881821A086A904267DA7448012281F86D
:1071A0002520026822F0040202605EE0BBF1000FBD
:1071B0000CD1D8F80000039B181A0028C0F20D81EA
:1071C000032E03DC00239A4684F81032F0B21AF042
:1071D00085FF07EE900AF8EE677AC0E75F4B9A7872
:1071E000002A7FF457AE01229A7053E6D4F8083291
:1071F000D9073FF5E5AD042010F01CFAE0E50123C6
:1072000084F829335EE69FED5A0A18464FF4487118
:107210001A46BBE5AEEB00024FF6DC709FED557AE7
:107220009042A8BF1046B0F5487FB8BF4FF44870F1
:1072300007EE900A81B2101AF8EEE77AB0FA80F001
:1072400087EE270A400979E5BBF1000F87D0BDE73B
:10725000464ECA680861801A326842F00402326001
:107260004A689042C8BF81F825A03B4E96F800C0FE
:10727000BCF1280F09D1D4ED887ADFF8D880FDEE73
:10728000E77A17EE902AA8F8062094F8A422013293
:1072900084F8A42241E594F8293384F82B331BE6C3
:1072A00007EE903A344884EDC58AB8EE670A3CF0A0
:1072B000FFF9BCEEC00A10EE103AA4F8B832D3E5DC
:1072C00007EE903A2D4884EDC98AB8EEE70A3CF003
:1072D000EFF9BDEEC00A10EE103AA8F80630D3E57B
:1072E00007EE903A264884EDC78AB8EEE70A3CF0EC
:1072F000DFF9BDEEC00A10EE103AA8F80230BCE586
:107300002048CDF800E00078CDE9023118F014F9FA
:10731000DDF800E0DDE9023100287FF4EEAD0C4835
:10732000019B006890F83600003818BF0120E4E5A2
:10733000F5F7F2FAD4F80833C01A134B98427FF7E6
:1073400063AD0023A4F8B8325EE500BF8C53002083
:1073500088550120B4280120B1280120205901209E
:1073600000A00C4500803B44087B0120745901209B
:1073700000409C44002474497C7C01208C7C0120CA
:10738000847C01209467012060E31600141C012016
:10739000807B0120754B764ADB7B04EB8303D3EDC6
:1073A000847AFDEEE77A17EE903A1BB2B3F5FA6FE6
:1073B000A8BF4FF4FA63B3F57A7FB8BF4FF47A737E
:1073C000A3F57A73C3EB8323A2FB0323C3F38F13C9
:1073D000A4F8B832A4F8BA3216E5D9ED007ABEE6C0
:1073E0001846002389E56348038807EE903AF8EED3
:1073F000677AB4E6DFF89C81A8F804005E48009341
:1074000080FB02C0D217C2EBA0025C48A0FB0101C6
:10741000C908A8F8061047F6FF718A42A8BF0A46B5
:10742000A8F800203BF08AF894F8B612B4F8B42219
:10743000009BA8F8080000293AD0A8F80C20A8F86A
:107440000E30B6E44E4B1B6893F869304345BFF4E9
:10745000CFAD0223002284F828334A4B5A60DA6108
:107460005A6343F8482F5A609A60C1E5DFF82CC18F
:10747000DFF82081ACFB0ECEDFF824C14FEA5E1EA0
:107480008CF80000A8F802E0B6E7036893F86C30C7
:10749000002B3FF4ADADD4F80C325B053FF5A8AD41
:1074A000EEE5394E0861306840F00400306071E666
:1074B000642101FB02F2354981FB02011144D2171C
:1074C000C2EB612292B2B8E7D4F80832DFF8D4E018
:1074D00083F4807A94F89B31DEF80020CAF3002A06
:1074E00003EA0A0A84F810A2294948E6002389E43D
:1074F000B9F1000F7FF426AD00297FF423ADD4F855
:107500003C1329B1D4F840335B1A2B44C4F8403300
:107510000023C4F83C33BEF11F0F7FF465AD4FF478
:107520007A72D4F84033B3FBF2F31A4AD3800023C3
:10753000938059E5DFED187A94EDCC7AB4EEE77AD2
:10754000F1EE10FABFF60AAD94EDCD7AB4EEE77A1B
:10755000F1EE10FABFF602AD94EDCE7AB4EEE77A12
:10756000F1EE10FAFFF6F7ACF8E400BF94550120F5
:10757000D34D6210D056012067666666CDCCCCCC68
:1075800088550120A057002074590120030820804D
:1075900020590120B42801209A99193E1F85EB51EA
:1075A00090620120141C0120C24BDB79022B40F0B9
:1075B00021812DE9F047C04CB4F85033B4F8522380
:1075C0009A422DED028B82B000F00981A4F852336B
:1075D0000126B4F8543313F4006300F0078194F8E3
:1075E0005873002F00F00A82DFF8008394ED4E8A72
:1075F00098F80050B4F9D0A34A2D00F04C81492DE1
:1076000012D10023B4F864C3B4F866131A46B4F870
:107610000E016CF30F036AF30F0260F31F4361F373
:107620001F42A649C1E90032B4F9D223DFF8C09263
:10763000AAEB0203DFEDA26ADFEDA27A07EE103AB1
:1076400099F81C30B8EEC77AA3F10503B3FA83F3B7
:10765000B4EEE67A5B0967EE277AF1EE10FA84F869
:10766000683300F20B819FED987A77EE877AF0EE1F
:10767000E78A4A2DA4F86623C4EDDB7AC4EDE08ADC
:1076800000F0CF80002E63D0D4EDF57A4C2D94ED30
:10769000F60AF8EE677A8D4A9FED8D7A916830EEA2
:1076A000670AC4EDD77A67EE876AC4EDF67AD2ED41
:1076B000037AB4F80C3120EE270AC4F87013C4ED35
:1076C000D86AB4F8E21384EDDD0AA4F8643300F05C
:1076D0004581A1B307EE903A94F8F933B1EE006A10
:1076E000F8EEE77A77EEC07AF0EEE77A67EE877A1F
:1076F00007EE103A774BB8EEC77AC7EE876A36EED8
:10770000867AC6EE077AC4EDF07AD3ED017AF5EE0B
:10771000C07AF1EE10FA40F388819FED6F6AB0EE07
:10772000007A67EE867AC7FEC77A042F05D1B0EEDD
:107730000C7AC6FEC76A76EEA77AC4EDE17A482DC8
:1077400000F057814A2D03D13AF0F8FE5B4B1880C8
:10775000F5F7E2F899F81C30052B40F0CB8094F84F
:10776000DC3013F0010200F0DF80D4F8FC235B4929
:10777000821A8A4240F3D68203F0020394F8102161
:10778000C4F8FC03002B15BF0023012301210021B5
:10779000032A84F8003494F902348CBF4FF0FF328E
:1077A00001221344022B1A46A8BF0222012B22EA0F
:1077B000E27284F8022400F3BD82002384F80134CD
:1077C00084F8C813082F3FD8DFE817F05901680282
:1077D000CB019301F3013201300033004B01B4F8C7
:1077E0005433002613F400637FF4F9AE1F4684F887
:1077F0005833F9E63A4B03F1780102E00633994237
:107800000ED01A780A2AF9D19878DA789042FFF4E3
:10781000D0AE5A79002A7FF4CCAE06339942F0D12B
:107820007047264BA3F808A05A812BE7304616F084
:107830000BF92C4BD4EDEC7A93ED187AB4EEE77A91
:10784000F1EE10FA00F3E58098F800304A2B29D0C9
:10785000242B09D1DFED1B7A94EDE20A20EE270AF2
:107860003AF06CFE154B188015F0A4FF304602B0BC
:10787000BDEC028BBDE8F04715F0AABCDFED1A6A3B
:10788000B4EEE67AF1EE10FA7FF7F1AE9FED0E7AE4
:1078900077EEC77AEBE6B0EE480A3AF04FFE074BB8
:1078A0009880C1E694EDE40A3AF048FE034BD88094
:1078B000DAE700BFD05601206C790120B4280120FE
:1078C0000000E1C4CDCCCC3D0000B443A8040120AD
:1078D0000AD7233C847D01203EC3AE393F420F00CE
:1078E000DC5601201C2400200000E144B1280120C6
:1078F000D85A0120002384F8C833082FA4D801A344
:1079000053F827F07F7A0108157D0108637B010891
:10791000F37A0108B37B0108317A01082D78010858
:1079200033780108637A010884F8C823082F8BD8BC
:1079300001A353F827F000BF7F7A01081D7D0108DD
:10794000637B0108F37A0108B37B0108317A0108EF
:107950002D78010833780108637A0108FDEEC07ABA
:10796000C44D17EE900A288100293FF4F1AE07EECE
:10797000903A94F8F933F1EE005ADFEDBF6AF8EE71
:10798000E77A77EEC07AF0EEE77A67EE877A07EE6D
:10799000103ABA4BB8EEC77A87EE876A36EE255AA8
:1079A00066EE267A85EE857AFDEEE77A84EDF07A4A
:1079B00093ED017A17EE903AB5EEC07A6B81F1EE55
:1079C00010FA40F3D181DFEDAE5AF0EE007A27EEE7
:1079D000257A87FE677A67EE267AFDEEE77A17EE5C
:1079E000903A1BB2042FAB8100F0C28184EDE17AA2
:1079F000AEE63AF0A3FD9F4B9880A9E601233846F6
:107A000084F8583315F0E4FB15F0D4FE94F858735D
:107A1000EAE59C4A0720136843F0805313600FF097
:107A200009FE002384F858330EE7DFED977A7CE6F1
:107A300094F804349FED907A07EE903AF8EEE77AE6
:107A400067EE877AB4EEE78AF1EE10FA05D50622E2
:107A5000002384F8582384F8A833304615F0F4FF47
:107A6000F2E6884A0120136843F0805313600FF058
:107A7000E1FD002384F8A83384F85833E4E6237941
:107A8000DA0704D4814B1B7A002B00F08A81D4EDF5
:107A9000E27AC8FE277AC4EDE27A002E3FF4D4AE33
:107AA000B4F8E033F6EE005AD4EDD86A06EE103A98
:107AB00094F8EF3366EEA56AB4F8F423B8EE466A9C
:107AC000012B07EE102A84EDE48AC6FEC66AC4EDD7
:107AD000E96A00F0AD81B8EEC77ADFED676A022B84
:107AE00027EE267A00F09D8177EE877AC4EDE37A5F
:107AF000AAE6B7EE007AD4EDEB7AF4EEC77AF1EEAF
:107B000010FA05D59FED627A77EE877AC4EDEB7AAD
:107B1000F3EE0E7AF4EEE78AF1EE10FA0DD5B4F832
:107B2000DC3307EE903A0423F8EE677A84F8583392
:107B30000023C4EDE77A84F8A833B4F8E23394ED77
:107B4000DD7A07EE903A534B84EDE67AF8EEE77A69
:107B5000B4EEE77AF1EE10FA4CBF012200225A741B
:107B600072E694EDE37A4B4BB4EEC87A1A7CF1EEF0
:107B700010FACCBF01230023934200F0E080B4F858
:107B8000EA33D4EDD86A07EE903A002384EDE47A24
:107B9000F8EEE77AC4F89433F4EEE76AF1EE10FAFF
:107BA00002DD032384F85833D4F87433C4F89833CF
:107BB0004AE6384AB7EE007AD4EDEB7AF4EEC77AAB
:107BC000F1EE10FA05D59FED327A77EE877AC4EDA3
:107BD000EB7AB4F8E23394EDE67A07EE903A537C10
:107BE000F8EEE77AF4EEC77AF1EE10FACCBF012294
:107BF00000229A4207D177EEC77ADFED256AA7EE19
:107C0000A67A84EDE67AF7EE006AD4EDF17A9FED7C
:107C1000226AB0EE007A76EEE76AE6EE867A37EE12
:107C2000677AC4EDF17A84EDEF7A002E3FF40CAE62
:107C3000B4F8DC33B6EE007AD4EDD85A06EE903ABA
:107C400094EDE96AF8EE666AF4EEC65A26EE877A93
:107C5000C4EDE76AF1EE10FA67EE277AC4EDE87A30
:107C60003FF6F2AD0522002384F8582384F8A833A8
:107C7000EAE500BFB42801200000C842847D01204D
:107C80003EC3AE397459012000000000285601207F
:107C90000AD7233CA80401200AD7A33BF1EE047ABB
:107CA00094EDD87AB4EEE77AF1EE10FA7DD4B4F818
:107CB000EA3307EE903AF8EEE77AB4EEE77AF1EEBF
:107CC00010FA00F19180D4EDE37AB4EEE78A002354
:107CD0000022D4F87413C4F8AC33F1EE10FAC4F8EF
:107CE000A033C4F89C33C4F8C433C4F894334FF0C1
:107CF0007E5384F8A823C4F8BC33C4F8C0334CBF07
:107D000001230023514AC4F898131374022384F802
:107D1000583399E594F8DC30DB07BFD4072384F8A7
:107D2000593391E594F800343BB994F8011481F08B
:107D3000010145E5012384F80134002140E5002BD1
:107D400047D0B4F8F0339FED427A07EE903AF8EE60
:107D5000E77A67EE877A94EDE47AC4EDE57A77EE18
:107D6000277AC4EDE47A1FE79FED3A7A002339E6DB
:107D7000F0EE0C7A0192C6FE677A77EE877AC4ED50
:107D8000E17AF4F7C9FD99F81C30019A052B44D12A
:107D900094F8DC3013F001017FF4E7AC84F8C813E9
:107DA00008E70023C4F888334EE594F80434DFED87
:107DB0002A6A07EE903AF8EEE77A67EEA67AB4EE12
:107DC000E78AF1EE10FA7FF572AF082384F8583392
:107DD0003AE5B4F8F2339FED217A07EE903AF8EEE7
:107DE000E77A67EE877AB6E7B4F8F433B6EE007A4E
:107DF000DFED195A06EE903A9FED196A67EE877A21
:107E0000F8EEE66AB0EE487AC4EDE97AA6EEA57A15
:107E1000C7FE067AC4EDE37A57E7002384F8C83337
:107E2000C8E678EE077AC7FE877AC4EDE37A0BE5F9
:107E3000B4F8DE339FED087A07EE903AF8EEE77A71
:107E400067EE877AC4EDE37AFEE400BFA804012060
:107E50000AD7233C000000000000C8420AD723BC18
:107E600000007A442DE9F843964B1B685A0701D469
:107E7000BDE8F883DFF890820446934F98F800300D
:107E8000BD7C372B01D1914B1D80914E33691A78FF
:107E9000012A07D0042D00F20A81DFE805F092B331
:107EA0009EA8180093F904308A4A03EB430302EBBF
:107EB000431393F85520202A00F0BD800123864803
:107EC00086494FF47A7280F820300B7073E0D6F850
:107ED000C83083489847002800F0B3808149D6F81D
:107EE000CC30081D9847D6F8D890B9F1000F40F370
:107EF000B78007EE909A9FED7C0ADFED7C0AF8EEE2
:107F0000E77A27EE800A3AF089FAF7EE007A7849A4
:107F10009FED787A77EEC07A774A087867EE877AAD
:107F200092ED007A002800F0A48077EEC77AC6EDC3
:107F3000347A98F80030372B17D107EE909A9FEDDE
:107F40006F0ADFF88881F8EEE77A27EE800A3AF0C8
:107F5000F5FAD6F8D43096ED340AA8F80200A8F85D
:107F600004303AF0EBFAA8F8060096F8AC30002B93
:107F70004DD105234FF47A78BB741F46564B01222E
:107F800006EB850583F82020F4F7C6FCD5F82034ED
:107F9000001B984206EB870388BFC5F82004D3F87E
:107FA00020043BF0A5FBB8F1000F3FF461AF42465F
:107FB0000A2AB8BF0A22524B1B681B681A61BDE827
:107FC000F883D6F8B83046489847002839D00123BE
:107FD0004FF47A78BB741F46D0E7D6F8C0304048DB
:107FE00098470323B6F8B080BB741F46C6E7D6F89F
:107FF000C4303B48984720B304234FF47A78BB74CD
:108000001F46BBE7D6F8BC3035489847C8B10223B5
:10801000BB7406EB8505F4F77FFC001BD5F8203414
:10802000834218D2C5F82004D6F828043BF060FB40
:108030004FF47A78BBE75B699B691B047FF52AAF35
:108040003CE7BB7C0121254A022B1170E1D01F4681
:108050004FF47A7892E7D6F828043BF049FBE7E73B
:10806000234B1B78002B7FF464AF0023C6F8D0307D
:108070005FE7DFF898C077EE877A224BB3F800E02D
:10808000BCF80030C2ED007A01339BB29E45ACF8DB
:108090000030EAD807EE103A0123ACF80000B8EE41
:1080A000C77A0B70C7EE876AC2ED006ADDE7D6F8C3
:1080B000B4300B4898470023B6F8AE80BB741F4617
:1080C0005CE700BFD45A0120A8040120B428012095
:1080D0006C7901206C1D01208C5300201824002095
:1080E0007C790120407A012008942537B1DC423E9A
:1080F0000C680120D048874A086801200AD7233C31
:10810000885300200E680120B1280120106801204A
:10811000F8B5384C2368002B57D00A2801D00D2819
:1081200051D1354D95F838340BB1F8F721FD334E68
:10813000232130463AF049FF08B1801B20602368B4
:10814000002273B902B12360F8F7DEFC95F83834E9
:10815000F3B12B48BDE8F840F8F702BD01220B4609
:10816000EFE7591E705C2028F8D092B90022254C08
:10817000224FF2543B26013E0DD13146224B9C4208
:1081800012D2E3682068984795F83934002BDBD188
:10819000F8BD2360EAE721683846FDF7CDF80146CF
:1081A0000028EBD11034E6E795F8383423B11749AD
:1081B0001748F9F7F9F9C7E71648F8F7D1FC0F485F
:1081C000F8F7EEFCC0E7FF2BE2D8A0F120025E2A10
:1081D000DED80BB92028DBD05A1C2260074AD054C5
:1081E000054B93F83834002BD2D0BDE8F840F8F7AF
:1081F00001BD00BF985A01206C79012096590120D9
:108200005E290608A481050844850508593F06082B
:10821000753F06087B3F060838B50546F8F784FC2D
:108220000A4B002418680CF0A9F9F8F76DFC084B0C
:1082300083F8394483F8384417F06CF925B12046A7
:10824000BDE83840FDF795B838BD00BFE4620120B5
:108250006C79012038B5074C074DAC4203D3074B6E
:1082600001221A7038BDA288D4E902103AF03EFE0D
:108270001C34F2E72887060804900608AC50012059
:108280002B4B30B583B09A790190BAB393F8242080
:10829000DFED286A07EE902ADB79274CF8EEE77AC3
:1082A000A3F10203254904F58D62B3FA83F386EE48
:1082B000A77A0D785B0984F86C3482ED007ADDB121
:1082C0001F4BDDED017AB3F84634F8EE677ADFED47
:1082D0001D0A00EE103A67EEA00AB8EE400AF6F763
:1082E000B5FC04F58E63002103EBC5021960083369
:1082F00003ED010A9A42F9D103B030BD124A126867
:108300001401F9D593F82420DFED0A6A07EE902ACC
:10831000DB79094AF8EEE77A981E02F58D6143424F
:1083200086EEA77A434182F86C3481ED007AE3E768
:108330000C240120555555408C530020A0070020E7
:108340006C790120BD37863578560120894B1B7822
:10835000002B00F0E680884B2DE9F04F2DED028BCD
:1083600093F804A183B0BAF1010F40F09380834BDE
:108370001C78082CA446A8BF4FF0080C002C61D034
:108380007F480021DFED7F7A40F6FF7E00F58D63A8
:10839000794A90F86C748B46D3ED006A7A4D66EE9C
:1083A000A76A0091CDF804A0938927B992F81E809E
:1083B000B8F1010F09D913F4706F4FEA2329C3F301
:1083C000032802D019F0010F69D0734500F08980AD
:1083D000C3F308085B0A08FA03F31FFA83F8B8F13D
:1083E000000F00F09280694E9BB206EB5808B8FB74
:1083F000F3F35FFA81F8444507D9DFF8A08198F8D4
:108400000080B8F12D0F08BF2B804FF6FF76B342E6
:1084100040F0888001311432043002358C45C3D1DC
:10842000BBF1000F0ED0DDED007A594BB8EE677A44
:1084300007EE90BAF8EE677A27EE267AC7EE276A3B
:10844000C3ED006ADFF85C919FED528A89ED008AE6
:10845000E4B159ED138A09F10408474F0025A9F149
:10846000440AFB890AEBC5000135143700EE103AC7
:10847000B8EEC00A20EE280A3BF01AF9AC4288FE9A
:10848000408AA8EC010A89ED008AEAD102233A4A1F
:1084900082F8043103B0BDEC028BBDE8F08F3E4E94
:1084A00001EB81095FFA83FA06EB5808324E98F81F
:1084B000B08308EB4909B8F1010F06EB4909019EA9
:1084C000A9F80EA006FA08F692F81E9049EA0609E5
:1084D00082F81E9040D192F81F80C2459AD9D37776
:1084E00098E7CBB29C422CD92C4B1B782D2B30D04B
:1084F0000023DFED2B7AD381937F43F00103937741
:108500000BF1010BC0ED007A84E7CBB29C4281D91C
:10851000224B1B782D2B7FF47DAF4FF6FF732B8002
:1085200078E77047009E07EE903A1E449BB2F8EE43
:10853000E77AD381937F67EEA67A009643F0010332
:10854000DDE70023DFED167AD381937F43F001034B
:10855000D5E700232B80CBE7B8F1000F7FF45AAFAB
:1085600007EE90AA009BF8EEE77A5344009367EE7B
:10857000A67AC5E7A8010020081D0020A00700205A
:108580008C53002000007042B4280120C02709004D
:108590003C580020FFFF7F7FA4810508B1280120FF
:1085A0000000000040580020F0B41A4C1A4BA4FB05
:1085B000024290F858505209A3FB0243DB0803EB38
:1085C0008303A2EB43030268DCB2A54220D000EB98
:1085D000830C476800269B00DCF80850521BDCF82F
:1085E00030507D1B4560CCF80860CCF8306080F8D6
:1085F00058400344013202609A6801329A6029B9F6
:108600004268013242601A6B01321A63F0BC704753
:108610009B00EEE71F85EB51CDCCCCCC38B5094D96
:108620002B7963B100242B6820465B6B13B10134B6
:10863000984708B9002038BD2B799C42F3D301201C
:1086400038BD00BF2C2500200B4B1A7E12B90B4BF6
:1086500098797047094A906800B97047084940F610
:10866000B83C0968091A614503DD00219079197643
:1086700070470020F1E700BFA80401202C2500204E
:10868000141C01202DE9F04FDFF834921F46531ED1
:1086900083B016460546D9F80040142B00F2CD8071
:1086A000DFE803F05959595959CB0B0B0B0BCB0B86
:1086B0000B0BCBCBCBCBCB0B0B004FF47A734FF028
:1086C0000A0A0193012F4CD0002F41D1774A784BF1
:1086D00014781878631C03F00303834238D01370B6
:1086E00004EB4403DFF8D4814FF47A724FEA440973
:1086F00008EBC30383F80CA09A60C1B11822A5F15E
:10870000FF0002FB0482B0FA80F00C32400905E061
:1087100038B9013702F8013F8F4208D0AF42034613
:10872000F6D1013733468F4202F8013FF6D1FFF709
:1087300075FF002800F0A98009EB0401012342F233
:108740001070C90008F8013041443AF099FF4860C0
:1087500003B0BDE8F08F574B012F4FF0010A019392
:10876000B2D1554A537C012B03D0022B00F09880E4
:10877000002799F8040008B34D4B1821A5F1FF0E0E
:108780001A780C23BEFA8EFE11FB02314B4B4FEAD6
:108790005E1E1944002307E0BEF1000F08D101332B
:1087A00001F801CF984209D0DAB2F446AA42F3D1D7
:1087B0000133B446984201F801CFF5D142F2283096
:1087C000F4F72EFC4FF47A70F4F72AFC97B3236A7F
:1087D00003B1984799F80430EBB1A5F1FF084FF0C9
:1087E000000BB8FA88F858464FEA5818E26B9047E1
:1087F0005D45A26A314603D0B8F1000F00D1414671
:10880000584690470BF1010399F804205FFA83FB67
:1088100093455846EAD3A36903B19847E36A98475A
:108820008FB90AF1FF3A1AF0FF0A18D04FF47A70A4
:10883000F4F7F6FBE3699847C9E74FF47A734FF012
:10884000010A01933EE70AF1FF3AE36998471AF0FB
:10885000FF0A04D04FF47A70F4F7E2FBB7E701980F
:10886000F4F7DEFB99F80420002A3FF471AF104CB6
:108870000D2118231148247813FB041300211844F8
:1088800003B0BDE8F04F3AF089BB09EB0403DB000D
:1088900008EB030208F80300506003B0BDE8F08F56
:1088A0009778083F18BF012763E700BF151D012017
:1088B000141D0120A08601000C240120B41C0120FD
:1088C0002C2500202DE9F041114C25780DB9BDE88B
:1088D000F08180460F4616461C4693B1012BF6D117
:1088E0000C4B98792F2EF2D80028F0D13AF008FFDF
:1088F0000028ECD12346324639464046BDE8F041D7
:10890000C0E6FFF7A1FE80F00100C0B2EAE700BFB9
:10891000506301202C25002010B5437B044682685B
:10892000581C6073D154627B237B934200D802B9F8
:1089300010BD2368D4E9010198470023637310BD7B
:10894000427B42B1036810B50446D0E90101984763
:108950000023637310BD70472DE9F04F056887B0A1
:108960002E78012E0CD0022E03D0002007B0BDE8D7
:10897000F08F2B6A002BF8D12CF088FC0120F5E752
:1089800095F904508DF817206B1C0279EDD0032D5A
:10899000EBDCDFF8309205EB45038C464FEA4508E7
:1089A00009EB431359690029DFD093F855002028BB
:1089B00040F08B8093F85400012800F086807C4FB3
:1089C00083F854603E6803E03B689B1B192B6ED80C
:1089D0008C6914F40044F7D1A84453002120009678
:1089E0004FEA4818039340230DF1170109EB080BD8
:1089F00008F1140A62464FEA45088BF85500CA444C
:108A00008BF856300123CBF838105046CBF858403D
:108A10000399ABF83E300A23CBF8484033F064F9B1
:108A2000002840F09280BBF83E309BB2FF2B40F212
:108A30008F80DBF81410FF235E48ABF83C304B68A6
:108A40005D4A0340039803431A434A6008EB050458
:108A5000234609EB441B34461E4605E0BBF83E3076
:108A60009BB2002B00F0878022460A2150462DF051
:108A7000EBFC50BBDBF83810DBF8140011F8012BCD
:108A8000BBF83C308262CBF83810013BBBF83E109B
:108A90009BB20139ABF83C3089B2ABF83E10BBF861
:108AA0003E1089B2002BD9D10029D7D017E0454418
:108AB0002021002209EB4515AB6D85F854200B43AE
:108AC000AB6585F8551085F856203C4A138801336C
:108AD0009BB2138049E73968091B0A2925D88369A5
:108AE00013F08003F7D0BBF83E309BB2FF2B0BD9BD
:108AF00043683049039A0B402F4913431943FF231E
:108B0000ABF83C304160A9E7BBF83E30039A9BB21A
:108B10004168ABF83C30DBB242EA0343254A1140DE
:108B20000B4343F00073436098E7194608EB0503D5
:108B3000202009EB43139A6D83F8541002439A6581
:108B400083F8550083F85610BFE78BF85440BCE714
:108B5000BBF83E30DBF814109BB2039A1548ABF813
:108B60003C30DBB242EA03434A680240134343F01D
:108B700000734B606AE733462646504631461C4632
:108B800033F0C6F9034600289FD1DBF8142009EB27
:108B9000441920240A48D4615168014001205160E1
:108BA0008BF8554089F854308BF85630DEE600BF1C
:108BB000A4280120009C00FC0000FF01CA5A0120EB
:108BC00000E800FE6C1D01202DE9F04F066885B01D
:108BD0003578012D09D0022D03D1346A002C00F024
:108BE0008C80002005B0BDE8F08F96F90460741CFD
:108BF000F7D0032EF5DC9C46DFF8389206EB4603EF
:108C000096464FEA460809EB43135A69002AE8D012
:108C100093F855400079202C40F0828093F854401E
:108C2000012C7DD07B4C83F85450256804E02368E8
:108C30005B1B192B00F29380936913F40043F6D168
:108C4000B0441F4643000A464FEA481822204021FC
:108C5000039308F1140B09EB080A00950A23CB448F
:108C60008AF85500CAF838E04FEA46088AF85610E4
:108C70005846CAF858700399AAF83EC0CAF8487016
:108C800033F09AF9002840F09980BAF83E309BB250
:108C9000FF2B40F29680DAF81420FF235E48AAF8F2
:108CA0003C3053685D4903400398034319435160C6
:108CB00008EB060A09EB4A1703E023685B1B0A2B43
:108CC00021D8916911F00401F7D0526ABB6B1A7078
:108CD000FB8FBA8F013B013A9BB292B2FB87BB6B11
:108CE000BA870133BB63FB8F9BB203B1F2B1FB8F39
:108CF0009BB2002B78D07A69E3E741F080012CF039
:108D0000EFFA01206EE74644202209EB4616B36DC8
:108D100086F854101343B36586F8552086F856102C
:108D20003F4A138801339BB213805AE7796903E005
:108D30002268521B0A2A31D88B6913F08003F7D0BE
:108D4000FB8F9BB2FF2B1AD94B68364A1340039A0C
:108D50001343354A1A43FF23BB874A60C7E708EB32
:108D600006032020002109EB43139A6D83F8541069
:108D700002439A6583F8550083F85610D0E7FB8FBD
:108D8000039A9BB22748BB87DBB242EA03434A6897
:108D90000240134343F000734B60A8E71A4608EB08
:108DA0000603202009EB4313996D83F854200143F7
:108DB000996583F8550083F85620B1E78AF8547016
:108DC000AEE7BAF83E3003999BB2DAF814201248A5
:108DD000AAF83C30DBB241EA0343516801400B433F
:108DE00012491943516063E72946584633F090F819
:108DF000002895D17B6920210D4C09EB4A19D961D6
:108E00005A6822405A6087F8551089F8540087F84C
:108E1000560076E7A4280120009800FC0024FF817A
:108E2000CA5A0120009C00FC0000FF0100240082BF
:108E300000E800FE6C1D01202DE9F043046883B0BA
:108E40002578012D08D0022D02D1246A002C6FD084
:108E5000002003B0BDE8F0839E4694F904305C1C0A
:108E6000F6D0032BF4DC1646DFF8088103EB43024F
:108E700084465F0008EB421250690028E8D092F85F
:108E80005540202CE4D1846914F40044E0D192F8D8
:108E900054000128DCD030489CF804C0D0F8009081
:108EA000222082F8545082F8550040202B4D82F841
:108EB00056002B489465A2F83EE01064D08F96636C
:108EC00080B29564FF2842D8B2F83EE04FF00076B9
:108ED0001FFA8EFEFD184FEA4C070A46CDF80090A7
:108EE00008EB4510192339460546A0F83CE014303C
:108EF00033F062F810BB6A693743DFF87CE05368EF
:108F000095F83CC003EA0E031649AE6C3B4343EAB6
:108F10000C431943144B9E42516085F8540003D012
:108F2000124B9E4218BFF42413682343136003E0DE
:108F300041F080012CF0D4F901208AE70C4A00218D
:108F4000138885F8541001339BB2138080E74FF0EB
:108F5000FF0E4FF08076BDE7A42801202D200408E5
:108F60000000FFFF00240080A1210408093F04083D
:108F7000CA5A01206C1D0120009800FCF8B5224E51
:108F80003378012B10D1042894BF002301235BB94F
:108F90001E4C0D461E4F04EB4000E188C7F84834D4
:108FA00042892078638800B1F8BD07EE903A6423C7
:108FB0009FED187AF8EEE77A03FB02F29FED166A4E
:108FC00003FB012167EE877A07EE102A06EE901A5E
:108FD000B8EEC77AF8EEE66A67EE877A96ED047A1D
:108FE000B8EE477A87EEA60A27EE067A20EE070A41
:108FF00039F0A4FAB268A3881060084A12681344D2
:109000002B44BB60F8BD00BFE8670120D467012096
:109010006C7901200AD7233CCA269B3E141C0120F0
:10902000036810B59B68044698470122FF236273CA
:10903000A37310BD036810B504461B68984701214F
:10904000236820469B689847E37B0133E37310BD98
:109050002DE9F041069F0D460446164638469846CF
:1090600037F0C4FE2844E672A072387850B10697F3
:1090700029462568204643463246AC69A446BDE8E9
:10908000F0416047BDE8F08103689B6A184700BF64
:1090900003685B6D03B11847704700BF0368DB6C62
:1090A00003B11847704700BF0B46002110B5C173CC
:1090B000044642749A6C0360017302B190472368BE
:1090C000012120469B689847FF2123680122A17354
:1090D000DB6C62731BB12046BDE81040184710BD21
:1090E0000E4B012210B482400D4C1B7854F8200026
:1090F000134071B1003B18BF012338B183F0010365
:10910000828801681B0102FA03F38B615DF8044B4E
:109110007047B3FA83F35B09EFE700BF281C012017
:109120001C1C01202DE9F0411E4C40F2DC57DFF8F9
:109130008C8023681C4D1B6B98471C4900231C4ADC
:109140008978A360A4F80530032998BF1746194C05
:10915000F3F7E2FB0646D8F80430C3F30803EBB993
:10916000EFF31183D3B94FF0E020296882692B68AF
:109170009942FAD123689A42F7D80F4B4FF47A708C
:10918000D3F800C000FB0CF39B1AB3FBFCF300FB0D
:109190000130831B9F42DED8BDE8F081F3F792FBDC
:1091A000F7E700BF2C250020141C01200C2401200F
:1091B000FCA60700A8280120A024012000ED00E063
:1091C0001B4B70B55B7906460D46012B18D1194B28
:1091D0001B68ABB1184B0846B3F94C44F9F7AEF92C
:1091E00098B92846F6F752FA00F543730446B3F5EA
:1091F000C36F0AD930461149BDE87040F8F7E6BAA6
:109200000F48BDE87040F7F7D1BC0E48F7F7CEFC29
:109210000D48F7F7A5FCF7F787FC0C4B18680BF027
:10922000ADF9FFF77FFF2046BDE87040F4F79CBD25
:109230004C2C0120DC1B01206C790120B53F060875
:10924000883F0608CD3F0608D23A0608E4620120AE
:1092500010B5044C23681B6998470023A371A360D1
:1092600010BD00BF2C25002010B5074C63791BB141
:109270002368DB68984700B910BD044B01221B68C6
:10928000A271A36010BD00BF2C250020141C01207A
:10929000F8B5114D002452272E1D013415F8010B8D
:1092A000F1F78AFB00222021E4B218B18771C47162
:1092B000F0F71AFE16F8010BF1F77EFB4FF0530C96
:1092C0000022402120B180F806C0C471F0F70CFEE6
:1092D000042CE2D1F8BD00BFBC7D0120C3B25E2BDF
:1092E00005D8044B03EB8003D3F8B803704702485A
:1092F000704700BFA481050878FA050803681B6859
:10930000184700BF03682DE9F0415F6A1FB13B4673
:10931000BDE8F041184704460D46164600E02368B4
:109320009B68204698478642F9D8002E08DD2E44D7
:109330002368204615F8011B1B689847AE42F7D1F9
:10934000BDE8F08103685B68184700BF03689B684D
:10935000184700BF0368DB68184700BF03685B69F4
:10936000184700BF03689B6A03B11847704700BFE6
:109370000368DB6A03B11847704700BF03689B6A44
:1093800070B504460D46164603B198473246294645
:109390002046FFF7B7FF2368DB6A1BB12046BDE814
:1093A0007040184770BD00BF70B504460E461546A4
:1093B000236820469B689847A842F9D32A4631463D
:1093C0002046BDE87040D9E72DE9F04FB74D8FB08A
:1093D00095F8393413B10FB0BDE8F08FB44E33684F
:1093E0005B05F8D5D5F884360446B24AC31A9342D1
:1093F00066DC95F88836002BEDD095F88C369F0703
:10940000E9D195F8942642B1D5F8980610B1AA4949
:10941000FFF7B4FF002385F8943695F8DC76002F2B
:1094200040F0A98095F87039002B4ED195F83B2675
:10943000002A40F06881A14BD5F87409196895F8A5
:1094400078393BB19E4BD5F87C799F4202D1884256
:10945000C0F06D8195F8A4299A4BB3FBF2F3D5F8CF
:109460006C2913449C42B6D395F89436C5F86C49E0
:10947000002BB0D195F8AF392B4493F8A849E007F9
:1094800000F1A783A10700F11C83620700F1D882D5
:10949000230700F1A382E10600F15082A20600F149
:1094A0003582630600F1118495F8AF3995F8A42947
:1094B0000133B3FBF2F102FB113385F8AF398AE7D0
:1094C00019F0ACF8C5F8844693E77F4BC8267F496E
:1094D00006A8A3F13F02CDE904237D4B7D4A00930A
:1094E0007D4B85F84466F5F729FFDDF810902921BA
:1094F000EA2209F1010306A8049389F80070049B8D
:1095000003F1010CCDF810C01970049B591C049193
:109510001A70049B5A1C04921E700B2637F066FCCE
:1095200000F1010806A90498424639F0DFFC049ACC
:1095300002EB08030133049302F80870049B013E18
:1095400003F1010204921F70F8D1049B012204A8C8
:10955000991804911E70049B991804911A70049B29
:10956000A3EB090389F800302AF0F2FD85F8706951
:10957000C5F86C492FE795F8DD66002E40F0848130
:10958000D5F84037002B00F0B980DFF85C81A8F5F2
:10959000227908F1680A63E0012A00F04881052F6A
:1095A00050D9437800F1060EC11985F86439438813
:1095B000A5F860398388C02B00F29F8300224B44BA
:1095C0004648A5F862290122C5F85899C5F85C39C2
:1095D00085F86829A3EB000BA1EB0E0285F869C999
:1095E0005A45C0F28881BBF1000F40F055813C4BD9
:1095F0003C4AC5F85C09D869002302F11001C5F89E
:10960000589985F86839C5F85039069306ABC5F8FE
:1096100048A9C5F84C2909F007F9013000F0658325
:10962000069B0BB100209847D5F84839C5F848A9E2
:10963000C5F84C3995F89436002B00F00A810123C7
:1096400085F8DD3601373E44EFF31183502282F373
:109650001288D5F84027964248DADBB283F31188A6
:10966000AB1993F8E076012FECD9711C6B1893F8C5
:10967000E036C3F3411203F00F0C032A85F84427A8
:1096800000F0EC8013F0100308EB010084D195F892
:109690006829002AD6D095F86929013202F00F0214
:1096A000624500F0E98085F86839CBE76C790120E4
:1096B00078560120BFC62D0008800120141C01200F
:1096C000EC820120A0860100F07F0120D8FA050875
:1096D00083500120CCFA0508C0FA0508C47D01209A
:1096E000A8040120B48201204C800120002295F8BA
:1096F000DD66DBB2C5F8402783F3118885F8DC66A8
:10970000C5F86C4967E6C64A4FF4327185F83B36B6
:1097100006A8A2F13A03A5F84816CDE90632C14BD6
:10972000C5F844362AF014FDC5F86C4953E695F89F
:109730003816002940F0B880D5F89479002F3FF40E
:1097400089AED7E9002191423FF484AED5F89C3927
:10975000D5F8A029E31A93427FF77CAEB04B95F879
:109760009829B14985F84A26A3F13802C5F844166C
:109770004FF4E47195F899E9A5F8481685F84BE699
:10978000CDE90623D7E90080404500F07483914677
:10979000A3F1060C8045ACEB090A98F8006000F0D4
:1097A00021834346002203E0984202F1010203D0E4
:1097B00013F8011B8E42F7D093B2012B00F2AF8257
:1097C0005FFA8AFA9A4580F00E83804500F0538351
:1097D000E145DFD3BEF1000F07D195F84A3663F0BB
:1097E0007F0385F84A36D7E90080804500F047833B
:1097F000069B06A88D4E9B1B85F845362AF0A8FCD3
:1098000095F894264AB1D5F8980618B106F1570193
:10981000FFF7B4FD002385F8943695F89939C5F81B
:109820009C490133C5F86C4985F89939D3E5022F75
:109830003FF408AF8378A5F860394378FF2B56D101
:10984000042F7FF6FFAEB0F8033000F1050EC1190A
:10985000B1E630F0A5FB85F8DD06F3E6744BC5F8FC
:1098600048390133C5F84C39002385F84837A3F54A
:109870002023C5F85039DDE600F1010EC119D5F8F5
:109880005C39D5F85809A5E695F89436002B00F018
:10989000B88295F8DD6631E771465A4639F026FB05
:1098A000D5F858095844A2E695F8981985F838264D
:1098B000013185F899295F4A82FB01020A4452115D
:1098C000C2EB8212891AA3F58D62A3F5517385F854
:1098D00098191F4695F83A16C5F8943995F839360F
:1098E000C5F83C2603FB0121C5F840162BE700F123
:1098F000030EC1195FE67146039239F0F7FAD5F805
:109900005839039A1344C5F858399BE6444B4FF431
:109910009961B5F8502106A807933B3B120AA5F8B8
:10992000441606930721B5F9503185F8472685F886
:10993000461685F848362AF00BFCB2E5B5F80C213E
:1099400024206426D5F8E83000FB02F2D5F8E410B4
:109950001BBA334F323209BAC5F84B36B5F80E315F
:10996000C5F84716002103EB830395ED490A0797D5
:109970002E3F5B00B2FBF6F2C2F3072060F3070153
:1099800062F30F21C3F307229BB262F3174163F323
:109990001F6141F2C813A5F844360223C5F84F16DB
:1099A00085F8463638F0CAFD234A034606A80697CE
:1099B0009342A8BF134623EAE373B3FBF6F303F520
:1099C0007A73C3F3072285F8543695F8103185F879
:1099D000532685F855362AF0BBFB5FE5C823104AAD
:1099E000A5F844362123079285F84636B5F8543356
:1099F0005F0540F11582114B393A18680692C5F897
:109A00004706069B0021094A581C069006A81970B3
:109A1000069B9B1A85F845362AF09AFB3BE500BF6A
